:100000000C9445160C9476160C9476160C94761671
:100010000C9476160C9476160C9476160C94761630
:100020000C9476160C9476160C9476160C94761620
:100030000C9476160C9447590C9476160C947616FC
:100040000C9476160C943FC40C9476160C94761689
:100050000C9476160C9476160C9472760C94FD58CB
:100060000C9476160C94B04B0C9476160C94761671
:100070000C9476160C9476160C9476160C947616D0
:100080000C9476160C9476160C9476160C947616C0
:100090000C9476160C9476160C9476160C947616B0
:1000A0000C9476160C9476160C9476160C947616A0
:1000B0000C9476160C9476160C9476160C94761690
:1000C0000C9476160C9476160C9476160C94761680
:1000D0000C9476160C9476160C9462580C94235853
:1000E0000C9476168631A331D431F13106322F3299
:1000F0009C320233AB33F3370138FA3721382538D5
:100100003F389A3C5438A038C738EE3817396D3923
:100110007E398F39A039B139C2399A3CA53B9A3C16
:10012000B03B203C263C463CF2B0F5B0E4B0E8B031
:10013000EEB02CB1F9B0FDB003B107B10BB111B104
:1001400015B119B12CB11FB123B127B18CB691B63D
:1001500096B6A0B6AAB623B7B4B6BCB6C4B6CEB6E9
:10016000D8B6E2B6F1B6FBB623B705B70FB719B7E5
:10017000084AD73B3BCE016E84BCBFFDC12F3D6C0E
:1001800074319ABD56833DDA3D00C77F11BED9E474
:10019000BB4C3E916BAAAABE000000803F05A84C54
:1001A000CDB2D44EB93836A9020C50B99186880820
:1001B0003CA6AAAA2ABE000000803F004E414E493C
:1001C0004E495459494E46CDCCCC3D0AD7233C1715
:1001D000B7D13877CC2B329595E6241FB14F0A0062
:1001E0000020410000C84200401C4620BCBE4CCA52
:1001F0001B0E5AAEC59D74434F4D4D554E4943415C
:1002000054494F4E0044525952554E004552524F98
:10021000525300494E464F004543484F0047322F46
:1002200047332062616420706172616D657465722C
:10023000730A00206F6620004D424C20473239205F
:10024000706F696E74200059206F7574206F66207E
:1002500072616E67652028312D35292E0A005820DD
:100260006F7574206F662072616E67652028312D6E
:1002700035292E0A004D6573682070726F62696EB1
:100280006720646F6E652E0A005374617274206D6E
:100290006573682070726F62696E67207769746831
:1002A0002022473239205331222066697273742E1E
:1002B0000A004732380A47323920533200537461FA
:1002C00074653A20004D65736820626564206C6532
:1002D00076656C696E6720686173206E6F2064615B
:1002E00074612E0A0053206F7574206F662072614E
:1002F0006E67652028302D35292E0A004D657368FC
:1003000020706F696E742063616E6E6F7420626519
:10031000207265736F6C7665640A00456E642066B2
:10032000696C65206C6973740A00426567696E20A8
:1003300066696C65206C6973740A00286E6F2066AC
:10034000696C6529005344207072696E74696E6728
:10035000206279746520004E6F74205344207072BF
:10036000696E74696E670A0043757272656E7420F7
:1003700066696C653A20002569730025696D202542
:100380006973002569682025696D2025697300253A
:100390006964202569682025696D20256973002519
:1003A000697920256964202569682025696D2025E3
:1003B0006973005072696E742074696D653A20002B
:1003C0006F6E2E0A006F66662E0A00473236204492
:1003D000656275672000180213020C020502F7011E
:1003E0006F66660044454255473A004B494C4C45C0
:1003F000442E20004D3131332053006F6B002C20F0
:10040000002C2000544845524D414C5F50524F54EF
:10041000454354494F4E004155544F5245504F5259
:10042000545F53445F53544154555300454D455216
:1004300047454E43595F5041525345520043415343
:10044000455F4C494748545F4252494748544E45DE
:10045000535300544F47474C455F4C49474854530A
:1004600000534F4654574152455F504F5745520035
:100470004255494C445F50455243454E54004C450B
:1004800056454C494E475F44415441005A5F5052D3
:100490004F4245004155544F4C4556454C00505233
:1004A000494E545F4A4F420050524F4752455353B2
:1004B000004155544F5245504F52545F54454D5092
:1004C00000564F4C554D45545249430045455052F6
:1004D0004F4D0053455249414C5F584F4E5F584F66
:1004E0004646004649524D574152455F4E414D45A3
:1004F0003A4D61726C696E20312E312E39202847B9
:1005000069746875622920534F555243455F434FC4
:1005100044455F55524C3A68747470733A2F2F6794
:1005200069746875622E636F6D2F4D61726C696EB0
:100530004669726D776172652F4D61726C696E20CC
:1005400050524F544F434F4C5F56455253494F4EB4
:100550003A312E30204D414348494E455F54595061
:10056000453A3344205072696E7465722045585480
:1005700052554445525F434F554E543A31205555DC
:1005800049443A63656465326132662D34316132C3
:100590002D343734382D396231322D633535633699
:1005A000326633363766660A002F2F20002054004B
:1005B000205200416363656C65726174696F6E3AC5
:1005C0002050005741524E494E4721204C6F772012
:1005D0005A204A65726B206D6179206C65616420D8
:1005E000746F20756E77616E7465642070617573C9
:1005F00065732E0A00546F6F206661722066726FF9
:100600006D207265666572656E636520706F696ED8
:10061000740A0020466C6F773A20000001363726B6
:10062000032BFFFFFF3C3D382AFFFFFFFF2E303E2C
:1006300012FFFFFFFFFFFFFF0809FF2C071A1C181E
:10064000FFFFFF08440A2C4324221E20643A0020A6
:10065000693A0020703A00496E76616C69642065E1
:10066000787472756465720A0043290A0061626CCD
:10067000656420286D696E2074656D702000436F7D
:100680006C6420657874727564657320617265208E
:100690000020643A0020693A0020703A004E6F2032
:1006A00063617365206C696768740A004545505240
:1006B0004F4D204F4B0A00205A004475616C204575
:1006C0006E6473746F702041646A7573746D656EC7
:1006D0007420286D6D293A20003F4B2076616C759F
:1006E00065206F7574206F662072616E67652028C3
:1006F000302D3130292E0A00416476616E63652009
:100700004B3D004163746976652045787472756469
:1007100065723A2000496E76616C69642065787470
:1007200072756465720A0043616E6E6F7420656E47
:10073000746572207375626469723A2000473931BA
:100740000A4731205A2D302E30320A4739300053B3
:1007500070656369616C204D656E753A205A20445E
:100760006F776E20302E310A004739310A47312029
:100770005A2D302E30320A47393000537065636984
:10078000616C204D656E753A205A20446F776E205B
:10079000302E30320A004739310A4731205A2B3087
:1007A0002E30320A473930005370656369616C201E
:1007B0004D656E753A205A20557020302E30320A21
:1007C000004739310A4731205A2B302E310A473938
:1007D00030005370656369616C204D656E753A2019
:1007E0005A20557020302E310A00473239205332BA
:1007F000005370656369616C204D656E753A204EDB
:10080000657874204D65736820506F696E740A00B6
:10081000473239205331005370656369616C204D54
:10082000656E753A205374617274204D657368204B
:100830004C6576656C696E670A004D313430205323
:100840003630005370656369616C204D656E753A92
:100850002050726568656174204265640A004D35F8
:100860003031005370656369616C204D656E753A77
:10087000205265616420454550524F4D0A004D3568
:100880003030005370656369616C204D656E753A58
:10089000205361766520454550524F4D0A004D3337
:1008A000303320452D312053383020433820553106
:1008B000005370656369616C204D656E753A204127
:1008C00075746F2054756E6520486F74626564207E
:1008D0005069640A004D31303620533137380A4DA3
:1008E00033303320453020533234302043382055C4
:1008F00031005370656369616C204D656E753A20F7
:100900004175746F2054756E6520486F74656E6410
:10091000205049440A003C5370656369616C5F4D27
:10092000656E753E003C5370656369616C5F4D6533
:100930006E753E002F002F002F002F2E2E0A002F45
:100940002E2E002F2E2E003C5370656369616C5F64
:100950004D656E753E0A003C5370656369616C209D
:100960004D656E753E003C5370656369616C204D4A
:10097000656E753E003C5265616420454550524F9E
:100980004D3E003C5265616420454550524F4D3EFE
:10099000003C4175746F2054756E6520486F746219
:1009A0006564205049443E003C4175746F20547585
:1009B0006E6520486F74626564205049443E003C77
:1009C0004175746F2054756E6520486F74656E6450
:1009D000205049443E003C4175746F2054756E654B
:1009E00020486F74656E64205049443E003C457851
:1009F00069743E003C457869743E003C53617665FD
:100A000020454550524F4D3E003C53617665204590
:100A10004550524F4D3E003C4E657874204D6573F5
:100A20006820506F696E743E003C4E657874204DAE
:100A300065736820506F696E743E003C5374617238
:100A400074204D657368204C6576656C696E673EF1
:100A5000003C5374617274204D657368204C657658
:100A6000656C696E673E003C507265686561742014
:100A70006265643E003C5072656865617420626521
:100A8000643E003C5A20446F776E20302E313E0089
:100A90003C5A20446F776E20302E313E003C5A2065
:100AA000446F776E20302E30323E003C5A20446F27
:100AB000776E20302E30323E003C5A205570203068
:100AC0002E30323E003C5A20557020302E30323EBF
:100AD000003C5A20557020302E313E003C5A2055A3
:100AE0007020302E313E0056313136004A333320EB
:100AF000004D3530300A4D3432302053310A473101
:100B0000205A313020463234300A473120583020C4
:100B10005930204636303030004A3232004A3232C4
:100B2000004731205A3520463234300A47312058A8
:100B3000313930205932302046363030300A473192
:100B4000205A302046323430004731205A35204672
:100B50003234300A47312058313930205931393058
:100B60002046363030300A4731205A302046323461
:100B700030004731205A3520463234300A47312080
:100B800058313930205932302046363030300A471B
:100B900031205A302046323430004739310A47314B
:100BA000205A313020463234300A4739300A473231
:100BB000380A4732390A473120583230205932300A
:100BC0002046363030300A4731205A302046323401
:100BD00030004A3032004A3132004731205A313039
:100BE000004F4B004731205A313000473930004721
:100BF00031204525694635303000473120452D30BC
:100C00002E314625690047312045302E3146256971
:100C1000004731205A2569462569004731205A2D61
:100C2000302E31462569004731205A302E31462575
:100C30006900473120592569462569004731205907
:100C40002D302E314625690047312059302E31464E
:100C5000256900473120582569462569004731201C
:100C6000582D302E314625690047312058302E311D
:100C7000462569004739310047323800473238206D
:100C80005A00473238205900473238205800413244
:100C9000305620004731205A3130004A3034004A63
:100CA0003231004A3230004B494C4C45442E200032
:100CB0004A303400454E4400464E20004A3032004F
:100CC0003939393A393939004D0048004137562011
:100CD00000413656202D2D2D004A30320041365627
:100CE00020005A3A2000593A2000583A2000413555
:100CF00056004134562000413356200041325620E0
:100D000000413156200041305620004D3834004A11
:100D10003136004A3138004739310A4731205A31DB
:100D20003020463234300A473930004A3134004AE4
:100D30003030004A3031004A31300024F4D4305091
:100D4000C38E20C2A24017828B7011127A910D813E
:100D50006CD90AA861E108C7586607615143061EAD
:100D60004B5D05C145A7041A411104093D98037163
:100D70003931034036DB0265339102D430540280AE
:100D80002E1D02632CEE01752AC501B028A00110AA
:100D90002781018F2564012B244B01E0223401AC13
:100DA000211F018D200D01801FFC00841EED009786
:100DB0001DDF00B81CD200E61BC600201BBC00646F
:100DC0001AB200B219A8000A19A0006A189900D135
:100DD00017910040178B00B516840031167E00B3C2
:100DE0001579003A157300C7146F0058146A00EEA5
:100DF0001366008813630025135E00C7125B006C46
:100E000012570015125400C111510070114F0021EA
:100E1000114B00D61049008D1047004610440002C7
:100E2000104200C00F4000800F3E00420F3C000601
:100E30000F3B00CB0E3800930E37005C0E350027B9
:100E40000E3400F30D3200C10D3100900D30006002
:100E50000D2E00320D2D00050D2C00D90C2B00AEEF
:100E60000C2900850C29005C0C2700350C27000E8E
:100E70000C2600E80B2400C40B2400A00B23007DEB
:100E80000B23005A0B2100390B2100180B2000F80E
:100E90000A1F00D90A1E00BB0A1E009D0A1D008001
:100EA0000A1D00630A1C00470A1B002C0A1B0011C4
:100EB0000A1A00F7091A00DD091900C4091900AB64
:100EC000091900920917007B091800630917004CE3
:100ED00009160036091600200916000A091500F542
:100EE000081500E0081400CC081400B8081400A489
:100EF000081400900813007D0812006B08130058B6
:100F000008120046081200340811002308110012CC
:100F100008110001081100F0071000E0071000D0D0
:100F2000071000C0071000B0070F00A107100091C4
:100F3000070E0083070F0074070F0065070E0057A8
:100F4000070E0049070E003B070D002E070E00207C
:100F5000070D0013070D0006070D00F9060C00ED44
:100F6000060D00E0060C00D4060C00C8060C00BC00
:100F7000060C00B0060C00A4060B0099060C008DB0
:100F8000060B0082060B0077060B006C060B006157
:100F9000060A0057060B004C060A0042060A0038F3
:100FA000060A002E060A0024060A001A060A001085
:100FB00006090007060A00FD050900F4050900EB13
:100FC000050900E2050900D9050900D0050900C797
:100FD000050900BE050900B5050800AD050800A516
:100FE0000509009C050800940508008C050800848C
:100FF0000508007C050800740508006C05070065FD
:101000000508005D050700560508004E0507004766
:101010000507004005080038050700310507002ACC
:10102000050700230507001C050600160507000F2D
:101030000507000805060002050700FB040600F589
:10104000040700EE040600E8040600E2040700DBE3
:10105000040600D5040600CF040600C9040600C338
:10106000040600BD040600B7040600B1040500AC88
:10107000040600A6040600A00405009B04060095D3
:10108000040500900406008A04050085040500801C
:101090000406007A04050075040500700405006B61
:1010A00004050066040500610405005C04050057A2
:1010B000040500520405004D0405004804050043E2
:1010C0000405003E0404003A040500350405003020
:1010D0000404002C04050027040400230405001E5A
:1010E0000404001A04040016040500110404000D91
:1010F000040400090405000404040000040400FCC6
:10110000030400F8030400F4030400F0030400ECFB
:10111000030400E8030400E4030400E0030400DC2B
:10112000030400D8030400D4030400D0030400CC5B
:10113000030400C8030300C503030024F404D920FA
:101140001BC40C5C0E9804C4095F0265077101F4AE
:1011500005F900FB04B30048048700C10369005887
:1011600003550003034500BE023A008402310053D8
:10117000022A002902250004022000E4011C00C804
:10118000011900AF011700980114008401130071C8
:101190000110006101100051010E0043010D0036E5
:1011A000010B002B010B0020010B00150109000CA5
:1011B00001090003010800FB000800F3000800EB30
:1011C000000700E4000600DE000600D8000600D29A
:1011D000000600CC000500C7000500C2000500BDE8
:1011E000000400B9000400B5000400B1000400AD23
:1011F000000400A9000400A5000300A20003009F52
:101200000004009B00030098000300950002009377
:10121000000300900003008D0002008B0003008893
:101220000002008600020084000300810002007FAB
:101230000002007D0002007B0002007900020077BE
:1012400000010076000200740002007200010071CB
:101250000002006F0002006D0001006C0002006AD5
:1012600000010069000200670001006600010065DE
:1012700000010064000200620001006100010060E2
:101280000001005F0002005D0001005C0001005BE6
:101290000001005A000100590001005800010057E8
:1012A00000010056000100550001005400010053E8
:1012B00000000053000100520001005100010050E5
:1012C0000001004F0001004E0000004E0001004DE3
:1012D0000001004C0001004B0000004B0001004ADF
:1012E00000010049000100480000004800010047DB
:1012F00000010046000000460001004500000045D6
:1013000000010044000100430000004300010042CE
:1013100000000042000100410000004100010040C7
:101320000001003F0000003F0001003E0000003EC1
:101330000001003D0000003D0001003C0000003CB9
:101340000000003C0001003B0000003B0001003AAF
:101350000000003A000100390000003900010038A7
:10136000000000380000003800010037000000379E
:101370000001003600000036000000360001003594
:10138000000000350000003500010034000000348A
:10139000000000340001003300000033000000337F
:1013A0000001003200000032000000320001003174
:1013B000000000310000003100010030000000306A
:1013C000000000300001002F0000002F0000002F5F
:1013D0000000002F0001002E0000002E0000002E53
:1013E0000001002D0000002D0000002D0000002D48
:1013F0000001002C0000002C0000002C0000002C3C
:101400000001002B0000002B0000002B0000002B2F
:101410000001002A0000002A0000002A0000002A23
:101420000001002900000029000000290000002917
:10143000000000290001002800000028000000280A
:1014400000000028000000280001002700000027FD
:1014500000000027000000270000002700010026F0
:1014600000000026000000260000002600000026E4
:1014700000010025000000250000002500000025D7
:1014800000000025000000250001002400000024C9
:1014900000000024000000240000002400010023BC
:1014A00000000023000000230000002300000023B0
:1014B00000000023000000230001002200000022A1
:1014C0000000002200000022000000220000002294
:1014D0000001002100000021000000210000002187
:1014E0000000002100000021000000210001002078
:1014F000000000200000002000000020000000206C
:101500000000002000000020000000200001001F5B
:101510000000001F0000001F0000001F0000001F4F
:101520000000001F0000001F0001001E0000001E40
:101530000000001E0000001E000000232C0000B868
:10154000220000561800003A0F0000B8080000B151
:10155000040000710200003E010000696E206D6F02
:1015600076655F746F282920666565645F76616CB7
:10157000756520666F722058593A002C2065793DB8
:101580000029202D3E202865783D002C2073793DD0
:101590000020436F6E6E656374696E6720776974AF
:1015A0006820766572746963616C206C696E652071
:1015B0002873783D002C2065793D0029202D3E20A0
:1015C0002865783D002C2073793D0020436F6E6EB6
:1015D000656374696E67207769746820686F7269E3
:1015E0007A6F6E74616C206C696E65202873783D2B
:1015F000003F53706563696669656420582C592003
:10160000636F6F7264696E617465206F7574206FAB
:101610006620626F756E64732E0A003F285229653A
:10162000706561742076616C7565206E6F742070D2
:101630006C61757369626C653B206D7573742062B3
:1016400065206174206C6561737420312E0A003F3F
:101650002852296570656174206D75737420626508
:1016600020737065636966696564207768656E20BC
:101670006E6F74207573696E6720616E204C4344F1
:101680002E0A003F537065636966696564206E6F5A
:101690007A7A6C652074656D7065726174757265B7
:1016A000206E6F7420706C61757369626C652E0AB0
:1016B000003F5370656369666965642066696C61A3
:1016C0006D656E742073697A65206E6F7420706C1E
:1016D00061757369626C652E0A003F5370656369BA
:1016E00066696564207072696D65206C656E6774EB
:1016F00068206E6F7420706C61757369626C652E02
:101700000A003F5072696D65206C656E67746820D1
:101710006D757374206265207370656369666965B1
:1017200064207768656E206E6F74207573696E67CC
:1017300020616E204C43442E0A003F53706563695C
:1017400066696564206E6F7A7A6C652073697A6564
:10175000206E6F7420706C61757369626C652E0AFF
:10176000003F5370656369666965642052657472F1
:10177000616374696F6E204D756C7469706C696516
:1017800072206E6F7420706C61757369626C652E67
:101790000A003F52657472616374696F6E204D7503
:1017A0006C7469706C696572206D75737420626504
:1017B000207370656369666965642E0A003F537023
:1017C00065636966696564206C6179657220686526
:1017D00069676874206E6F7420706C6175736962DC
:1017E0006C652E0A003F5370656369666965642005
:1017F0006265642074656D706572617475726520D0
:101800006E6F7420706C61757369626C652028342A
:10181000302D31343043292E0A0047323620636F91
:101820006D6D616E6420737461727465642E2057EF
:10183000616974696E6720666F722068656174659E
:10184000722873292E0A00024A3135004A313200CB
:101850004A3137002020506C616E6E6572427566A9
:1018600066657242797465733A2000204672656538
:10187000204D656D6F72793A2000436F6D70696C11
:1018800065643A2044656320313320323031380AB0
:1018900000207C20417574686F723A20286461765C
:1018A000696472616D69726F2C20666F7220416E7F
:1018B000796375626963206933204D656761290A20
:1018C00000323031382D31322D313300204C6173EC
:1018D0007420557064617465643A2000312E312E95
:1018E000390A004D61726C696E0020536F6674771F
:1018F0006172652052657365740A002057617463D4
:1019000068646F672052657365740A002042726FC5
:10191000776E206F75742052657365740A002045D8
:10192000787465726E616C2052657365740A00503C
:101930006F77657255700A0073746172740A004D96
:101940003234004D3233202573006175746F256980
:101950002E67006572726F722077726974696E67A4
:1019600020746F2066696C650A00205A3A0020597D
:101970003A0020583A00656E6473746F7073206883
:1019800069743A2000446F6E6520736176696E67F2
:101990002066696C652E0A004D32390020746F6F25
:1019A000206C6F6E6720657874727573696F6E2036
:1019B00070726576656E7465640A0020636F6C648E
:1019C00020657874727573696F6E207072657665C4
:1019D0006E7465640A00454550524F4D2064617431
:1019E0006173697A65206572726F722E0A00290A26
:1019F000002062797465733B206372632000536535
:101A00007474696E67732053746F72656420280064
:101A1000290A002062797465733B20637263200099
:101A20002073746F7265642073657474696E677374
:101A300020726574726965766564202800202863C9
:101A4000616C63756C6174656429210A0020213D15
:101A50002000454550524F4D20435243206D69733D
:101A60006D61746368202D202873746F726564291A
:101A700020002053697A653A2000496E6465783AFF
:101A80002000204D61726C696E3D563535290A0083
:101A900028454550524F4D3D00454550524F4D2031
:101AA00076657273696F6E206D69736D61746368BA
:101AB00020001000C90210012C0140012201700118
:101AC0001801B0010E01F00104015002FA00B00249
:101AD000F0003003E600D003DC009004D200700573
:101AE000C800A006BE000008B400B009AA00D00BD0
:101AF000A000600E960060118C0000158200201975
:101B00007800C01D6E00A0226400B0275A00902CFF
:101B1000500000314600E0343C0010383200903A6A
:101B20002800603C1E00A03D1400803E0A00203FBB
:101B300000002CFFFFFFFFFF0001010101016265B2
:101B4000640A002C2073797374656D2073746F7050
:101B500070656421204865617465725F49443A206C
:101B6000004265642068656174696E67206661691A
:101B70006C65640048656174696E67206661696CB4
:101B800065640045312048656174696E672066614F
:101B9000696C65640048656174696E672066616997
:101BA0006C65640070012C0190012701B0012201D5
:101BB000C0011D01F00118011002130130020E01D5
:101BC0006002090190020401C002FF000003FA0054
:101BD0004003F5008003F000D003EB002004E60092
:101BE0007004E100E004DC004005D700C005D2002D
:101BF0004006CD00D006C8008007C3003008BE00F4
:101C0000F008B900C009B400B00AAF00B00BAA00D8
:101C1000D00CA500000EA000500F9B00C010960035
:101C20005012910000148C00C0158700B01782007C
:101C3000B0197D00D01B7800001E730040206E009C
:101C400090226900F024640040275F0090295A0028
:101C5000E02B5500102E500020304B001032460073
:101C6000E033410090353C001037370070383200C7
:101C7000A0392D00B03A2800A03B2300603C1E0094
:101C8000103D1900903D1400103E0F00703E0A00F8
:101C9000C03E0500003F0000403FFBFF803FF6FFD5
:101CA000C03FF1FF453120544845524D414C205230
:101CB000554E415741590042454420544845524DE4
:101CC000414C2052554E4157415900546865726D40
:101CD000616C2052756E61776179004531204572E3
:101CE000723A204D415854454D50004572723A2089
:101CF0004D415854454D5020424544004D415854A3
:101D0000454D50207472696767657265640045319E
:101D1000204572723A204D494E54454D500045724F
:101D2000723A204D494E54454D5020424544004D95
:101D3000494E54454D5020747269676765726564F9
:101D4000004D383420582059205A204500202F00BB
:101D50002042403A0020403A006F70656E20666174
:101D6000696C65642C2046696C653A200043616E9D
:101D70006E6F74206F70656E207375626469722077
:101D8000004A3035004A3233004739310A473120A2
:101D90005A2D313020463234300A4739300053440E
:101DA0002063617264206F6B0A006F70656E526F02
:101DB0006F74206661696C65640A00766F6C756D7E
:101DC000652E696E6974206661696C65640A0045F8
:101DD00072726F723A00534420696E6974206661B2
:101DE000696C0A006563686F3A00205A3A0020590E
:101DF0003A0020436F756E7420583A0020453A002F
:101E0000205A3A0020593A00583A003A004361708B
:101E10003A00205A00205900580020204D61783A9D
:101E20002000205A00205900580020204D696E3AA9
:101E300020004F6E20004F666600536F6674206569
:101E40006E6473746F70733A20004B6420002364D7
:101E50006566696E652044454641554C545F004BAC
:101E600069200023646566696E65204445464155D6
:101E70004C545F004B70200023646566696E6520DA
:101E800044454641554C545F0050494420417574C7
:101E90006F74756E652066696E697368656421206C
:101EA00050757420746865206C617374204B702CBD
:101EB000204B6920616E64204B6420636F6E7374E5
:101EC000616E74732066726F6D2062656C6F77202F
:101ED000696E746F20436F6E6669677572617469AD
:101EE0006F6E2E680A00504944204175746F7475F6
:101EF0006E65206661696C6564212074696D656F2B
:101F000075740A00453120544845524D414C2052C9
:101F1000554E415741590042454420544845524D81
:101F2000414C2052554E4157415900546865726DDD
:101F3000616C2052756E617761790045312048658A
:101F40006174696E67206661696C656400426564EE
:101F50002068656174696E67206661696C656400FC
:101F600048656174696E67206661696C65640050DC
:101F70004944204175746F74756E65206661696CA3
:101F80006564212054656D70657261747572652099
:101F9000746F6F20686967680A00204B643A2000FC
:101FA000204B693A2000204B703A20000A20436CF5
:101FB000617373696320504944200A002054753AC4
:101FC0002000204B753A2000206D61783A200020D7
:101FD0006D696E3A200020643A20002062696173C6
:101FE0003A2000504944204175746F74756E652025
:101FF0006661696C65642120426164206578747251
:1020000075646572206E756D6265720A0050494490
:10201000204175746F74756E652073746172740AF3
:10202000004F66660A004661646520486569676816
:10203000742000426564204C6576656C696E67208B
:10204000004661696C656420746F20656E61626C26
:102050006520426564204C6576656C696E670A0090
:102060004D65736820426564204C6576656C20641C
:102070006174613A0A004D65736820706F696E740F
:102080002063616E6E6F74206265207265736F6C81
:102090007665640A004D34323120696E636F727266
:1020A00065637420706172616D657465722075730B
:1020B0006167650A00656E7175657565696E672093
:1020C00022004B494C4C45442E20005072696E74DE
:1020D00065722073746F7070656420647565207418
:1020E0006F206572726F72732E2046697820746853
:1020F00065206572726F7220616E64207573652051
:102100004D39393920746F20726573746172742E81
:10211000202854656D7065726174757265206973ED
:102120002072657365742E20536574206974206174
:10213000667465722072657374617274696E672962
:102140000A004E6F20436865636B73756D20776975
:102150007468206C696E65206E756D6265722C20E6
:102160004C617374204C696E653A20004E6F2043B9
:102170006865636B73756D2077697468206C696E30
:1021800065206E756D6265722C204C617374204CF5
:10219000696E653A2000636865636B73756D206DC9
:1021A00069736D617463682C204C617374204C6991
:1021B0006E653A20004C696E65204E756D626572E1
:1021C000206973206E6F74204C617374204C696EAB
:1021D00065204E756D6265722B312C204C617374D5
:1021E000204C696E653A20004D313130004D33315D
:1021F0000053442072656164206572726F720A0038
:10220000446F6E65207072696E74696E67206669CE
:102210006C650A007C3C3E5E2B3D3F2F5B5D3B2C9A
:102220002A225C00627573793A2070617573656467
:1022300020666F7220696E7075740A00627573791A
:102240003A2070617573656420666F7220757365DE
:10225000720A00627573793A2070726F63657373E6
:10226000696E670A004A3135004B494C4C45442E93
:1022700020004B494C4C2063617573656420627982
:10228000204B494C4C20627574746F6E2F70696ED0
:102290000A004B494C4C45442E20004B494C4C20E5
:1022A00063617573656420627920746F6F206D754A
:1022B000636820696E6163746976652074696D6511
:1022C000202D2063757272656E7420636F6D6D6171
:1022D0006E643A20004A3131005072696E74657242
:1022E0002068616C7465642E206B696C6C282920F1
:1022F00063616C6C6564210A000000A0C0000000EE
:1023000000000000005761726E696E673A20486FE6
:102310006D696E672042756D702044697669736FD0
:1023200072203C20310A000202040000A04000009C
:10233000A040000000400000614300005C4300003A
:102340004D43FFFFFF20496E76616C69642065781C
:1023500074727564657220000000A0C00000000067
:102360000000000000005C4300005C4300004D439F
:10237000486F6D696E67206661696C656400206EE8
:102380006F7420656E74657265642E0A0046696C10
:10239000652064656C657465643A0044656C6574B9
:1023A000696F6E206661696C65642C2046696C6596
:1023B0003A200050726F7465637465642050696ED2
:1023C0000A004A3036004A3034004A30370020577D
:1023D0003A004A3038004A30390020573A000000AD
:1023E0002100240027002A002D00300033000101C5
:1023F0000000040107010A01000022002500280056
:102400002B002E00310034000201000005010801FC
:102410000B01000020002300260029002C002F00C3
:102420003200000100000301060109010505050550
:10243000070508080808020202020A0A080804043C
:10244000040401010101010101010303030303036A
:102450000303040707070C0C0C0C0C0C0C0C0202F9
:10246000020206060606060606060B0B0B0B0B0BF6
:102470000B0B010210202008081020401020408083
:102480000201020108040201010204081020408038
:1024900080402010080402018004020180402010C6
:1024A000080402010804020101020408102040800F
:1024B000010204081020408000000A0B02090C0DE4
:1024C0000E080703040100000000000000000000E7
:1024D00000000000000000000000000000000000FC
:1024E00000000000121110000000000000000000B9
:1024F0000000000000000000000000000000556E19
:102500006B6E6F776E20636F6D6D616E643A202223
:10251000002066697273740A005A00590058004816
:102520006F6D6520000000484200004842000080B6
:102530004000000000545249474745524544006F4F
:1025400070656E003A20007A325F6D696E007A5FC6
:102550006D696E00795F6D696E00785F6D696E0000
:102560005265706F7274696E6720656E6473746F04
:1025700070207374617475730A000A4D6561737518
:1025800072656420706F696E74733A0A005A206F26
:1025900066667365743A20004E756D20582C593A62
:1025A00020352C350A000000000100000001000069
:1025B0008000555555000000400033333300AAAA6F
:1025C0002A004992240000002000C7711C0099993C
:1025D0001900D1451700555515003BB1130024498A
:1025E000120011111100000010000F0F0F00E3384E
:1025F0000E0043790D00CCCC0C00C3300C00E8A2D7
:102600000B0064210B00AAAA0A00703D0A009DD8A5
:102610000900427B090092240900DCD30800888865
:1026200008001042080000000800F0C1070087877A
:10263000070075500700711C07003EEB0600A1BCA7
:1026400006006990060066660600703E0600611886
:10265000060017F4050074D105005BB00500B290C8
:102660000500627205005555050078390500B81E51
:102670000500050505004EEC040087D40400A1BD4B
:10268000040090A7040049920400C17D0400EE6993
:102690000400C7560400444404005C3204000821CE
:1026A000040041100400000004003FF00300F8E0C3
:1026B000030026D20300C3C30300CCB503003AA82D
:1026C00003000A9B0300388E0300C08103009F753E
:1026D0000300D0690300505E03001D53030034481B
:1026E0000300913D03003333030016290300381F14
:1026F000030097150300300C0300030303000BFADB
:10270000020049F10200BAE802005CE002002DD8A4
:1027100002002DD0020059C80200B0C0020031B939
:102720000200DAB10200AAAA0200A0A30200BC9C27
:102730000200FA9502005C8F0200DF8802008282AC
:102740000200457C02002776020027700200436ADF
:1027500002007C640200D05E02003F590200C853B0
:10276000020048617264636F646564204465666159
:10277000756C742053657474696E6773204C6F6157
:102780006465640A00B80B0000B80B00003C000050
:1027900000102700000000FA430000FA430000C0C8
:1027A00040000070420000A0420000A0420000C8AB
:1027B000433333B94220286D6D290020204D393034
:1027C00030204B004C696E65617220416476616E09
:1027D00063653A0A0020440020490020204D333030
:1027E0003420500020440020490020204D33303157
:1027F0002050005049442073657474696E67733AC1
:102800000A00205A0020204D36363600456E64738B
:10281000746F702061646A7573746D656E743A0AC2
:1028200000205A00205900202047323920533320FD
:102830005800205A0020204D3432302053004D657E
:10284000736820426564204C6576656C696E673AF2
:102850000A00205A0020590020204D3230362058DE
:1028600000486F6D65206F66667365743A0A0020D4
:102870004500205A002059002058002054002053C1
:102880000020204D32303520510020453C6D6178CC
:102890005F655F6A65726B3E0020583C6D61785FD2
:1028A000785F6A65726B3E20593C6D61785F795F35
:1028B0006A65726B3E205A3C6D61785F7A5F6A652B
:1028C000726B3E00416476616E6365643A20513CF0
:1028D0006D696E5F7365676D656E745F74696D6554
:1028E0005F75733E20533C6D696E5F66656564720B
:1028F0006174653E20543C6D696E5F7472617665EB
:102900006C5F66656564726174653E0020540020EA
:10291000520020204D323034205000416363656CFA
:1029200065726174696F6E2028756E6974732F7398
:1029300032293A20503C7072696E745F616363653E
:102940006C3E20523C726574726163745F616363B4
:10295000656C3E20543C74726176656C5F616363A4
:10296000656C3E0A00204500205A002059002020B6
:102970004D3230312058004D6178696D756D2041C0
:102980006363656C65726174696F6E2028756E692A
:1029900074732F7332293A0A00204500205A002010
:1029A000590020204D3230332058004D6178696D38
:1029B000756D206665656472617465732028756E37
:1029C0006974732F73293A0A00204500205A0020A9
:1029D000590020204D3932205800537465707320FF
:1029E00070657220756E69743A0A0020204D32308D
:1029F000302044300A0020204D3230302044002066
:102A000044697361626C65640A0046696C616D6556
:102A10006E742073657474696E67733A0020204782
:102A20003231202020203B00FFFDFCFAF8F6F4F2C2
:102A3000F0EEECEAE9E7E5E3E1E0DEDCDAD9D7D570
:102A4000D4D2D0CFCDCBCAC8C7C5C3C2C0BFBDBC0E
:102A5000BAB9B7B6B4B3B2B0AFADACAAA9A8A6A57F
:102A6000A4A2A1A09E9D9C9A9998979594939290C8
:102A70008F8E8D8B8A8988878684838281807F7EF2
:102A80007D7B7A797877767574737271706F6E6DFD
:102A90006C6B6A696867666564636261605F5E5DEE
:102AA0005C5B5A5958585756555453525150504FD1
:102AB0004E4D4C4B4A4A494847464645444342429C
:102AC00041403F3E3E3D3C3B3B3A39383837363556
:102AD00035343332323130302F2E2E2D2C2B2B2A01
:102AE00029292827272625252423232221212020A0
:102AF0001F1E1E1D1C1C1B1B1A1919181817161631
:102B0000151514131312121111100F0F0E0E0D0DB7
:102B10000C0C0B0A0A090908080707060605050434
:102B20000403030202010000526573656E643A20DB
:102B3000006F6B0020746F6F206C6F6E672065787C
:102B400074727573696F6E2070726576656E7465E8
:102B5000640A0020636F6C64206578747275736911
:102B60006F6E2070726576656E7465640A004572DA
:102B7000726F722077726974696E6720746F204576
:102B80004550524F4D210A0057726974696E672093
:102B9000746F2066696C653A20006F70656E206600
:102BA00061696C65642C2046696C653A20006F7021
:102BB000656E206661696C65642C2046696C653AB7
:102BC000200046696C652073656C65637465640AF2
:102BD000002053697A653A200046696C65206F7061
:102BE000656E65643A20002066696C653A20006471
:102BF0006F696E67006672657368004E6F772000BC
:102C0000454E4420535542524F5554494E450A00B3
:102C10002220706F73002220706172656E743A22F8
:102C200000535542524F5554494E452043414C4C58
:102C3000207461726765743A22004B494C4C4544DC
:102C40002E2000747279696E6720746F2063616C46
:102C50006C207375622D67636F64652066696C65AF
:102C600073207769746820746F6F206D616E7920AE
:102C70006C6576656C732E204D4158206C657665C9
:102C80006C2069733A00B3DF69E111241FBECFEFF6
:102C9000D1E2DEBFCDBF00E00CBF14E0A0E0B2E0A7
:102CA000ECE8FCED01E00BBF02C007900D92A431EF
:102CB000B107D9F728E1A4E1B4E001C01D92A83C16
:102CC000B207E1F716E1C4E4D6E100E006C02197BF
:102CD0000109802FFE010E949EEDC334D10780E0E0
:102CE0000807A9F70E9413DA0C9435EE0C94000043
:102CF0002F923F924F925F926F927F928F929F920C
:102D0000AF92BF92CF92DF92EF92FF920F931F93F9
:102D1000CF93DF93CDB7DEB7CA58D1090FB6F89479
:102D2000DEBF0FBECDBF21E020933F10809115186C
:102D30008D3411F40C947621843511F40C949E2E6C
:102D4000873411F00C94EA2E809113189091141886
:102D50008A31910509F4BEC79CF4843091053CF496
:102D600082309105B4F597FF2DC00C947221843008
:102D7000910509F4D2C1059709F40EC20C94722191
:102D80008A32910511F40C9469204CF48C31910530
:102D900009F4A4C74D9709F4A6C70C9472218B358A
:102DA000910511F40C94F4208C35910511F40C94D8
:102DB000F8208A35910511F00C94722110922704A5
:102DC0000C94EC2E8091270281110C94F12E0C941E
:102DD000EC2E20912702222311F40C94EC2E11E00A
:102DE000029709F010E00E94C8AA19821A821B8279
:102DF0001C821D821E821F82188682E50E948A4CD8
:102E0000882309F43AC10E940A4C4B015C0120E07E
:102E100030E0A9010E9456E6882309F444C1C0901D
:102E20003204D0903304E0903404F0903504CCAAFE
:102E3000DDAAEEAAFFAAC0903604D0903704E09035
:102E40003804F0903904C8AED9AEEAAEFBAEC090FB
:102E5000AE10D090AF10E090B010F090B110CCAEAA
:102E6000DDAEEEAEFFAEC090B210D090B310E090E9
:102E7000B410F090B5102496CCAEDDAEEEAEFFAE41
:102E800024972CAD3DAD4EAD5FAD6CA97DA98EA94B
:102E90009FA90E9456E681110BC0A701960168AD5B
:102EA00079AD8AAD9BAD0E9456E6882309F4FBC03C
:102EB00020E030E0A901C501B4010E9456E6881F58
:102EC0008827881F181739F0C12CD12C80E8E82EEC
:102ED0008FEBF82E06C0C12CD12C00E8E02E0FE3BA
:102EE000F02E2C96CCAEDDAEEEAEFFAE2C972CA91C
:102EF0003DA94EA95FA96CAD7DAD8EAD9FAD0E9481
:102F0000A1EA28966CAF7DAF8EAF9FAF289728AD12
:102F100039AD4AAD5BAD24966CAD7DAD8EAD9FAD48
:102F200024970E94A1EA6B017C0128962CAD3DAD4F
:102F30004EAD5FAD2897CA01B9010E94BBE62B01D7
:102F40003C01A7019601C701B6010E94BBE69B01A7
:102F5000AC01C301B2010E94A2EA0E940DED2B0157
:102F60003C0120E030E040E05FE30E94BBE6609679
:102F70006CAF7DAF8EAF9FAF6097A5019401C50187
:102F8000B4010E94BBE64B015C0160962CAD3DADE7
:102F90004EAD5FAD6097CA01B9010E94BBE69B01CF
:102FA000AC01C501B4010E94A1EA0E940DED2C966E
:102FB0002CAD3DAD4EAD5FAD2C970E94BBE64B01F5
:102FC0005C01C701B6019058A30192010E947EEBFB
:102FD000A50194010E94BBE66B017C012CAD3DADC7
:102FE0004EAD5FAD6CA97DA98EA99FA90E94A2EAF2
:102FF00020E030E040E05FE30E94BBE69B01AC01D3
:10300000C701B6010E94A2EA2CA93DA94EA95FA959
:103010000E94A1EA69837A838B839C8324962CADDA
:103020003DAD4EAD5FAD249768AD79AD8AAD9BAD3A
:103030000E94A2EA20E030E040E05FE30E94BBE6AD
:103040006B017C01A301920128966CAD7DAD8EAD24
:103050009FAD28970E947EEBA50194010E94BBE6DC
:103060009B01AC01C701B6010E94A2EA28AD39ADAF
:103070004AAD5BAD0E94A1EA12C089E40E948A4C6D
:10308000882331F00E940A4C69837A838B839C8366
:103090008AE40E948A4C882331F00E940A4C6D8396
:1030A0007E838F83988720E030E0A90169817A814F
:1030B0008B819C810E9456E681110EC020E030E099
:1030C000A9016D817E818F8198850E9456E68111CC
:1030D00003C0EFECFDE10DC0412FBE016F5F7F4FDC
:1030E0008EEA90E10E94EAA40C94EC2E0E94E093F8
:1030F000F80184918F010F5F1F4F8111F7CFEDE130
:10310000F2E084918F010F5F1F4F882311F40C941C
:10311000EC2E0E94E093F801F4CF80E50E948A4CE7
:10312000882379F08091210490912204009749F03E
:103130004AE050E060E070E00E94D5E46B017C0161
:1031400003C0C12CD12C760183E50E948A4C8823D0
:1031500061F00E940A4C20E030E04AE754E40E940B
:10316000BBE60E94EBEB6B017C010E94116A0E949E
:10317000F158C60ED71EE81EF91E0E94F158DC0158
:10318000CB018C199D09AE09BF09B7FD02C00C9493
:10319000EC2E0E941EA1F1CF80912702882311F40A
:1031A0000C94EC2E0E94C8AA89E40E948A4C8823C1
:1031B00029F00E940A4C2B013C0103C0412C512CE8
:1031C00032018AE40E948A4C882329F00E940A4C2A
:1031D0004B015C0103C0812C912C540180E50E94BD
:1031E0008A4C882329F00E940A4C6B017C0103C0A1
:1031F000C12CD12C760181E50E948A4C882339F0BC
:103200000E940A4C6CAB7DAB8EAB9FAB04C01CAA7A
:103210001DAA1EAA1FAA20913E10C657DF4F288361
:10322000CA58D0406091020270910302072E000C30
:10323000880B990B0E945CE620913002309131029C
:1032400040913202509133020E94BBE62AE037EDF2
:1032500043E25CE30E94BBE668AB79AB8AAB9BAB15
:1032600040913204509133046091340470913504DC
:1032700048AF59AF6AAF7BAF9A01AB01C301B2014E
:103280000E94A2EAA1966CAF7DAF8EAF9FAFA197CF
:1032900040903604509037046090380470903904A0
:1032A000A3019201C501B4010E94A2EAA5966CAFE8
:1032B0007DAF8EAF9FAFA5972091AE103091AF102C
:1032C0004091B0105091B110C701B6010E94A2EA1E
:1032D000A9966CAF7DAF8EAF9FAFA9972091B2102A
:1032E0003091B3104091B4105091B5106CA97DA9E4
:1032F0008EA99FA90E94A2EAAD966CAF7DAF8EAF5A
:103300009FAFAD97C8ACD9ACEAACFBACC982DA824E
:10331000EB82FC824D825E826F8278860E94F15839
:103320009B01AC0128533F4F4F4F5F4FCB57DF4FAF
:10333000288339834A835B83C558D040BDEC8B2EEC
:10334000BCEC9B2EA92CBDE3BB2E25961FAE25976A
:1033500029961FAE29972D961FAE2D9761961FAE09
:1033600061970E94C27B0E94F1588B019C01CB5750
:10337000DF4FC880D980EA80FB80C558D0400C1947
:103380001D092E093F0937FD10C09B01AC012853D0
:103390003F4F4F4F5F4FCB57DF4F288339834A83CF
:1033A0005B83C558D0400E941EA125967FAD25970E
:1033B00029966FAD29972D969FAD2D9761968FAD6C
:1033C0006197272F362F492F582FC501B4010E942E
:1033D000A2EA6CAB78AF8CAF21969FAF219720E02B
:1033E00030E040E85FE30E94C8EC181644F41CAAE1
:1033F00018AE30E83CAF4FE321964FAF2197609174
:10340000AE107091AF108091B0109091B110E19614
:103410006CAF7DAF8EAF9FAFE197809132049091FA
:103420003304A0913404B0913504E5968CAF9DAF80
:10343000AEAFBFAFE59721969FAD21979F93ACADFF
:10344000AF93B8ADBF93ECA9EF93E196ACACBDAC34
:10345000CEACDFACE197A996ECACFDAC0EAD1FADE8
:10346000A997A1962CAD3DAD4EAD5FADA197E59668
:103470006CAD7DAD8EAD9FADE5970E94A1C50F905F
:103480000F900F900F9062966FAF629763967FAF29
:10349000639764968FAF649765969FAF6597C0906A
:1034A000B210D090B310E090B410F090B510E9963F
:1034B000CCAEDDAEEEAEFFAEE99720913604309192
:1034C00037044091380450913904ED962CAF3DAF4C
:1034D0004EAF5FAFED9721963FAD21973F934CAD37
:1034E0004F9358AD5F936CA96F93E996ACACBDACAC
:1034F000CEACDFACE997AD96ECACFDAC0EAD1FAD3C
:10350000AD97A5962CAD3DAD4EAD5FADA597ED96B3
:103510006CAD7DAD8EAD9FADED970E94A1C50F90B6
:103520000F900F900F9066966FAF669767967FAF7C
:10353000679768968FAF689769969FAF69978981FB
:103540009A81AB81BC81C358DF4F88839983AA835A
:10355000BB83CD57D040CD80DE80EF80F884CF573D
:10356000DF4FC882D982EA82FB82C158D0406A9676
:103570001FAE6A9725967FAD259729966FAD29973F
:103580002D969FAD2D9761968FAD6197272F362F82
:10359000492F582FBCA9A8ADFCAD2196EFAD2197BE
:1035A0006B2F7A2F8F2F9E2F0E94A1EA2FE632E1F8
:1035B00043E05BE30E9456E687FD29C125967FAD77
:1035C000259729966FAD29972D969FAD2D976196DA
:1035D0008FAD6197272F362F492F582FBCA9A8AD43
:1035E000FCAD2196EFAD21976B2F7A2F8F2F9E2F59
:1035F0000E94A2EA20E030E040E05FE30E94BBE6E8
:10360000662E972E882E792E9F938F937F936F939C
:10361000E196ACACBDACCEACDFACE197A996ECAC1E
:10362000FDAC0EAD1FADA997A1962CAD3DAD4EAD35
:103630005FADA197E5966CAD7DAD8EAD9FADE59785
:103640000E94A1C50F900F900F900F906B966FAFD7
:103650006B976C967FAF6C976D968FAF6D97C757D2
:10366000DF4F9883C958D0407F928F929F926F927C
:10367000E996ACACBDACCEACDFACE997AD96ECACAA
:10368000FDAC0EAD1FADAD97A5962CAD3DAD4EADCD
:103690005FADA597ED966CAD7DAD8EAD9FADED9711
:1036A0000E94A1C50F900F900F900F90162F072F1B
:1036B000B82EA92E66962FAD669767963FAD679791
:1036C00068964FAD689769965FAD6997CF57DF4FA2
:1036D000688179818A819B81C158D0400E94A2EA89
:1036E00020E030E040E05FE30E94BBE61B012C01DC
:1036F00062962FAD629763963FAD639764964FAD28
:10370000649765965FAD6597C358DF4F688179818F
:103710008A819B81CD57D0400E94A2EA20E030E010
:1037200040E05FE30E94BBE69B01AC016B966FAD8E
:103730006B976C967FAD6C976D968FAD6D97C757F5
:10374000DF4F9881C958D0400E94A1EA6B017C01EB
:1037500020E030E0A9010E94C8EC87FF04C0F7FA1E
:10376000F094F7F8F094A2019101612F702F8B2D46
:103770009A2D0E94A1EA1B012C0120E030E0A90152
:103780000E94C8EC87FF04C057FA509457F8509431
:10379000A2019101C701B6010E94A2EA2DEC3CEC06
:1037A0004CEC5DE30E9456E618168CF566961FAF4A
:1037B000669767960FAF67976896BFAE68976996EA
:1037C000AFAE69976B96DFAC6B976296DFAE629790
:1037D0006C96EFAC6C976396EFAE63976D96FFAC0B
:1037E0006D976496FFAE6497C757DF4F2881C9581D
:1037F000D04065962FAF65976CAA98AE8CAE219697
:103800007FAE219731E06A963FAF6A97B3CE6A9652
:103810004FAD6A97411144C125967FAD25972996F2
:103820006FAD29972D969FAD2D9761968FAD6197BE
:10383000272F362F492F582FBCA9A8ADFCAD2196B4
:10384000EFAD21976B2F7A2F8F2F9E2F0E94A1EA29
:103850006B017C012DEC3CEC4CEC5DE30E94C8EC70
:1038600018160CF41DC1A7019601C701B6010E94EC
:10387000A2EA2596EFAD25972996BFAD29972D96FB
:10388000AFAD2D976196FFAD61972E2F3B2F4A2F3D
:103890005F2F0E94A2EA662E972E882E792E20E0B6
:1038A00030E040E85FE30E94C8EC87FFF9C07F92F8
:1038B0008F929F926F92E196ACACBDACCEACDFAC78
:1038C000E197A996ECACFDAC0EAD1FADA997A19602
:1038D0002CAD3DAD4EAD5FADA197E5966CAD7DAD28
:1038E0008EAD9FADE5970E94A1C50F900F900F90F0
:1038F0000F906A966FAF6A976B967FAF6B976C96D7
:103900008FAF6C976D969FAF6D977F928F929F92BE
:103910006F92E996ACACBDACCEACDFACE997AD969E
:10392000ECACFDAC0EAD1FADAD97A5962CAD3DAD8D
:103930004EAD5FADA597ED966CAD7DAD8EAD9FADF7
:10394000ED970E94A1C50F900F900F900F90162F2A
:10395000072FB82EA92E262F372F482F592FCF5794
:10396000DF4F688179818A819B81C158D0400E9454
:10397000A2EA20E030E040E05FE30E94BBE66B019A
:103980007C016A962FAD6A976B963FAD6B976C96EC
:103990004FAD6C976D965FAD6D97C358DF4F6881E3
:1039A00079818A819B81CD57D0400E94A2EA20E094
:1039B00030E040E05FE30E94BBE69B01AC01629611
:1039C0006FAD629763967FAD639764968FAD649792
:1039D00065969FAD65970E94A1EA1B012C0120E02E
:1039E00030E0A9010E94C8EC87FF04C057FA509448
:1039F00057F85094A701960166966FAD6697679643
:103A00007FAD679768968FAD689769969FAD699708
:103A10000E94A1EA6B017C0120E030E0A9010E9434
:103A2000C8EC87FF04C0F7FAF094F7F8F094A2010D
:103A30009101C701B6010E94A2EA2DEC3CEC4CECCE
:103A40005DE30E94C8EC18165CF166961FAF66979E
:103A500067960FAF67976896BFAE68976996AFAEE7
:103A600069976A965FAD6A9762965FAF62976B9649
:103A70006FAD6B9763966FAF63976C967FAD6C97E6
:103A800064967FAF64976D968FAD6D9765968FAF97
:103A900065976CAA98AE8CAE21967FAE2197BCCE6E
:103AA00025967FAD259729966FAD29972D969FADC9
:103AB0002D9761968FAD6197272F362F492F582F5D
:103AC000BCA9A8ADFCAD2196EFAD21976B2F7A2F45
:103AD0008F2F9E2F0E94A1EA4B015C0162968FAD51
:103AE000629763969FAD63976496AFAD6497659652
:103AF000BFAD659789839A83AB83BC8366968FAD90
:103B0000669767969FAD67976896AFAD6897699619
:103B1000BFAD69978D839E83AF83B8877CA968AD5D
:103B20009CAD21968FAD2197272F362F492F582FE7
:103B300060E070E080E89FE30E94A1EA6B017C01F5
:103B400020913A0430913B0440913C0450913D0453
:103B50000E94BBE62B013C012091B6103091B710BA
:103B60004091B8105091B910BCA9A8ADFCAD2196F8
:103B7000EFAD21976B2F7A2F8F2F9E2F0E94BBE6E0
:103B80009B01AC01C301B2010E94A2EA69877A8756
:103B90008B879C8720913E0430913F0440914004E4
:103BA00050914104C701B6010E94BBE66B017C0144
:103BB0002091BA103091BB104091BC105091BD10B3
:103BC000BCA9A8ADFCAD2196EFAD21976B2F7A2F44
:103BD0008F2F9E2F0E94BBE69B01AC01C701B6014F
:103BE0000E94A2EA6D877E878F87988BCE0101960F
:103BF0000E94DEC91CA61DA61EA61FA689819A8149
:103C0000AB81BC8188A399A3AAA3BBA38D819E810C
:103C1000AF81B8858CA39DA3AEA3BFA389859A85E8
:103C2000AB85BC8588A799A7AAA7BBA7AE01485DAD
:103C30005F4FBE016C5D7F4FCE0180960E94E4BC59
:103C4000DE019C966D01C657DF4FE880CA58D04010
:103C50008E01005D1F4F9E01235F3F4FAE01485D07
:103C60005F4FBE016C5D7F4FCE0180960E94ED5983
:103C7000882329F120E030E040E85FE3BCA9A8AD4B
:103C8000FCAD2196EFAD21976B2F7A2F8F2F9E2FB2
:103C90000E9456E687FF13C03CA925963FAF2597A3
:103CA00048AD29964FAF29975CAD2D965FAF2D9704
:103CB00021966FAD219761966FAF619752CB80E1EE
:103CC000EEEAF0E1A2E3B4E001900D928A95E1F70B
:103CD0000C94EC2E0E94274E0C94EC2E80E00E9457
:103CE00068AC0C94EC2E83E50E948A4C882321F169
:103CF0000E94EA4B182F863070F0E5EEF2E08491D6
:103D00008F010F5F1F4F882311F40C94EC2E0E943B
:103D1000E093F801F4CF833009F44AC130F48130E4
:103D200091F1823009F43FC008C0843009F49FC18A
:103D3000853009F4ACC101C010E00E941BAC8111B8
:103D400003C0E5ECF2E013C080917C10882319F0E9
:103D500063E173E002C067E173E08DEB92E00E94E3
:103D600086C58AE00E94E0930E941EBD96C18491A0
:103D70007F01BFEFEB1AFB0A882309F48EC10E9472
:103D8000E093F701F4CF0E94D1BD1092010210928E
:103D9000000282EB92E09093A4078093A3070E9415
:103DA0000C940C94EC2E809100029091010297FFEC
:103DB0000EC0E9E8F2E084918F010F5F1F4F882366
:103DC00011F40C94EC2E0E94E093F801F4CF0097CC
:103DD000A1F4809152028093280419821A821B82D6
:103DE0001C8218A219A21AA21BA2BE016F5F7F4FEC
:103DF000CE0180960E9467B427C0815065E00E9482
:103E00006AED80FF03C024E0291B922F25E0920277
:103E1000F0011124E80FF11D87FDFA95EE0FFF1F49
:103E2000EE0FFF1FEA53FF4E80913A0490913B043E
:103E3000A0913C04B0913D0480839183A283B3831D
:103E40008091280480935202809100029091010297
:103E5000893191050CF067C0109252029C012F5FCE
:103E60003F4F309301022093000265E00E946AED0B
:103E700080FF03C024E0291B922F40913A04509107
:103E80003B0460913C0470913D0448A359A36AA38C
:103E90007BA319821A821B821C8244E08402900157
:103EA0001124B9016751764F4B01DB012D913D91F2
:103EB0004D915C91B4E09B02C0011124FC01E350E0
:103EC000F64F5F016081718182819381DE011196DD
:103ED0006D01E12CF12C00EA10E40E949AB31982E2
:103EE0001A821B821C82B601CE0180960E9467B4A2
:103EF000F50180819181A281B381809332049093F6
:103F00003304A0933404B0933504F401808191818B
:103F1000A281B3818093360490933704A093380430
:103F2000B0933904BCC080E090E0A0EAB0E4809394
:103F30003A0490933B04A0933C04B0933D040E9448
:103F40005BAD0E94116A8FEF9FEF90930102809307
:103F50000002E5E7F2E084918F010F5F1F4F882395
:103F600021F00E94E093F801F6CF83E992E09A8372
:103F7000898304E610E019A308A3BE016F5F7F4F99
:103F8000CE0180960E9482B58AEB92E09A83898363
:103F900019A308A3BE016F5F7F4FCE0180960E94D8
:103FA00082B581E00E9468AC81E00E9448AC77C095
:103FB00088E50E948A4C8823A1F00E94DA4B1FEF0B
:103FC000160F1530A8F0EEE5F2E084918F010F5F37
:103FD0001F4F882311F40C94EC2E0E94E093F801FB
:103FE000F4CF88E50E94E0930E94A5E10C94EC2EAA
:103FF00089E50E948A4C8823A1F00E94DA4B0FEFDA
:10400000060F0530A8F0E7E4F2E084918F010F5F1E
:104010001F4F882311F40C94EC2E0E94E093F801BA
:10402000F4CF89E50E94E0930E94A5E10C94EC2E68
:104030008AE50E948A4C882399F00E940A4C25E068
:10404000129FF0011124E00FF11DEE0FFF1FEE0F84
:10405000FF1FEA53FF4E608371838283938335C0D1
:104060008AE50E94E0930E94A5E10C94EC2E8AE57B
:104070000E948A4C8823A1F30E940A4C6093C210CC
:104080007093C3108093C4109093C5101EC080E03D
:104090000E9448AC0E94D1BD18C01230B1F46091AA
:1040A0000002709101026931710514F069E170E05C
:1040B00088E392E00E946DC569E170E083E392E0DD
:1040C0000E946DC58AE00E94E0930E94348D0C949A
:1040D000EC2E80912702882311F40C94EC2E89E4B5
:1040E0000E948A4CE82E882321F00E94DA4B062F8A
:1040F00001C000E08AE40E948A4CF82E882321F057
:104100000E94DA4B162F01C010E0EE2011F00530AE
:1041100020F4FF2081F0153070F0ECEFF2E0849194
:104120008F010F5F1F4F882311F40C94EC2E0E9417
:10413000E093F801F4CF0E94964CEE2091F034E029
:104140000302F0011124E350F64F80819181A28196
:10415000B3818093AE109093AF10A093B010B09342
:10416000B110FF2091F044E01402F0011124E75156
:10417000F64F80819181A281B3818093B210909398
:10418000B310A093B410B093B51080E50E948A4C90
:10419000882319F00E94FB4B03C080E50E94414C2C
:1041A00086E40E948A4C8823D9F00E940A4C6B0155
:1041B0007C0120E030E0A9010E94C8EC181684F4CC
:1041C00020E030E040E752E4C701B6010E947EEBF8
:1041D00060933002709331028093320290933302E5
:1041E0000E9475CA0C94EC2E209327040C94EC2E9C
:1041F00097E5292E92E0392E2DE4E22E20E1F22ED1
:1042000062E374E07DAB6CAB34E1C32E34E0D32EBB
:1042100000E010E0D1018D911D010E948A4C88239D
:1042200009F44BC00E940A4C2B013C01133049F0A9
:10423000F60120813181428153810E94A1EA2B0144
:104240003C01ACA9BDA92D913D914D915C91C3015B
:10425000B2010E94A1EA4B015C012DEB37E346E875
:1042600055EB0E94C8EC87FD0AC02DEB37E346E80A
:1042700055E3C501B4010E9456E61816F4F4133054
:1042800051F440923E0450923F0460924004709278
:10429000410401E012C0A5019401F7016081718120
:1042A000828193810E94A2EAD7016D937D938D93C1
:1042B0009C931397812F0E94B2AD1F5FB4E0EB0E69
:1042C000F11CECA9FDA93496FDABECABF4E0CF0EEC
:1042D000D11C143009F09ECF002309F4F6CE0E94C1
:1042E00036B3F3CE0E94B6B50C94EC2E8091131821
:1042F000909114188537910511F40C94EC2E0CF064
:10430000C0C08C34910509F43CC40CF058C08A310B
:10431000910509F42EC224F58531910509F4E7C110
:1043200084F48231910509F4A9C58431910509F419
:104330009EC1419711F00C949B2E0E94DFA40C9417
:10434000EC2E8731910509F4DCC10CF4D4C188311D
:10435000910509F4ECC1499709F4F4C10C949B2E22
:104360008F31910509F401C39CF48C31910509F456
:10437000A6C20CF40CC28D31910511F40C94EC2EF4
:104380004E9711F00C949B2E0E9431B00C94EC2EA1
:104390008A32910509F49CC32CF4809709F499C2E0
:1043A0000C949B2E8133910509F4C6C38B3491057F
:1043B00011F00C949B2E0E94B6780C94EC2E8A3649
:1043C000910509F40AC5B4F58435910509F456C57B
:1043D000E4F48135910509F42CC54CF48D34910534
:1043E00011F00C949B2E0E94ED780C94EC2E8235EB
:1043F000910509F440C58335910511F00C949B2E6D
:1044000081E0809326040C94EC2E8C35910509F400
:104410007BC534F48535910509F45DC50C949B2E5C
:104420008836910509F4B1C38936910509F475C43C
:104430000C949B2E8F36910509F4E3C384F48C36DB
:10444000910509F431C40CF4E4C48D36910509F4E6
:10445000A6C48E36910509F4C1C30C949B2E8137F6
:10446000910509F42DC40CF423C48237910509F495
:10447000D3C58337910511F00C949B2EE3EEF4E045
:1044800008C68E3221E0920711F40C94D72C0CF060
:1044900071C08B3C910509F416C7CCF58C38910599
:1044A00009F481C4ACF48737910509F49AC60CF479
:1044B0004BC68837910509F497C68937910511F0E5
:1044C0000C949B2E10923705109236050C94EC2E0E
:1044D0008E3B910509F47DC434F48B39910509F4C0
:1044E00037C40C949B2E883C910509F483C6893C03
:1044F000910511F00C949B2EF7E5EF2EF2E0FF2EC4
:104500000FE411E1AFE5CA2EA1E1DA2EC3C68C3D5E
:10451000910511F40C946A2B9CF48D3C910509F4DF
:1045200063C70CF4ECC68E3C910509F4EAC7833DE1
:10453000910511F00C949B2E0E94298C0C94EC2E6A
:10454000823E910511F40C94E52B3CF48D3D9105D0
:1045500011F40C94772B0C949B2E8C3241E0940731
:1045600011F40C940E2C8D32914011F40C94372CD4
:104570000C949B2E853F61E0960711F40C94C42D9A
:10458000DCF58A39A1E09A0709F496C3BCF48033BC
:10459000E1E09E0711F40C942E2D14F40C942B2DB5
:1045A000833621E0920709F45EC08039914011F012
:1045B0000C949B2E0E94116A0C94EC2E853A41E0DB
:1045C000940711F40C94C12D4CF4843A914011F0ED
:1045D0000C949B2E0E94FA8D0C94EC2E8C3A71E078
:1045E000970709F4B1C7843F914011F00C949B2EBA
:1045F0000E9458700C94EC2E8A39B2E09B0711F49B
:104600000C94032EB4F4873FF1E09F0711F40C944F
:10461000CA2D14F40C94C72D883F31E0930711F490
:104620000C94D62D8C30924011F40C94FA2D0C94ED
:104630009B2E8B3853E0950711F40C94EC2E3CF430
:104640008438934011F40C94302E0C949B2E803AB5
:10465000A3E09A0709F47CC1873E934011F40C94BF
:10466000882E0C949B2EEFECFDE10C94AE2DEAE22B
:10467000F3E084918F010F5F1F4F882321F00E9488
:10468000E093F801F6CF1092AF0C82E69AE00E9418
:10469000589A8BE1E2E6FAE0DE01159601900D9260
:1046A0008A95E1F78091600A9091610A9C838B83DF
:1046B0008DEE92E09A83898340E050E0BE016F5F07
:1046C0007F4F80E090E00E94DF82CE0101960E9441
:1046D000B4A0EBE1F3E084918F010F5F1F4F8823BB
:1046E00011F40C94EC2E0E94E093F801F4CF0E9498
:1046F000AE800C94EC2E1092310A1092320A0C9477
:10470000EC2EE0911118F09112188081882329F085
:10471000803209F410823196F8CF40E061E0809158
:104720001118909112180E94A4D50C94EC2E80912F
:10473000320A882319F081E08093310A0E94B6780A
:104740000C94EC2E1092310A80912B07813011F0DD
:104750000C94EC2E82E080932B070E94F15860931A
:104760002707709328078093290790932A070C94B2
:10477000EC2E8091320A882311F40C94EC2E83E500
:104780000E948A4C81110C94F62E0C94EC2E83E43A
:104790000E94414C882309F450C0E8E6F3E084917C
:1047A0008F010F5F1F4F882321F00E94E093F801D3
:1047B000F6CF8091FD0B811103C0EBE3F3E012C053
:1047C000BE016F5F7F4F8AEF9BE00E9420998E01B0
:1047D0000F5F1F4FF80181918F01882349F10E94DB
:1047E000E093F8CF84918F010F5F1F4F882301F171
:1047F0000E94E093F801F6CF06EDC02E03E0D02E24
:10480000E12CF12C20E08091100790E00E2C02C0EA
:10481000959587950A94E2F780FD23C2BFEFEB1AC6
:10482000FB0AE2E0CE0ED11CF5E0EF16F10459F7D9
:104830008AE00E94E0930C94EC2E8091320A882347
:1048400039F08091310A882319F0E5E4F3E003C0E0
:10485000E7E5F3E028C084918F010F5F1F4F8823A5
:1048600021F00E94E093F801F6CF6091AB0C7091BB
:10487000AC0C8091AD0C9091AE0C4AE00E94019777
:104880008FE20E94E0936091A70C7091A80C809138
:10489000A90C9091AA0C4AE00E9401978AE00E941C
:1048A000E0930C94EC2E84918F010F5F1F4F8823AF
:1048B00011F40C94EC2E0E94E093F801F4CF40E048
:1048C00060E080911118909112180E94A4D50C9468
:1048D000EC2E8091310A81110E94116A8091320A76
:1048E000882311F40C94EC2E80E50E948A4C8823D6
:1048F00019F00E94FB4B03C080E50E94414C182F29
:10490000482F61E080911118909112180E94A4D54F
:1049100083E50E948A4C882381F00E94DA4BAB0128
:10492000BC014093AB0C5093AC0C6093AD0C7093F6
:10493000AE0C8AEF9BE00E9411988091320A882386
:1049400019F081E08093310A11110C94EC2EF6CE0F
:10495000809111189091121821E02093300A40E0C4
:1049600060E00E94A4D50C94EC2E0E9467787B0135
:104970008C0120E831E541E050E00E9444EAC901A1
:104980006DE671E00E9477ED4B015C01C801B70153
:1049900020E13EE040E050E00E9444EACA01B90153
:1049A00028E130E040E050E00E9444EA762E672E95
:1049B000C62ED72E8CE3282E312C412C512CC80129
:1049C000B701A20191010E9444EAF62EE72ECA0126
:1049D000B901A20191010E9444EACB018E010F5F4F
:1049E0001F4F81149104D1F0EF92FF927F936F9348
:1049F0006F927F92BF92AF929F928F928FE993E0D6
:104A00009F938F931F930F930E9428E60FB6F894FD
:104A1000DEBF0FBECDBFE4EEFDE145C0A114B10481
:104A200089F0EF92FF927F936F936F927F92BF9284
:104A3000AF928FE893E09F938F931F930F930E9401
:104A400028E6E4CFCD2879F0EF92FF927F936F9321
:104A50006F927F9283E893E09F938F931F930F93BE
:104A60000E9428E6D3CF892B69F0EF92FF927F93C3
:104A70006F938BE793E09F938F931F930F930E9405
:104A800028E6C4CFEF92FF9287E793E09F938F933E
:104A90001F930F930E9428E60F900F900F900F9096
:104AA0000F900F90B8CF84917F019FEFE91AF90A18
:104AB000882321F00E94E093F701F5CFB80183EB42
:104AC00093E00E9486C58AE00E94E0930C94EC2E4D
:104AD00083E50E948A4C882311F40C94EC2E0E94EA
:104AE000EA4BE82E80E50E948A4C882339F00E9428
:104AF000EA4B182F87FF03C00C94EC2E1DE089E4CD
:104B00000E948A4C882341F00E94FB4B81110C9437
:104B1000722FEBE1F6E00BC089E40E94414CF6CF26
:104B20003196A6E0EB34FA0711F40C94722F8491BD
:104B30001813F6CF0C94472FF090200481E0F8264C
:104B4000F0922004EBECF3E084918F010F5F1F4F94
:104B5000882321F00E94E093F801F6CFFF2019F09E
:104B6000E0ECF3E002C0E5ECF3E084918F010F5F2D
:104B70001F4F882311F40C94EC2E0E94E093F8014F
:104B8000F4CF0E94D8780C94EC2E88E690E00E9436
:104B9000F2AD81110C94EC2E8091100783FF02C0BE
:104BA0000C94EC2E83E50E948A4C882399F00E9495
:104BB0000A4C0E94E6EBCB010E94E6590E940A4C87
:104BC00020E030E044EB52E40E9456E6181614F060
:104BD0000E94ED780E94B0C70C94EC2E8EE40E94E7
:104BE0008A4C882311F40C94EC2E0E94DA4B6093CB
:104BF000BE187093BF188093C0189093C1180C947E
:104C0000EC2E83E50E94414C882359F083E50E94F5
:104C10008A4C882319F00E94EA4B01C080E08093FF
:104C20001007E4EEFDE184918F010F5F1F4F8111AA
:104C300003C0E4EEF3E004C00E94E093F801F3CF78
:104C400084918F010F5F1F4F882321F00E94E09312
:104C5000F801F6CF809110078111CECDE0EEF3E0A0
:104C600018C0BB24B394B20E222319F08CE20E9428
:104C7000E093F60185919491FC0184918F010F5F7F
:104C80001F4F882321F00E94E093F801F6CF2B2DCF
:104C9000C5CD84918F010F5F1F4F882309F4C8CDC4
:104CA0000E94E093F801F5CF109220020C94EC2EB4
:104CB0008BEE93E00E94D7A00E948D860C94EC2E80
:104CC00083E50E948A4C811103C0E4EEFDE10DC032
:104CD0000E94EA4B8D3320F480932B020C94EC2E2F
:104CE0008CE380932B020C94EC2E84918F010F5F48
:104CF0001F4F882321F00E94E093F801F6CF4091E6
:104D00002B0250E060E070E084EF93E00E9433C536
:104D10008AE00E94E0930C94EC2E89E690E00E94D9
:104D2000F2AD811111C0EBEFF3E084918F010F5FC1
:104D30001F4F882321F00E94E093F801F6CF0E94D4
:104D4000EF758AE00E94E09310923F100C94872F39
:104D500083E50E948A4C882311F40C94EC2E0E9467
:104D6000EA4B182F8D3308F01CE310934C100E946F
:104D7000F1586B017C01212F30E0A8EEB3E00E94D6
:104D800092EAC60ED71EE81EF91EC0924810D092B5
:104D90004910E0924A10F0924B100C94EC2E0E94B5
:104DA00034AE0C94EC2E8091100783FF02C00C945B
:104DB000EC2E83E50E948A4C882311F40C94EC2E8F
:104DC0000E940A4C0E94E6EBCB010E94194E0C9403
:104DD000EC2E0E94F8A80C94EC2E80E50E948A4CE0
:104DE000811106C083E50E948A4C882359F005C0D2
:104DF0000E94EA4B8111F0C7F5CF0E94DA4B6F3F5A
:104E0000710510F06FEF70E07093430460934204FB
:104E1000E3C780E50E948A4C811105C010924304CB
:104E200010924204D9C70E94DA4B672B09F0D4C70D
:104E3000F5CF0E9402790E94C6B7109243041092E7
:104E4000420400E010E062E370E080E090E00E9445
:104E50002CB70E94C27B0F5F1F4F0331110599F7DA
:104E600062E370E080E090E00E942CB70E94C27B79
:104E70000E94A12FB1C710922604AEC783E50E94FD
:104E80008A4C882399F00E940A4C20E030E04AE7DF
:104E900054E40E94BBE60E94EBEB60932C027093FB
:104EA0002D0280932E0290932F0296C788E50E94D0
:104EB000414C8111ACC789E50E94414C8111A7C7C3
:104EC0008AE50E94414C8111A2C785E40E94414CB1
:104ED00081119DC7CEC783E50E94414C882309F408
:104EE0007BC70E940A4C20E030E04AE754E40E946D
:104EF000BBE60E94EBEB60934410709345108093E7
:104F000046109093471068C7B7E5CB2EB2E0DB2E72
:104F100012E9E12E10E1F12E10E0D6018D916D0124
:104F20000E94414C882309F46DC0133009F063C01E
:104F30000E940A4C4B015C0120E030E040EA51E461
:104F40000E9456E687FF4EC0A501940160919E1015
:104F500070919F108091A0109091A1100E947EEB03
:104F60002B013C019B01AC016091DF067091E006D2
:104F70008091E1069091E2060E94BBE66093DF0615
:104F80007093E0068093E1069093E206A3019201FC
:104F90006091FF06709100078091010790910207D0
:104FA0000E94BBE66093FF067093000780930107A1
:104FB0009093020760914B1170914C1180914D11AB
:104FC00090914E110E945AE6A30192010E94BBE605
:104FD0000E94EBEB60934B1170934C1180934D1139
:104FE00090934E1180929E1090929F10A092A010CC
:104FF000B092A11007C00E940A4CF7016083718330
:10500000828393831F5FF4E0EF0EF11C143009F0EC
:1050100084CF0E9451C9E0C60E94116A83E50E94B4
:105020008A4C882309F451C80E94DA4B623071051A
:1050300009F04BC80E94C2C98BE50E94E0936091C1
:10504000A4187091A5188091A6189091A71842E015
:105050000E9486974091A8185091A9186091AA18AB
:105060007091AB1881E094E00E9450C54091AC185B
:105070005091AD186091AE187091AF188EEF93E01B
:105080000E9450C58DE50E94E0938AE00E94E09363
:10509000A3C684918F010F5F1F4F882321F00E94C8
:1050A000E093F801F6CF60E083ED94E00E94018D7B
:1050B00061E08CEC94E00E94018D61E081EC94E071
:1050C0000E94018D61E081EB94E00E94018D60E01F
:1050D00088EA94E00E94018D61E08EE994E00E94EC
:1050E000018D60E084E994E00E94018D60E08CE82D
:1050F00094E00E94018D61E08EE794E00E94018DB2
:1051000060E080E794E00E94018D60E081E694E039
:105110000E94018D60E083E594E00E94018D60E0D3
:105120008DE394E00E94018D60E08CE294E00E94A7
:10513000018D60E087E194E00E94018D61E084E0F0
:1051400094E00E94018D48C6009111181091121828
:1051500083E0D12C40E08150E9F0D8019C91292FC7
:105160002B7F2134C1F711962C912133A1F7913473
:1051700021F0953421F441E002C0DD24D39498015C
:105180002E5F3F4F89012F5F3F4FF8019081903292
:10519000C9F3E1CF442369F0E4EEFDE184917F019E
:1051A0002FEFE21AF20A882321F00E94E093F70120
:1051B000F5CFDD2069F0E9EAF5E084917F013FEF6A
:1051C000E31AF30A882321F00E94E093F701F5CF58
:1051D000D8018D918D01882309F42ACB0E94E09398
:1051E000F7CF0E9469BEF8C581E0809337058093B0
:1051F0003605F2C588EC90E00E94F2AD8111ECC555
:1052000084E40E94414C882309F441C00E940A4C66
:105210006B017C0111E020E030E0A9010E9456E61C
:10522000811101C010E010932A1120E030E0A901A3
:10523000C701B6010E9456E6882349F10E940A4C34
:10524000E0914E07B4E0EB9FF0011124E15DFE4ECA
:10525000608371838283938320E030E0A9016091B1
:105260002F117091301180913111909132110E9463
:1052700056E681110CC080E090E0A0EEBFE3809381
:105280002F1190933011A0933111B09332110E94DD
:1052900004B8A2C5F70181917F010E94414C882387
:1052A00051F00E940A4C0E94EBEBD8016D937D9364
:1052B0008D939C9313970C5F1F4FC016D10651F727
:1052C0000E94E0C789C5E7E5EE2EE2E0FE2E03EF7F
:1052D00016E0F70181917F010E94414C882341F043
:1052E0000E940A4CD8016D937D938D939C931397E4
:1052F0000C5F1F4FB7E003301B0759F76DC583E5FF
:105300000E948A4C8823A1F00E940A4C6093EB060D
:105310007093EC068093ED069093EE066093E7069B
:105320007093E8068093E9069093EA0610E001C0C6
:1053300011E080E50E948A4C882359F00E940A4CB3
:105340006093EB067093EC068093ED069093EE0667
:1053500010E082E50E948A4C882359F00E940A4C92
:105360006093EF067093F0068093F1069093F20637
:1053700010E084E50E948A4C882359F00E940A4C70
:105380006093E7067093E8068093E9069093EA0637
:1053900023C5112309F420C54091EB065091EC067A
:1053A0006091ED067091EE0683EB95E00E9450C58A
:1053B0004091EF065091F0066091F1067091F2066F
:1053C00080EB95E00E9450C54091E7065091E806B9
:1053D0006091E9067091EA068DEA95E00E9450C559
:1053E0008AE00E94E093F8C481E50E94414C882342
:1053F000C1F08091210490912204009739F04AE095
:1054000050E060E070E00E94D5E403C060E070E02E
:10541000CB01609303077093040780930507909373
:10542000060783E50E94414C882351F00E940A4CF4
:1054300060930B0770930C0780930D0790930E07F2
:1054400084E50E94414C882351F00E940A4C6093ED
:105450000707709308078093090790930A0788E568
:105460000E94414C882351F00E940A4C6093D3065D
:105470007093D4068093D5069093D60689E50E9452
:10548000414C882351F00E940A4C6093D7067093D8
:10549000D8068093D9069093DA068AE50E94414C9B
:1054A0008823F1F00E940A4C6093DB067093DC06BF
:1054B0008093DD069093DE062DEC3CEC4CEC5DE336
:1054C0000E9456E6181664F0E3ECF5E084918F0133
:1054D0000F5F1F4F882321F00E94E093F801F6CF61
:1054E00085E40E94414C882309F476C40E940A4C4A
:1054F0006093DF067093E0068093E1069093E206E6
:105500006BC467E5C62E62E0D62E78E3E72E75E021
:10551000F72E10E0F60181916F010E94414C882323
:1055200059F00E940A4CD7016D937D938D939C9303
:105530001397812F0E94B2AD1F5FB4E0EB0EF11CF8
:10554000133041F70C9465200E9485B4811144C446
:1055500009EF12E2E2E3F4E0FDABECAB9E012F5F5A
:105560003F4F590152E4852E53E2952E1901F8015F
:105570006591759185919491ACA9BDA9CD90DD906F
:10558000ED90FD90BDABACABA70196010E94A1EAE6
:105590002B013C01F101608371838283938320E0BE
:1055A00030E040EA51EC0E94C8EC87FD0AC020E0E0
:1055B00030E040EA51E4C301B2010E9456E61816F9
:1055C0002CF4F401849118160CF456C4D101CD903A
:1055D000DD90ED90FD901D0120E030E040EA51ECBF
:1055E000C701B6010E94C8EC87FD0AC020E030E088
:1055F00040EA51E4C701B6010E9456E618164CF580
:10560000EFECFDE184918F010F5F1F4F811103C00B
:10561000E5EFF5E004C00E94E093F801F3CF849138
:105620008F010F5F1F4F882321F00E94E093F80144
:10563000F6CF88E290E099A388A388EC90E09DA73C
:105640008CA7BE01605E7F4FCE018C960E9482B512
:10565000C3C30C5F1F4FBFEF8B1A9B0AE5E0F3E259
:10566000E017F10709F083CF48E3E42E45E0F42E7C
:1056700010E0F50181919191A191B1915F01F70144
:1056800081939193A193B1937F01812F0E94B2AD39
:105690001F5F133071F70E94348D83E992E09DA75C
:1056A0008CA704E610E019A308A3BE01645D7F4F38
:1056B000CE0180960E9482B58AEB92E09DA78CA7CE
:1056C00019A308A3BE01645D7F4FCE0180960E949E
:1056D00082B582C383E50E948A4C882309F47CC387
:1056E0000E94DA4B709303026093020275C38DED42
:1056F00090E00E94F2AD81116FC383E50E948A4C55
:10570000811103C0E4EEFDE13AC000914E0710E0C4
:105710000E94DA4B000F111FF801E85CFD4F718306
:10572000608380914E0790E07C01EE0CFF1CEE0C34
:10573000FF1C87010F5D1D4F880F991FFC01E85C5E
:10574000FD4F60817181072E000C880B990B0E9420
:105750005CE62AE037ED43E25CE30E94BBE6F7013A
:10576000E55DFE4E20813181428153810E94BBE67E
:10577000D8016D937D938D939C9313972DC3849142
:105780008F010F5F1F4F882321F00E94E093F801E3
:10579000F6CF85E40E94E09380914E07805D0E94E1
:1057A000E093E0914E07F0E0EE0FFF1FE85CFD4F45
:1057B0006081718183E196E00E946DC585E20E945F
:1057C000E0938AE00E94E09307C380E50E94414C89
:1057D000882309F401C30E94DA4B6B017C0183E545
:1057E0000E948A4C882321F00E94DA4B8B0102C070
:1057F0000FEF1FEFC8010196039708F0EDC2D7FC29
:10580000EBC28C2DEBE1F6E09491891709F43FC3CC
:105810003196B6E0EB34FB07B9F73CC383E50E9451
:105820008A4C882319F00E94DA4B02C064E071E0D0
:1058300079A368A380E50E948A4C882339F00E94EE
:10584000DA4B6938E3E17E0730F402C068EE73E0BA
:105850007A83698304C088E893E19A838983BE01CF
:10586000605E7F4FCE0101960E9482B5B5C285E48D
:105870000E948A4C811110C080E50E94414C88230F
:1058800091F00E940A4C60933C0770933D0780930F
:105890003E0790933F0707C00E94EA4B882361F3BD
:1058A000EFECFDE171C089E40E94414C882381F056
:1058B0000E940A4C2CEA35EC47E25EE30E94BBE60C
:1058C000609338077093390780933A0790933B07AA
:1058D00084E40E94414C882381F00E940A4C2CEA07
:1058E00035EC47E25EE30E947EEB609340077093E5
:1058F00041078093420790934307E4EEFDE18491D2
:105900008F010F5F1F4F882321F00E94E093F80161
:10591000F6CF40913C0750913D0760913E07709152
:105920003F0783E596E00E9450C52CEA35EC47E23C
:105930005EE3609138077091390780913A07909142
:105940003B070E947EEBAB01BC018FE496E00E9416
:1059500050C52CEA35EC47E25EE360914007709158
:10596000410780914207909143070E94BBE6AB013B
:10597000BC018BE496E00E9450C58AE00E94E0934F
:105980002BC20E94E093F80184918F010F5F1F4F9B
:105990008111F7CFE7E5F6E084918F010F5F1F4F8C
:1059A000882309F419C20E94E093F801F5CF83E53A
:1059B0000E94414C182F882371F00E940A4C0E94CB
:1059C000E6EB709326026093250221E0672B09F035
:1059D00020E020930F0780E50E94414C882359F076
:1059E0002091250230912602232B11F00E94FB4BBF
:1059F00080930F07F1C11111EFC1E4EEFDE1849135
:105A00008F010F5F1F4F882321F00E94E093F80160
:105A1000F6CF80910F07882319F06BE173E002C085
:105A20006EE173E08EE796E00E9486C560912502E4
:105A3000709126028DE696E00E946DC5E9E6F6E0DB
:105A400084918F010F5F1F4F882309F4C5C10E9405
:105A5000E093F801F5CF0E94CA86BEC180E50E949E
:105A6000414C882351F00E940A4C60933407709394
:105A70003507809336079093370789E40E94414C9D
:105A8000882381F00E940A4C2CEA35EC47E25EE361
:105A90000E94BBE660933007709331078093320712
:105AA0009093330784E40E94414C882381F00E9444
:105AB0000A4C2CEA35EC47E25EE30E947EEB6093F1
:105AC0002C0770932D0780932E0790932F07E4EEF9
:105AD000FDE184918F010F5F1F4F882321F00E9409
:105AE000E093F801F6CF409134075091350760916B
:105AF00036077091370789E996E00E9450C52CEA75
:105B000035EC47E25EE36091300770913107809198
:105B10003207909133070E947EEBAB01BC0185E90F
:105B200096E00E9450C52CEA35EC47E25EE36091B6
:105B30002C0770912D0780912E0790912F070E94BE
:105B4000BBE6AB01BC0181E996E00E9450C58AE04A
:105B50000E94E09341C10E94E093F80184918F017B
:105B60000F5F1F4F8111F7CFEDE9F6E084918F01B0
:105B70000F5F1F4F882309F42FC10E94E093F801A3
:105B8000F5CF0E94A28528C10E944C7025C10E94B9
:105B90000DC322C183E50E94414C882321F00E945D
:105BA000FB4B91E089270E949EBE16C181E0809345
:105BB00017070E94426A10921707882309F40CC144
:105BC000E4EEFDE184918F010F5F1F4F811103C04F
:105BD000ECEAF6E004C00E94E093F801F3CF849170
:105BE0008F010F5F1F4F882309F4F6C00E94E093D6
:105BF000F801F5CF8091310A882309F4EDC081E0E6
:105C00008093340AE9C08AE50E948A4C811103C05E
:105C1000EAEBF6E00BC00E940A4C609337117093D8
:105C200038118093391190933A11D6C084918F0125
:105C30000F5F1F4F882321F00E94E093F801F6CFF9
:105C400040913711509138116091391170913A118A
:105C500087EB96E00E9450C58AE00E94E093BCC0AA
:105C60008BE40E948A4C811103C0E4EEFDE136C052
:105C70008BE40E948A4C8823C1F00E940A4C6B017D
:105C80007C0120E030E0A9010E94C8EC87FD0AC039
:105C900020E030E040E251E4C701B6010E9456E640
:105CA000181634F4E9EDF6E00EC0C12CD12C7601C3
:105CB0000E94116AC092E306D092E406E092E506E3
:105CC000F092E60689C084918F010F5F1F4F8823F1
:105CD00009F482C00E94E093F801F5CF84918F010E
:105CE0000F5F1F4F882321F00E94E093F801F6CF49
:105CF0004091E3065091E4066091E5067091E60656
:105D000088EF96E00E9450C58AE00E94E09364C04C
:105D100081E08093270283E50E948A4C882339F032
:105D20000E94FB4B811158C00E9466CE55C083E58E
:105D30000E94414CF7CF0E94B6B54EC0F0901318A8
:105D40000E94116A10917C1080E00E9448ACFF20F4
:105D500029F1E4EEFDE184918F010F5F1F4F88234D
:105D600021F00E94E093F801F6CF84E50E94E093D1
:105D70006F2D70E080E090E04AE00E94019780E2A1
:105D80000E94E093E5E1F7E084918F010F5F1F4FE0
:105D9000882311F10E94E093F801F6CF10923E1093
:105DA000812F0E9448ACE4EEFDE184918F010F5FEA
:105DB0001F4F882321F00E94E093F801F6CF6091F5
:105DC0003E1070E083E097E00E946DC58AE00E947B
:105DD000E09302C00E94B6B510923F100E9449CED7
:105DE00096C00E94C8AA0E9475CAF6CF0E94DA4BDC
:105DF000AB01BC014093AB0C5093AC0C6093AD0C69
:105E00007093AE0C8AEF9BE00E941198E5CF0E9440
:105E1000116A88E50E94414C882331F05F9A809195
:105E200031048E7F8093310489E50E94414C8823A0
:105E300039F08A9A479A809131048D7F809331049A
:105E40008AE50E94414C882361F080910801809589
:105E5000817080930601479A809131048B7F8093F3
:105E6000310485E40E94414C882309F4B5CF129A8D
:105E7000B3CF0E94C6B7B0CFF7FAF094F7F8F0941A
:105E8000D101CD92DD92ED92FC9213979FCB0E94AF
:105E90008AE1A2CF0E94116ABC2C60E08C2D0E9486
:105EA00029B60F3FBFEF1B0759F48C2D0E94D3B5C5
:105EB00031E020E0892B09F030E0032F122F05C0DC
:105EC0000130110561F401E010E08B2D0E94D3B583
:105ED0008017910709F480CF0E941EA1F6CF00E041
:105EE00010E0F3CF61E0812F0E9429B66E2D812F43
:105EF0000E94FBB5F12CB701812F0E9465B61930C5
:105F000009F06ACFF0924304E092420465CFC6578D
:105F1000DF4F0FB6F894DEBF0FBECDBFDF91CF913C
:105F20001F910F91FF90EF90DF90CF90BF90AF90B7
:105F30009F908F907F906F905F904F903F902F90A9
:105F400008952F923F924F925F926F927F928F921D
:105F50009F92AF92BF92CF92DF92EF92FF920F93F8
:105F60001F93CF93DF93CDB7DEB76F970FB6F8943B
:105F7000DEBF0FBECDBFC0904C04D0904D04E0906A
:105F80004E04F0904F0420E030E040EA50E4C701B6
:105F9000B6010E9456E687FD19C120E030E041E9D4
:105FA00053E4C701B6010E94C8EC18160CF40EC1E8
:105FB00010924E0E10924D0E8091090140914C0EA0
:105FC000042E000C550B817021E0822790E04817C9
:105FD000590709F433C08091090181702827209363
:105FE0004C0E81111BC00E94AE80EFE2FDE0849157
:105FF0008F01882351F0082E000C990B0E94A98074
:106000000F5F1F4FF8018491F4CF8DE090E00E9464
:10601000A9808AE090E00E94A98010C0E3E3FDE03F
:1060200084918F01882389F3082E000C990B0E941C
:10603000A9800F5F1F4FF8018491F4CF80913F0E2C
:10604000833009F44CC02CF4882351F08130D9F00E
:1060500072C0843009F43EC0853009F44DC06BC075
:106060008091310A882309F466C081E080933F0E55
:106070000E94F1586093430E7093440E8093450E36
:106080009093460E58C08091310A811154C080917E
:10609000FD0B882321F082E080933F0E4CC01092CC
:1060A0003F0EEBE2FDE084918F01882351F0082E32
:1060B000000C990B0E94A9800F5F1F4FF80184917B
:1060C000F4CF8DE090E00E94A9808AE090E00E94E9
:1060D000A98031C080918C0E8823E9F22CC0809178
:1060E000310A811128C08091B3099091B409891BAC
:1060F0008F7009F496C01FC08091310A81111BC0B6
:106100008091B3099091B409891B8F7009F4ABC0D9
:1061100012C08DE090E00E94A9808AE090E00E9489
:10612000A98010923F0E8BE09DE09093A40780938E
:10613000A3070E940C948091340E9091350E039722
:106140004CF57FE3272E79E0372EE0E68E2EEAEE3F
:106150009E2EA12CB12C8AE99FE00E945C4B181660
:106160001906C4F48091340E9091350E049794F47E
:106170008AE99FE00E94204B80933A0EE0913B0E0B
:10618000F0913C0E8A3019F08D3009F07DC03097C7
:1061900009F083C08091340E9091350E009711F470
:1061A0000C94223F01979093350E8093340E80918A
:1061B000360E9091370E019664E070E00E948BEDF0
:1061C0009093370E8093360E0C94223F80914D0EA3
:1061D00090914E0E8136FAEE9F07E8F010924E0E27
:1061E00010924D0EE7E3FDE084918F01882351F07A
:1061F000082E000C990B0E94A9800F5F1F4FF80119
:106200008491F4CF8DE090E00E94A9808AE090E034
:106210000E94A980D1CE019690934E0E80934D0E90
:10622000CBCE87E19DE09093A4078093A3070E94C3
:106230000C9480918C0E882311F082E001C084E0E0
:1062400080933F0EE3E1FDE084918F01882309F400
:1062500038CF082E000C990B0E94A9800F5F1F4FAA
:10626000F8018491F3CFEFE0FDE084918F01882362
:1062700009F44FCF082E000C990B0E94A9800F5FE4
:106280001F4FF8018491F3CF8A3309F480CFEF35A3
:10629000F10514F40C94B63C7ACF8091380E9091AD
:1062A000390E20E6289F7001299FF00C11248701E8
:1062B0000C54134FE00FF11F108261E470E0C8012D
:1062C0000E94F2ED009711F40C949A3C90933E0ECC
:1062D00080933D0E801B910B8E0D9F1D60E070E042
:1062E0008B54934F0E9457E20E94E6EBCB01770F4D
:1062F000AA0BBB0B8232910510F00C949A3CFC0166
:106300008827EE58FF4F8F4F0C949EEDE6E0FDE09E
:1063100084918F01882351F0082E000C990B0E9464
:10632000A9800F5F1F4FF8018491F4CF20E030E087
:1063300040E05FE360914C0470914D0480914E0405
:1063400090914F041EC0E1E0FDE084918F0188230D
:1063500051F0082E000C990B0E94A9800F5F1F4F6F
:10636000F8018491F4CF60914A0470914B04072E98
:10637000000C880B990B0E945CE620E030E040E0C6
:106380005FE30E94A2EA0E94E6EBCB010E94E34D8C
:106390000E94DAD78DE090E00E94A9808AE090E028
:1063A0000E94A9800C949A3CECEFFCE084918F0150
:1063B000882351F0082E000C990B0E94A9800F5FD2
:1063C0001F4FF8018491F4CF20E030E040E05FE31C
:1063D000609146047091470480914804909149046B
:1063E000D0CFE7EFFCE084918F01882351F0082E95
:1063F000000C990B0E94A9800F5F1F4FF801849138
:10640000F4CF6091440470914504B1CF20914204CF
:106410003091430444E6429FC001439F900D1124F4
:106420006FEF70E00E948BED8B016536710510F007
:1064300004E610E0E2EFFCE084917F01882359F04C
:10644000082E000C990B0E94A980FFEFEF1AFF0A9B
:10645000F7018491F3CFB80180E090E036C7EEEE0B
:10646000FCE084918F01882351F0082E000C990BD9
:106470000E94A9800F5F1F4FF8018491F4CF80E242
:1064800090E00E94A980EAEEFCE084918F018823CD
:1064900051F0082E000C990B0E94A9800F5F1F4F2E
:1064A000F8018491F4CF60913204709133048091AB
:1064B0003404909135040E94DBD780E290E00E9482
:1064C000A980E6EEFCE084918F01882351F0082E2C
:1064D000000C990B0E94A9800F5F1F4FF801849157
:1064E000F4CF609136047091370480913804909114
:1064F00039040E94DBD780E290E00E94A980E2EE9E
:10650000FCE084918F01882351F0082E000C990B38
:106510000E94A9800F5F1F4FF8018491F4CF609112
:106520003A0470913B0480913C0490913D040E9498
:10653000DBD780E290E0A0C58091310A882309F47E
:1065400050C0EDEDFCE084918F01882351F0082EBE
:10655000000C990B0E94A9800F5F1F4FF8018491D6
:10656000F4CF8091320A882359F18091FD0B882362
:1065700029F18091A70C9091A80CA091A90CB09141
:10658000AA0C0097A105B105C1F0BC01CD016D5960
:106590007F4F8F4F9F4F24E630E040E050E00E9455
:1065A00044EA6091AB0C7091AC0C8091AD0C909171
:1065B000AE0C0E9444EA822F01C080E090E0E6CE5B
:1065C000E9EDFCE084918F01882309F4E3CE082EE5
:1065D000000C990B0E94A9800F5F1F4FF801849156
:1065E000F3CFE1EDFCE084918F01882309F4D2CE52
:1065F000082E000C990B0E94A9800F5F1F4FF80115
:106600008491F3CFECECFCE084918F01882351F06E
:10661000082E000C990B0E94A9800F5F1F4FF801F4
:106620008491F4CF8091430E9091440EA091450E39
:10663000B091460E892B8A2B8B2B09F477C00E94D0
:10664000F158A50194010E9444EA69017A01609120
:10665000430E7091440E8091450E9091460EA50117
:1066600094010E9444EA8601021B130BC8016CE3EB
:1066700070E00E9477EDCB019927EAE0F0E0BF01DE
:106680000E948BED282FCB01BF010E948BED805D16
:1066900080932904205D20932A0410922B0489E220
:1066A00094E00E94DAD780E290E00E94A980EAECB0
:1066B000FCE084917F01882359F0082E000C990B8F
:1066C0000E94A980FFEFEF1AFF0AF7018491F3CF30
:1066D00080E290E00E94A980C8016CE370E00E9413
:1066E00077ED6AE070E00E948BED605D60932904B5
:1066F000805D80932A0410922B0489E294E00E942A
:10670000DAD780E290E00E94A980E8ECFCE0849176
:106710008F01882309F43ECE082E000C990B0E94AD
:10672000A9800F5F1F4FF8018491F3CF80E290E0C2
:106730000E94A980E0ECFCE084918F01882309F499
:1067400029CE082E000C990B0E94A9800F5F1F4FC5
:10675000F8018491F3CF10926D0E8091090180FFB2
:1067600011C0ECEBFCE084918F01882309F412CE78
:10677000082E000C990B0E94A9800F5F1F4FF80193
:106780008491F3CF83E50E9476D7882341F00E945D
:1067900091D70E94EBEB7093420E6093410EE8EBB1
:1067A000FCE084918F01882351F0082E000C990B96
:1067B0000E94A9800F5F1F4FF8018491F4CF8DE0F4
:1067C00090E00E94A9808AE090E00E94A9808091D8
:1067D0008B0E882309F442C28091410E9091420EA3
:1067E0008430910509F4C8C08830910509F47DC151
:1067F000892B09F0E7C3ECEDFAE084918F0188233F
:1068000051F0082E000C990B0E94A9800F5F1F4FBA
:10681000F8018491F4CF8DE090E00E94A9808AE095
:1068200090E00E94A980E1EDFAE084918F01882335
:1068300051F0082E000C990B0E94A9800F5F1F4F8A
:10684000F8018491F4CF8DE090E00E94A9808AE065
:1068500090E00E94A980E5ECFAE084918F01882302
:1068600051F0082E000C990B0E94A9800F5F1F4F5A
:10687000F8018491F4CF8DE090E00E94A9808AE035
:1068800090E00E94A980E9EBFAE084918F018823CF
:1068900051F0082E000C990B0E94A9800F5F1F4F2A
:1068A000F8018491F4CF8DE090E00E94A9808AE005
:1068B00090E00E94A980EBEAFAE084918F0188239E
:1068C00051F0082E000C990B0E94A9800F5F1F4FFA
:1068D000F8018491F4CF8DE090E00E94A9808AE0D5
:1068E00090E00E94A980EDE9FAE084918F0188236D
:1068F00051F0082E000C990B0E94A9800F5F1F4FCA
:10690000F8018491F4CF8DE090E00E94A9808AE0A4
:1069100090E00E94A980E0E9FAE084918F01882349
:1069200051F0082E000C990B0E94A9800F5F1F4F99
:10693000F8018491F4CF8DE090E00E94A9808AE074
:1069400090E00E94A980E3E8FAE084918F01882317
:1069500051F0082E000C990B0E94A9800F5F1F4F69
:10696000F8018491F4CF8DE090E00E94A9808AE044
:1069700090E00E94A98026C3E5E7FAE084918F01A8
:10698000882351F0082E000C990B0E94A9800F5FFC
:106990001F4FF8018491F4CF8DE090E00E94A98010
:1069A0008AE090E00E94A980E7E6FAE084918F01F6
:1069B000882351F0082E000C990B0E94A9800F5FCC
:1069C0001F4FF8018491F4CF8DE090E00E94A980E0
:1069D0008AE090E00E94A980E1E5FAE084918F01CD
:1069E000882351F0082E000C990B0E94A9800F5F9C
:1069F0001F4FF8018491F4CF8DE090E00E94A980B0
:106A00008AE090E00E94A980EBE3FAE084918F0194
:106A1000882351F0082E000C990B0E94A9800F5F6B
:106A20001F4FF8018491F4CF8DE090E00E94A9807F
:106A30008AE090E00E94A980E9E2FAE084918F0167
:106A4000882351F0082E000C990B0E94A9800F5F3B
:106A50001F4FF8018491F4CF8DE090E00E94A9804F
:106A60008AE090E00E94A980E7E1FAE084918F013A
:106A7000882351F0082E000C990B0E94A9800F5F0B
:106A80001F4FF8018491F4CF8DE090E00E94A9801F
:106A90008AE090E00E94A980E9E0FAE084918F0109
:106AA000882351F0082E000C990B0E94A9800F5FDB
:106AB0001F4FF8018491F4CF8DE090E00E94A980EF
:106AC0008AE090E00E94A980EBEFF9E084918F01C9
:106AD000882309F448CF082E000C990B0E94A98046
:106AE0000F5F1F4FF8018491F3CFE4EFF9E0849139
:106AF0008F01882351F0082E000C990B0E94A98069
:106B00000F5F1F4FF8018491F4CF8DE090E00E9459
:106B1000A9808AE090E00E94A980EDEEF9E08491DE
:106B20008F01882351F0082E000C990B0E94A98038
:106B30000F5F1F4FF8018491F4CF8DE090E00E9429
:106B4000A9808AE090E00E94A980E6EDF9E08491B6
:106B50008F01882351F0082E000C990B0E94A98008
:106B60000F5F1F4FF8018491F4CF8DE090E00E94F9
:106B7000A9808AE090E00E94A980EFEBF9E084917F
:106B80008F01882351F0082E000C990B0E94A980D8
:106B90000F5F1F4FF8018491F4CF8DE090E00E94C9
:106BA000A9808AE090E00E94A980E8EAF9E0849157
:106BB0008F01882351F0082E000C990B0E94A980A8
:106BC0000F5F1F4FF8018491F4CF8DE090E00E9499
:106BD000A9808AE090E00E94A980E1E9F9E084912F
:106BE0008F01882351F0082E000C990B0E94A98078
:106BF0000F5F1F4FF8018491F4CF8DE090E00E9469
:106C0000A9808AE090E00E94A980E3E8F9E08491FD
:106C10008F01882351F0082E000C990B0E94A98047
:106C20000F5F1F4FF8018491F4CF8DE090E00E9438
:106C3000A9808AE090E00E94A980E5E7F9E08491CC
:106C40008F01882309F48FCE082E000C990B0E9427
:106C5000A9800F5F1F4FF8018491F3CF8091320A12
:106C6000882309F486C181E08093AF0C1092B10CA7
:106C70001092B00C81E89AE00E94589A8BE1E1E80A
:106C8000FAE0DE01159601900D928A95E1F7809168
:106C90007F0A9091800A9C838B838DEE92E09A8389
:106CA000898340E050E0BE016F5F7F4F80E090E05D
:106CB0000E94DF82CE0101960E94B4A0C090B00C69
:106CC000D090B10C0091410E1091420EC601801B74
:106CD000910B049720F06801F3E0CF0ED11C56E62B
:106CE000452E59E0552E67E5662E69E0762EC016D2
:106CF000D10608F467C10115110509F0A1C065E3CB
:106D00007AE081E89AE00E94209962E273E085E3EC
:106D10009AE00E94FDED892B09F04AC0F2018491AE
:106D200046E6E42E49E0F42E882359F0082E000CA4
:106D3000990B0E94A980FFEFEF1AFF0AF7018491D7
:106D4000F3CF8DE090E00E94A9808AE090E00E945D
:106D5000A980F301849137E5E32E39E0F32E8823EF
:106D600059F0082E000C990B0E94A980FFEFEF1A32
:106D7000FF0AF7018491F3CF8DE090E00E94A98093
:106D80008AE090E00E94A9804AE060E070E0CB01D8
:106D90000E940197E7E4F9E084917F012FEFE21A66
:106DA000F20A882309F4E2C00E94E093F701F4CFCD
:106DB000E3E4F9E084917F01882359F0082E000C68
:106DC000990B0E94A980FFEFEF1AFF0AF701849147
:106DD000F3CF8DE090E00E94A9808AE090E00E94CD
:106DE000A980F10184912FE3E22E29E0F22E88237D
:106DF00059F0082E000C990B0E94A980FFEFEF1AA2
:106E0000FF0AF7018491F3CF8DE090E00E94A98002
:106E10008AE090E00E94A9804AE060E070E0CB0147
:106E20000E940197EAE3F9E084917F012FEFE21AD3
:106E3000F20A882309F49AC00E94E093F701F4CF84
:106E400060E070E0C80101970E94A5848091330A38
:106E5000882309F45FC0E8E3F9E084917F01882387
:106E600059F0082E000C990B0E94A980FFEFEF1A31
:106E7000FF0AF7018491F3CF85E39AE00E94DAD705
:106E80008DE090E00E94A9808AE090E00E94A980B5
:106E9000E6E3F9E084917F01882359F0082E000C85
:106EA000990B0E94A980FFEFEF1AFF0AF701849166
:106EB000F3CF82E49AE00E94DAD78DE090E00E945E
:106EC000A9808AE090E00E94A980C801A0E0B0E01B
:106ED0004AE0BC01CD010E940197E4E3F9E084910E
:106EE0007F012FEFE21AF20A882321F00E94E0933B
:106EF000F701F5CF92E4E92E9AE0F92EF70181919E
:106F00007F01882319F00E94E093F8CF8AE00E9465
:106F1000E0932CC085E39AE00E94DAD78DE090E000
:106F20000E94A9808AE090E00E94A98082E49AE011
:106F30000E94DAD78DE090E00E94A9808AE090E07C
:106F40000E94A980C801A0E0B0E04AE0BC01CD01E8
:106F50000E94019782E4E82E8AE0F82EF7018191E1
:106F60007F01882399F20E94E093F8CF0F5F1F4FB3
:106F7000BECEE5E2F9E084918F01882351F0082E1E
:106F8000000C990B0E94A9800F5F1F4FF80184919C
:106F9000F4CF8DE090E00E94A9808AE090E00E940A
:106FA000A980E6E1F9E084918F01882309F4DBCC24
:106FB000082E000C990B0E94A9800F5F1F4FF8014B
:106FC0008491F3CFE4EBFCE084918F01882309F4F2
:106FD000E1C9082E000C990B0E94A9800F5F1F4F7A
:106FE000F8018491F3CF8091310A882339F00E940F
:106FF0001182A0C48091310A8823E9F00E942DB14A
:1070000099C480913F0E823019F0833609F092C402
:107010000E94F081E0EBFCE084918F01882309F469
:10702000B9C9082E000C990B0E94A9800F5F1F4F51
:10703000F8018491F3CF80913F0E833609F07AC432
:10704000DDCF87EA9CE00E94D7A08091B3099091A0
:10705000B409891B8F7009F06DC480913F0E823096
:1070600009F468C4833609F099C464C48DE090E0E3
:107070000E94A9808AE090E00E94A9808BC980913B
:10708000B3099091B409891B8F7009F053C48091A2
:107090003F0E823009F44EC4833609F44BC480910C
:1070A000FD0B8111CFC446C483E50E9476D78111C0
:1070B00026C083E40E9476D7882309F43BC48091DC
:1070C000B3099091B409891B8F7009F033C420E093
:1070D00030E040E251E460913A0470913B048091C9
:1070E0003C0490913D040E9456E687FF08C084E965
:1070F0009CE09093A4078093A3070E940C940E94A5
:1071000091D720E030E0A9010E9456E687FD10C02B
:107110000E9491D720E030E849E853E40E94C8EC8F
:1071200018164CF00E9491D70E94EBEBCB0105C0E2
:1071300080E090E002C083E191E00E94E659FAC34A
:1071400083E50E9476D7882309F4F4C30E9491D77F
:1071500020E030E0A9010E9456E687FD10C00E94A1
:1071600091D720E030E046E153E40E94C8EC1816C5
:107170004CF00E9491D70E94EBEBCB0105C080E060
:1071800090E002C086E990E00E94194ED3C383E5E7
:107190000E9476D78823D9F00E9491D720E030E072
:1071A0004FE753E40E94BBE620E030E048EC52E4B5
:1071B0000E947EEB0E94EBEB6F3F710519F010F01F
:1071C0006FEF70E07093430460934204E3C88FEF65
:1071D00090E09093430480934204DCC88091B3090B
:1071E0009091B409891B8F7009F0D4C88091310A3D
:1071F0008111D0C80E948D865F9A809131048E7F64
:10720000809331048A9A479A809131048D7F8093CC
:107210003104809108018095817080930601479A1E
:10722000809131048B7F80933104129AB3C883E537
:107230000E9476D7882319F10E9491D720E030E090
:1072400040E252E40E9456E687FD0FC00E9491D7AB
:1072500020E030EC49E754E40E94C8EC181644F0F2
:107260000E9491D70E94E6EB05C068E270E002C080
:1072700067EE73E070930302609302025BC3EEE873
:10728000FCE084918F01882351F0082E000C990BAB
:107290000E94A9800F5F1F4FF8018491F4CFC09026
:1072A0000202D09003020D2C000CEE08FF08F7FE3E
:1072B0000EC06DE28AE99FE00E94D34A66277727D5
:1072C000CB016C197D098E099F094AE003C04AE091
:1072D000C701B6010E949AD75DC88091B309909109
:1072E000B409891B8F7009F025C380913F0E82304D
:1072F00009F420C3833609F0EBC21CC38091B309A3
:107300009091B409891B8F7009F044C880913F0E99
:10731000823009F43FC8833609F0B6C33BC8809178
:10732000B3099091B409891B8F7009F003C3809150
:107330003F0E823009F4FEC2833609F0FBC4FAC264
:107340008091B3099091B409891B8F7009F0F2C242
:1073500080913F0E823009F4EDC2833609F020C5DA
:10736000E9C28091B3099091B409891B8F7009F02B
:10737000E1C280913F0E823009F4DCC2833609F00D
:1073800045C5D8C280916D0E811103C00E94AE80A8
:10739000C4C18E3271F580916E0E8E3209F046C1F5
:1073A0008091D20B882309F4B8C181508093D20B0D
:1073B000882361F090E001974FE1489F9001499F39
:1073C000300D1124C9018456954F02C08EE59AE014
:1073D0002BE1FC013496A1E8BAE001900D922A95C8
:1073E000E1F7FC01828193819093800A80937F0A68
:1073F00094C18C3309F01AC164E273E08DE69EE01B
:107400000E94FDED892B21F481E080938B0E85C1D4
:1074100063E373E08DE69EE00E94FDED892B79F435
:10742000E2EFF8E084918F010F5F1F4F882321F076
:107430000E94E093F801F6CF85ED98E0E4C06AE49D
:1074400073E08DE69EE00E94FDED892B79F4E1EB7F
:10745000F8E084918F010F5F1F4F882321F00E9475
:10746000E093F801F6CF8EE998E0CDC061E673E0D5
:107470008DE69EE00E94FDED892B79F4E3E8F8E0CB
:1074800084918F010F5F1F4F882321F00E94E093AA
:10749000F801F6CF8EE798E0B6C06FE673E08DE6B0
:1074A0009EE00E94FDED892B79F4E3E6F8E08491FB
:1074B0008F010F5F1F4F882321F00E94E093F80196
:1074C000F6CF8EE598E09FC06DE773E08DE69EE015
:1074D0000E94FDED892B79F4E3E4F8E084918F01BB
:1074E0000F5F1F4F882321F00E94E093F801F6CF31
:1074F0008AE398E088C06BE873E08DE69EE00E9426
:10750000FDED892B71F407E118E0F80184918823DF
:1075100029F00F5F1F4F0E94E093F7CF80E198E0C2
:1075200072C061EA73E08DE69EE00E94FDED892B5A
:1075300079F4E1EFF7E084918F010F5F1F4F88230B
:1075400021F00E94E093F801F6CF8AEE97E05BC04D
:1075500063EB73E08DE69EE00E94FDED892B79F4EC
:10756000E2EDF7E084918F010F5F1F4F882321F038
:107570000E94E093F801F6CF81EC97E044C06EEBF7
:1075800073E08DE69EE00E94FDED892B79F4E8EA38
:10759000F7E084918F010F5F1F4F882321F00E9435
:1075A000E093F801F6CF86E997E02DC06AEC73E02E
:1075B0008DE69EE00E94FDED892B79F4EBE7F7E084
:1075C00084918F010F5F1F4F882321F00E94E09369
:1075D000F801F6CF89E697E016C068ED73E08DE616
:1075E0009EE00E94FDED892BA9F4EFE4F7E0849181
:1075F0008F010F5F1F4F882321F00E94E093F80155
:10760000F6CF8DE397E09093A4078093A3070E94A1
:107610000C9483C065EE73E08DE69EE00E94FDED64
:10762000892B09F07AC010928B0E77C01D821886C4
:107630001C821B828DEE92E09A8389838091840A5A
:10764000811103C06EE57AE002C06DE77AE0611552
:10765000710519F06C5F7F4F02C060E070E021E0BF
:107660004DE65EE0CE0105960E94879E882361F17B
:107670008BE1FE013596A1E8BAE001900D928A9562
:10768000E1F72B813C813093800A20937F0A80911F
:10769000D20B8A3008F03DC091E0980F9093D20B46
:1076A000FFE18F9FC0011124DC01A056B54F4BE1D3
:1076B000E1E8FAE001900D924A95E1F7FC01E45609
:1076C000F54F3383228325C0E4EEFDE184918F01E1
:1076D0000F5F1F4F882321F00E94E093F801F6CF3F
:1076E000E7E2F7E084918F010F5F1F4F882321F0BD
:1076F0000E94E093F801F6CF0DE61EE0F8018191BB
:107700008F01882319F00E94E093F8CF8AE00E944D
:10771000E093CE0101960E94B4A010926D0E80916C
:10772000090180FF07C1E2EDFBE084918F0188230E
:1077300011F40C94CA31082E000C990B0E94A980F8
:107740000F5F1F4FF8018491F2CF8FE40E9476D72C
:1077500081110C94CA3183E40E9476D70C94CA310B
:1077600083E50E9476D7811159C08FE40E9476D7B5
:10777000882319F08AE99BE007C084E50E9476D748
:10778000882349F082E79BE09093A4078093A307A6
:107790000E940C9443C083E40E9476D7882319F09A
:1077A00089E49BE0F1CF81E50E9476D7882319F028
:1077B00081E29BE0E9CF88E40E9476D78823C9F074
:1077C000EDE1FBE084918F01882351F0082E000C3D
:1077D000990B0E94A9800F5F1F4FF8018491F4CF8D
:1077E0008DE090E00E94A9808AE090E00E94A9804C
:1077F00015C08CE40E9476D7882381F0E9E1FBE094
:1078000084918F01882361F3082E000C990B0E944C
:10781000A9800F5F1F4FF8018491F4CFE1EEFBE0E8
:1078200084918F01882311F40C94CA31082E000C26
:10783000990B0E94A9800F5F1F4FF8018491F2CF2E
:107840008091B3098091B4090C94CA3183E50E94F8
:1078500076D7882309F46EC081EF9AE09093A4074D
:107860008093A3070E940C94E1EEFBE084918F01CA
:10787000882311F40C94CA31082E000C990B0E9435
:10788000A9800F5F1F4FF8018491F2CFECEEFAE070
:1078900084918F01882351F0082E000C990B0E94CF
:1078A000A9800F5F1F4FF8018491F4CFE7EEFAE053
:1078B00084918F01882311F40C94CA31082E000C96
:1078C000990B0E94A9800F5F1F4FF8018491F2CF9E
:1078D00088E50E9476D7811106C089E50E9476D797
:1078E000882309F4C3C088E50E9476D7882341F035
:1078F00088E89CE09093A4078093A3070E940C94CF
:1079000089E50E9476D7882341F082E89CE0909335
:10791000A4078093A3070E940C948AE50E9476D75F
:10792000882341F08CE79CE09093A4078093A30701
:107930000E940C948091380E9091390E019664E06B
:1079400070E00E948BED9093390E8093380E8091F9
:10795000340E9091350E01969093350E8093340E2F
:1079600010923C0E10923B0E0C94AB304091380EAE
:107970005091390E9F012F5F3F4F30933C0E209363
:107980003B0E90E6949F9001959F300D11242C544E
:10799000334FE20FF31F80830C94AB3000913D0E08
:1079A00010913E0E780124E0E20EF11C6AE270E0D4
:1079B000C7010E94F2EDF80124812F3221F4B801B1
:1079C0006B5F7F4F03C02C3339F4B7018DE69EE027
:1079D0000E9406EE0C94CA3110926D0E009719F0B9
:1079E000FC013197108280913D0E90913E0E40E057
:1079F00061E004960E94A4D58091FD0B882389F054
:107A0000E3EAFCE084918F01882309F42FCB082E50
:107A1000000C990B0E94A9800F5F1F4FF801849101
:107A2000F3CFEFE9FCE084918F01882309F41ECBAA
:107A3000082E000C990B0E94A9800F5F1F4FF801C0
:107A40008491F3CF0E94F081EBE9FCE084918F01F7
:107A5000882311F40C94CA31082E000C990B0E9453
:107A6000A9800F5F1F4FF8018491F2CF8AE50E9431
:107A700076D7811138CF83E40E9476D7882309F422
:107A800059CF88E79CE050CF86E40E9476D78823C0
:107A900009F44DC10E9491D70E94EBEB8B0184E762
:107AA0009CE09093A4078093A3070E940C9488E520
:107AB0000E9476D7882309F451C00E9491D72B01E8
:107AC0003C012DEC3CEC4CE45EE30E9456E69E014A
:107AD0002F5F3F4F7901181674F020E030E0A901C4
:107AE000C301B2010E94C8EC18162CF41F930F9327
:107AF00089E69CE005C12DEC3CEC4CEC5DEBC30150
:107B0000B2010E9456E618167CF020E030E040E812
:107B10005FEBC301B2010E94C8EC18162CF41F934E
:107B20000F938DE59CE0ECC01F930F93C301B2014E
:107B30000E94E6EB7F936F9383E59CE09F938F9386
:107B4000FF92EF920E9428E60FB6F894DEBF0FBEB8
:107B5000CDBFCE0101960E94E793DFC089E50E9468
:107B600076D7882309F441C00E9491D72B013C01AC
:107B70002DEC3CEC4CE45EE30E9456E6FE013196AF
:107B80007F01181674F020E030E0A901C301B201B2
:107B90000E94C8EC18162CF41F930F9388E49CE005
:107BA000AFC02DEC3CEC4CEC5DEBC301B2010E948C
:107BB00056E618167CF020E030E040E85FEBC301A9
:107BC000B2010E94C8EC18162CF41F930F938CE39B
:107BD0009CE096C01F930F93C301B2010E94E6EB95
:107BE0007F936F9382E39CE0A9CF8AE50E9476D7CA
:107BF000882309F441C00E9491D72B013C012DEC50
:107C00003CEC4CE45EE30E9456E6FE0131967F01B7
:107C1000181674F020E030E0A901C301B2010E94FF
:107C2000C8EC18162CF41F930F9387E29CE068C0F1
:107C30002DEC3CEC4CEC5DEBC301B2010E9456E62E
:107C400018167CF020E030E040E85FEBC301B201A1
:107C50000E94C8EC18162CF41F930F938BE19CE044
:107C60004FC01F930F93C301B2010E94E6EB7F93B5
:107C70006F9381E19CE062CF85E40E9476D78823F0
:107C800009F44BC00E9491D72B013C012DEC3CEC38
:107C90004CE45EE30E9456E6FE0131967F01181621
:107CA00074F020E030E0A901C301B2010E94C8ECE9
:107CB00018162CF41F930F9386E09CE021C02DEC46
:107CC0003CEC4CEC5DEBC301B2010E9456E6181689
:107CD0007CF020E030E040E85FEBC301B2010E949D
:107CE000C8EC18162CF41F930F938AEF9BE008C082
:107CF000C301B2010E94E6EB7F936F938FEE9BE08E
:107D00009F938F93FF92EF920E9428E60F900F901F
:107D10000F900F900F900F901CCF8BEE9BE09093E5
:107D2000A4078093A3070E940C940C94CA3100E02E
:107D300010E0B5CE20E030E040E251E460913A043A
:107D400070913B0480913C0490913D040E9456E662
:107D500087FF08C084EE9BE09093A4078093A3075D
:107D60000E940C9482E390E0909345048093440435
:107D70000E94A97688EC90E00E94E659E1EEFBE0D3
:107D800084918F01882311F40C94CA31082E000CC1
:107D9000990B0E94A9800F5F1F4FF8018491F2CFC9
:107DA00020E030E040E251E460913A0470913B04FD
:107DB00080913C0490913D040E9456E687FF08C0E4
:107DC0008AED9BE09093A4078093A3070E940C94F4
:107DD00080E590E090934504809344040E94A97646
:107DE00080EF90E00E94E659E1EEFBE084918F0184
:107DF000882311F40C94CA31082E000C990B0E94B0
:107E0000A9800F5F1F4FF8018491F2CF80E090E0CE
:107E10000E94E65910924504109244040E94A976EB
:107E2000E6EDFBE084918F01882311F40C94CA31B4
:107E3000082E000C990B0E94A9800F5F1F4FF801BC
:107E40008491F2CF6F960FB6F894DEBF0FBECDBF10
:107E5000DF91CF911F910F91FF90EF90DF90CF9026
:107E6000BF90AF909F908F907F906F905F904F905A
:107E70003F902F9008952F923F924F925F926F9272
:107E80007F928F929F92AF92BF92CF92DF92EF92AA
:107E9000FF920F931F93CF93DF93CDB7DEB7629717
:107EA0000FB6F894DEBF0FBECDBFF8948FEF9FEFF3
:107EB00090938900809388002AE02A8B212C312C12
:107EC00078948091A2049091A304A091A404B0910D
:107ED000A504892B8A2B8B2B09F00FC280911A07DE
:107EE0008823E1F010921A078091180790911907E2
:107EF000892B09F402C210925A04109219071092A9
:107F000018079091B3098091B409981709F4F5C145
:107F10008091B4098F5F8F708093B40980911807A6
:107F200090911907892B09F4E8C140919E04509162
:107F30009F046091A0047091A10480919A04909193
:107F40009B04A0919C04B0919D040091910410E0C9
:107F500020E030E0841B950BA60BB70B0817190720
:107F60002A073B0710F4D901C801E82F840F951F99
:107F7000A61FB71F80939E0490939F04A093A00414
:107F8000B093A1042091840030918500245E3F4F7E
:107F9000409176045091770460917804709179044F
:107FA0008091660490916704A0916804B09169047F
:107FB000840F951FA61FB71F8093760490937704B4
:107FC000A0937804B0937904B7FD1CC0889A80917F
:107FD000821090918310A0918410B09185104091EF
:107FE0000402042E000C550B660B770B840F951FB3
:107FF000A61FB71F8093821090938310A0938410C4
:10800000B093851040917A0450917B0460917C0478
:1080100070917D0480916A0490916B04A0916C042E
:10802000B0916D04840F951FA61FB71F80937A042B
:1080300090937B04A0937C04B0937D04B7FD1CC097
:108040008E9A8091861090918710A0918810B0919F
:10805000891040910502042E000C550B660B770B1E
:10806000840F951FA61FB71F8093861090938710CB
:10807000A0938810B093891040917E0450917F04A2
:10808000609180047091810480916E0490916F04DE
:10809000A0917004B0917104840F951FA61FB71FA3
:1080A00080937E0490937F04A0938004B093810416
:1080B000B7FD3FC080915404F09106028823C9F0B7
:1080C0008091520482FF02C0F7FD06C080915104E6
:1080D000882311F40C94E548809152049091530444
:1080E00093FF02C0F7FD0CC080915004811108C0BD
:1080F00006C080910B018095887080930901419A98
:1081000040918A1050918B1060918C1070918D105D
:108110008F2FFF0F990BAA0BBB0B840F951FA61F68
:10812000B71F80938A1090938B10A0938C10B093FC
:108130008D10409182045091830460918404709169
:1081400085048091720490917304A0917404B0919D
:108150007504840F951FA61FB71F80938204909308
:108160008304A0938404B0938504B7FD3AC0409182
:108170008E1050918F106091901070919110C0905E
:1081800007020C2C000CDD08EE08FF084C0D5D1DED
:108190006E1D7F1D40938E1050938F106093901032
:1081A0007093911040916204509163046091640453
:1081B00070916504841B950BA60BB70B809382040A
:1081C00090938304A0938404B09385049091550404
:1081D00080918F0493FF02C0815001C08F5F809314
:1081E0008F048091760490917704A0917804B091E7
:1081F0007904B7FD15C04091620450916304609109
:10820000640470916504841B950BA60BB70B8093D7
:10821000760490937704A0937804B09379048898B7
:1082200080917A0490917B04A0917C04B0917D04AC
:10823000B7FD15C0409162045091630460916404DD
:1082400070916504841B950BA60BB70B80937A0481
:1082500090937B04A0937C04B0937D048E988091CE
:108260007E0490917F04A0918004B0918104B7FDB9
:108270003AC040916204509163046091640470912B
:108280006504841B950BA60BB70B80937E0490931B
:108290007F04A0938004B0938104809154048823C8
:1082A000E1F08091520482FF04C08091060287FDB4
:1082B00005C080915104882309F48FC7809152042E
:1082C0009091530493FF04C08091060287FD0BC078
:1082D00080915004811107C005C080910B01887006
:1082E000809309014198E15041F080918400909180
:1082F000850082179307C8F34BCE809111029091AD
:108300001202A0911302B0911402892B8A2B8B2B9D
:1083100009F08AC080919004882309F453C08090AA
:108320009E0490909F04A090A004B090A104C090DF
:108330008B04D0908C04E0908D04F0908E044091DA
:108340008F04C814D904EA04FB0480F480915B0410
:1083500090915C0420915F043091600428173907E4
:1083600028F4415040938F04019714C08C149D044D
:10837000AE04BF04E0F480915B0490915C04209112
:108380005D0430915E048217930788F44F5F409339
:108390008F04019690935C0480935B0440910D02DE
:1083A00050910E0260910F02709110020EC08FEF7B
:1083B0009FEFDC0180930D0290930E02A0930F02B9
:1083C000B09310024FEF5FEFBA0180918F0487FDE9
:1083D00002C0169A01C01698809184009091850081
:1083E0004C9620918F042223B9F0149A20918F0487
:1083F00027FF02C02F5F01C0215020938F041498E3
:1084000020918F04222369F320918400309185000C
:1084100028173907C8F3E5CF409311025093120291
:1084200060931302709314028091A2049091A304AC
:10843000A091A404B091A504892B8A2B8B2B09F061
:1084400049C6A0911807B0911907109711F40C9420
:108450008F4A80909E0490909F04A090A004B090BA
:10846000A10440919A0450919B0460919C047091E6
:108470009D0484169506A606B706D8F010925A04F5
:1084800010921907109218079091B3098091B409BE
:10849000981711F40C948F4A8091B4098F5F8F70F4
:1084A0008093B40940EDC42E47E0D42EE12CF12C8A
:1084B0001AC4409196045091970460919804709169
:1084C0009904481559056A057B0508F4AAC140912D
:1084D0009204509193046091940470919504D696FF
:1084E0000D911D912D913C91D9974017510762072D
:1084F000730708F077C1411551056105710549F40D
:108500008090560490905704A0905804B09059045D
:1085100064C1E12CF980842E952F862F0A811B815E
:10852000FD81EE813F8128859C80E091EF17E89DD9
:10853000912CFF273091F017389D900CF11D109071
:10854000F117189CF00DE99F900CF11D399FF00D6B
:10855000E89FF00D092D1F2F099DE12D33272227BC
:108560000F9FE00D311D2E1D199DE00D311D2E1D9B
:108570001F9F300D211D032F122F099DF12C332732
:1085800022270F9FF00C311D2E1D199DF00C311D5F
:108590002E1D1F9F300D211D032F122FEE278090BF
:1085A000560490915704809158040090B2040E280C
:1085B00009F483C03091AE04309FE1198E089E0902
:1085C0008E092091AF04209FE01981089E098E0931
:1085D000F090B004F09E801891098E09319FE01947
:1085E00081089E098E09219F801891098E09F19EAC
:1085F00090198109099DF12C332722270F9FF00C38
:10860000311D2E1D199DF00C311D2E1D1F9F300D8B
:10861000211D032F122F3091AA04309FE10D8E1CD3
:108620009E1D8E1D2091AB04209FE00D811C9E1D80
:108630008E1DF090AC04F09E800C911D8E1D319F1C
:10864000E00D811C9E1D8E1D219F800C911D8E1D95
:10865000F19E900D811D099DF12C332722270F9F3C
:10866000F00C311D2E1D199DF00C311D2E1D1F9F6C
:10867000300D211D032F122F3091A604309FE119D8
:108680008E089E098E092091A704209FE019810879
:108690009E098E09F090A804F09E801891098E0919
:1086A000319FE01981089E098E09219F8018910948
:1086B0008E09F19E9019810982C03091AE04309FDD
:1086C000E10D8E1C9E1D8E1D2091AF04209FE00D9C
:1086D000811C9E1D8E1DF090B004F09E800C911D9B
:1086E0008E1D319FE00D811C9E1D8E1D219F800CD3
:1086F000911D8E1DF19E900D811D099DF12C33273A
:1087000022270F9FF00C311D2E1D199DF00C311DDD
:108710002E1D1F9F300D211D032F122F3091AA04F3
:10872000309FE1198E089E098E092091AB04209F8D
:10873000E01981089E098E09F090AC04F09E801823
:1087400091098E09319FE01981089E098E09219FA8
:10875000801891098E09F19E90198109099DF12CCB
:10876000332722270F9FF00C311D2E1D199DF00C71
:10877000311D2E1D1F9F300D211D032F122F3091F3
:10878000A604309FE10D8E1C9E1D8E1D2091A70416
:10879000209FE00D811C9E1D8E1DF090A804F09E70
:1087A000800C911D8E1D319FE00D811C9E1D8E1D24
:1087B000219F800C911D8E1DF19E900D811D112415
:1087C0009C82F9820A831B83FD83EE833F83288783
:1087D000912C992AA12CB12CA82A8BE395E121E0B8
:1087E000298B14C0D2968D909D90AD90BC90D5975A
:1087F000F4CFB694A79497948794D988DD0CD98A3E
:10880000049625E18735920709F4EDC4FC01059132
:10881000159125913491081519052A053B0548F352
:10882000E2C440908B0450908C0460908D04709052
:108830008E04481459046A047B0408F0C3C1809173
:108840008A04811121C0FD01EE5BFF4FE080F180C1
:108850000281138178962081318142815381D296A1
:108860006D917D918D919C91D5970E947FC4DD245F
:10887000D394D0928A04E0911807F091190782A945
:1088800093A9A4A9B5A98EC14091860450918704EB
:108890006091880470918904DA960D911D912D9153
:1088A0003C91DD97401751076207730708F073C1C9
:1088B000411551056105710549F480915604909167
:1088C0005704A0915804B09159046CC1F0E0E985B7
:1088D000842F352F262FAA857B856C855D85BE85E7
:1088E0004F859889B091EF17B89F612D552740911A
:1088F000F017489F600D511D1090F117189E500DF4
:10890000B39F600D511D439F500DB29F500DA62F78
:10891000752FA69FB12D44279927A59FB00D411D06
:108920009F1F769FB00D411D9F1F759F400D911D8C
:10893000A42F792FA69FE12D44279927A59FE00D0D
:10894000411D9F1F769FE00D411D9F1F759F400D8C
:10895000911DA42F792FBB27809156043091570485
:10896000209158040090B2040F2A09F483C040916A
:10897000AE044A9FB1198F0B3F0B2F0B9091AF04A0
:108980009A9FB01981093F0B2F0BE091B004EA9F29
:10899000801931092F0B479FB01981093F0B2F0B0D
:1089A000979F801931092F0BE79F30192109A69F46
:1089B000E12D44279927A59FE00D411D9F1F769F1C
:1089C000E00D411D9F1F759F400D911DA42F792F14
:1089D0004091AA044A9FB10D8F1F3F1F2F1F9091F6
:1089E000AB049A9FB00D811D3F1F2F1FE091AC0477
:1089F000EA9F800D311D2F1F479FB00D811D3F1F26
:108A00002F1F979F800D311D2F1FE79F300D211DB8
:108A1000A69FE12D44279927A59FE00D411D9F1F8B
:108A2000769FE00D411D9F1F759F400D911DA42F46
:108A3000792F4091A6044A9FB1198F0B3F0B2F0B42
:108A40009091A7049A9FB01981093F0B2F0BE091D9
:108A5000A804EA9F801931092F0B479FB01981099B
:108A60003F0B2F0B979F801931092F0BE79F301970
:108A7000210982C04091AE044A9FB10D8F1F3F1F54
:108A80002F1F9091AF049A9FB00D811D3F1F2F1F84
:108A9000E091B004EA9F800D311D2F1F479FB00D5C
:108AA000811D3F1F2F1F979F800D311D2F1FE79F97
:108AB000300D211DA69FE12D44279927A59FE00D8C
:108AC000411D9F1F769FE00D411D9F1F759F400D0B
:108AD000911DA42F792F4091AA044A9FB1198F0BA1
:108AE0003F0B2F0B9091AB049A9FB01981093F0B5C
:108AF0002F0BE091AC04EA9F801931092F0B479F9F
:108B0000B01981093F0B2F0B979F801931092F0B4B
:108B1000E79F30192109A69FE12D44279927A59F9A
:108B2000E00D411D9F1F769FE00D411D9F1F759F0A
:108B3000400D911DA42F792F4091A6044A9FB10D9D
:108B40008F1F3F1F2F1F9091A7049A9FB00D811D6B
:108B50003F1F2F1FE091A804EA9F800D311D2F1F9A
:108B6000479FB00D811D3F1F2F1F979F800D311D07
:108B70002F1FE79F300D211D1124E987AA877B87CE
:108B80006C875D87BE874F87988B90E0932BA0E022
:108B9000B0E0A22B07C0A65ABF4F8D919D910D90BA
:108BA000BC91A02D2BE335E141E0498BF9014591C2
:108BB000559165917491481759076A077B0708F426
:108BC0009CC3AAC380918F048823E1F0FD01E85B78
:108BD000FF4F4081518160E070E000910D021091E3
:108BE0000E0220910F0230911002401751076207C8
:108BF000730741F0109211021092120210921302A8
:108C0000109214024091090250910A0260910B02E5
:108C100070910C0277FF5FC0AE5ABF4FCD90DD90D0
:108C2000ED90FC908BE395E121E0FC01459155919D
:108C3000659174914C155D056E057F0550F4F694B1
:108C4000E794D794C794220F049675E18735970768
:108C500061F72093910480E2C816D104E104F10485
:108C600028F470E2C72ED12CE12CF12C90E2C91A25
:108C7000D108E108F108C114A8E0DA06E104F10422
:108C800008F406C4B4E0DB9EC0011124855C9E4E4E
:108C9000FC01329625913491EC2D6627E39FA001CB
:108CA000E29F410D561F0694461F561F112460E097
:108CB00070E0FC0125913491C901A0E0B0E0841B73
:108CC000950BA60BB70B8093090290930A02A09311
:108CD0000B02B0930C02C0900902D0900A02E090FF
:108CE0000B02F0900C028091180790911907892BC4
:108CF00009F0E8C10E94FEC49093190780931807F9
:108D0000892B09F4DFC1E0911807F09119078081E0
:108D100083FF3EC085899689A789B08D8093821094
:108D200090938310A0938410B0938510818D928DC1
:108D3000A38DB48D8093861090938710A093881094
:108D4000B0938910858D968DA78DB0A180938A10E0
:108D500090938B10A0938C10B0938D1081A192A151
:108D6000A3A1B4A180938E1090938F10A093901024
:108D7000B09391109091B3098091B409981709F4B8
:108D8000B9CF8091B4098F5F8F708093B409B2CF4F
:108D9000C588D688E788F08C81E0C114D104E1044D
:108DA000F10409F480E0018D128D238D348D0115BD
:108DB00011052105310509F08260458D568D678DBD
:108DC00070A1411551056105710509F0846080931A
:108DD0005A0410928604109287041092880410920C
:108DE00089041092920410929304109294041092A9
:108DF000950485A196A1A7A1B0A580939A0490930C
:108E00009B04A0939C04B0939D048824992454014E
:108E1000881A990AAA0ABB0A809282049092830453
:108E2000A0928404B092850480927E0490927F0484
:108E3000A0928004B092810480927A0490927B0484
:108E4000A0927C04B0927D04809276049092770484
:108E5000A0927804B0927904CC0CDD1CEE1CFF1CAF
:108E6000C0926604D0926704E0926804F0926904AC
:108E7000000F111F221F331F00936A0410936B040D
:108E800020936C0430936D04440F551F661F771FA9
:108E900040936E0450936F04609370047093710458
:108EA00041A152A163A174A1440F551F661F771FF2
:108EB0004093720450937304609374047093750428
:108EC000880F991FAA1FBB1F8093620490936304AD
:108ED000A0936404B093650410929E0410929F04C2
:108EE0001092A0041092A10482A593A5A4A5B5A5F3
:108EF0008093960490939704A0939804B093990458
:108F000086A597A5A0A9B1A980938B0490938C0402
:108F1000A0938D04B0938E0481A580936104DF013A
:108F2000A95BBF4F9C9190939004992339F11596BA
:108F30002D913C9111973093600420935F04129718
:108F40002D913C91119730935E0420935D04109213
:108F50001102109212021092130210921402129730
:108F60002D913C91A90160E070E040930D02509377
:108F70000E0260930F02709310020CC088248A9432
:108F8000982C540180920D0290920E02A0920F0232
:108F9000B0921002EA5BFF4F90812091550492132A
:108FA0000AC02091080230E0482F082E000C550B13
:108FB0004217530731F090935504809308020E94A2
:108FC000D1C48091370581110E94E1BD2FEF3FEFA1
:108FD000A9012093090230930A0240930B02509397
:108FE0000C02E0911807F0911907DF01DE96ED9071
:108FF000FD900D911C9122A933A944A955A9EA5AC3
:10900000FF4F60817181828193810E947FC41092A1
:109010008A04E0911807F0911907EA5AFF4F8080FF
:109020009180A280B3808BE395E121E0FC01459122
:10903000559165917491481559056A057B0558F459
:10904000B694A79497948794220F0496A7E5B5E168
:10905000A817B90759F720939104B0E28B16910431
:10906000A104B10428F4B0E28B2E912CA12CB12CD8
:1090700030E2831A9108A108B108811448E09406EF
:10908000A104B10408F428C254E0959EC001112443
:10909000855C9E4EFC01329625913491782D662791
:1090A000739FA001729F410D561F0694461F561FC5
:1090B0001124FC01C590D490E12CF12CC41AD50ADE
:1090C000E108F108C092A204D092A304E092A404A3
:1090D000F092A5040091A2041091A3042091A4048D
:1090E0003091A50440911102509112026091130237
:1090F00070911402F02E198BF22FE32F40175107B5
:109100006207730720F4F42E598BF62FE72F8F2D6B
:109110009989AF2FBE2F0097E1E0AE07B10520F08F
:109120008FEF9FEFA0E0B0E0081B190B2A0B3B0B61
:109130000093A2041093A3042093A4043093A504E5
:109140004F3FFFEF5F076F077F0761F0481B590B29
:109150006A0B7B0B4093110250931202609313022F
:1091600070931402F8942091840030918500205F60
:109170003F4F4A8941504A8B442341F0280E391E03
:109180002216330610F40C94603F01C0190130928E
:10919000890020928800789462960FB6F894DEBF1A
:1091A0000FBECDBFDF91CF911F910F91FF90EF9038
:1091B000DF90CF90BF90AF909F908F907F906F90F7
:1091C0005F904F903F902F90089580910B01809574
:1091D0008870809309010C946C4080910B01887019
:1091E000809309016BC839893093910480E2881615
:1091F0009104A104B10428F430E2832E912CA12C17
:10920000B12C30E2831A9108A108B108811488E0DA
:109210009806A104B10420F1E4E09E9EC00111244F
:10922000855C9E4EFC01329625913491F82DEE27F7
:10923000F39F7001F29FE10CFE1E0694EE1EFE1ECF
:109240001124FC01C590D490860120E030E0480153
:1092500059018E189F08A108B1087501640122C048
:10926000950184013695279517950795F801EC7FB0
:10927000CF01855C924FFC01C590D490FC013296E1
:1092800025913491E82DE770E29FC001E39F900D96
:10929000112423E0969587952A95E1F7C81AD90AF3
:1092A000E12CF12C4C0D5D1D6E1D7F1D4093920431
:1092B0005093930460939404709395049091900458
:1092C00080918F04992309F474C0882309F40BCD8D
:1092D000A85BBF4F8D919C91A0E0B0E040910D0242
:1092E00050910E0260910F02709110028417950741
:1092F000A607B70709F060C0F6CCB695A795979575
:109300008795D988DD0CD98A2C5F3F4F47E555E119
:109310004217530709F04ACC59895093910480327F
:109320009105A105B10520F480E290E0A0E0B0E055
:109330008097A109B109811558E09507A105B105EC
:1093400008F443C074E0979F90011124255C3E4EC1
:10935000F901329645915491EE27859FB001849F83
:10936000610D7E1F06946E1F7E1F1124F901C590AA
:10937000D490E12CF12CC61AD70AE108F1088091AB
:10938000860490918704A0918804B09189048C0D83
:109390009D1DAE1DBF1D8093860490938704A093EE
:1093A0008804B093890480919004811130C0809129
:1093B0008F04882309F497CC1092110210921202A4
:1093C00010921302109214028ECCAC01BD0176955E
:1093D000679557954795FA01EC7F9F01255C324FC1
:1093E000F901C590D490F901329645915491877056
:1093F000849F9001859F300D1124F3E036952795C9
:10940000FA95E1F7C21AD30AE12CF12CB8CF898979
:10941000480E511C611C711C80911807909119070E
:10942000481459046A047B04D8F420918F04222341
:1094300009F459CCFC01E85BFF4F20813181A9017F
:1094400060E070E000910D0210910E0220910F0279
:1094500030911002401751076207730709F443CC9B
:109460001092110210921202109213021092140222
:10947000FC01E85BFF4F80819181A0E0B0E0809328
:109480000D0290930E02A0930F02B09310022BCC0A
:10949000D701C601B695A79597958795FC01EC7FF6
:1094A000CF01855C924FFC0125913491FC013296ED
:1094B000459154916C2D6770649FC001659F900D1C
:1094C000112463E0969587956A95E1F7281B390B7F
:1094D000C901A0E0B0E0F7CBD501C401B695A795CE
:1094E00097958795FC01EC7FCF01855C924FFC013D
:1094F000C590D490FC01329625913491482D477047
:10950000429FC001439F900D1124A3E0969587953B
:10951000AA95E1F7C81AD90AE12CF12CD3CD80ED38
:10952000C82E87E0D82EE12CF12CE4CBCF92DF922D
:10953000EF92FF92CF93DF936B017C01EA0121E36D
:1095400038E040EA50EC0E94C8EC87FD23C022E4DA
:1095500030E04CE553E4C701B6010E9456E6181608
:10956000CCF0C880D980EA80FB802FE632E143E866
:109570005AEBC701B6010E94C8EC87FD0BC0C1E0E1
:1095800022E430E04CE553E4C701B6010E9456E600
:1095900018160CF4C0E08C2FDF91CF91FF90EF9064
:1095A000DF90CF9008950F931F93CF93DF93FC012B
:1095B000A685B7858D0100581F4FE80188819981E4
:1095C00001968F779927AD014E575F4FEA012881A9
:1095D000398128173907D1F3E80128813981A20F91
:1095E000B31F6C93A685B785A058BF4F11969C9367
:1095F0008E93A689B7892C9181E090E0078C02C0F8
:10960000880F991F0A94E2F7822B8C9381E081A343
:109610000488F589E02D80818064808381E090E07A
:10962000DF91CF911F910F910895FC0181A18823B3
:1096300029F0A489B5898C9186FFFBCF11A20895EA
:10964000FC01A485B585FD01E058FF4F20813181E3
:109650003296808191812817390779F08081918134
:10966000A80FB91F8C91208131812F5F3F4F2F7739
:1096700033273183208390E008958FEF9FEF089583
:10968000DC011C96ED91FC911D97DF01A058BF4FA6
:109690002D913C91119712968D919C9111972817BD
:1096A000390739F08D919C91E80FF91F808190E086
:1096B00008958FEF9FEF0895FC0124853585F9010A
:1096C000E058FF4F8081918132962081318180580E
:1096D0009F4F821B930B60E870E00C948BED089514
:1096E000089580E090E00895CF92DF92EF92FF928C
:1096F000C0903002D0903102E0903202F0903302FC
:10970000FC0180819181A281B3818093300290938A
:109710003102A0933202B09333020E9475CAC09204
:109720003002D0923102E0923202F0923302FF9086
:10973000EF90DF90CF9008958091961890919718B0
:10974000981759F0E92FF0E0EA5EF74E80819F5FAD
:109750009F779093971890E008958FEF9FEF08956B
:109760001F920F920FB60F9211240BB60F922F93E8
:109770008F939F93EF93FF9320919718E091961802
:1097800081E08E0F8F779091C600281729F0F0E0C6
:10979000EA5EF74E9083E82FE0939618FF91EF91E1
:1097A0009F918F912F910F900BBE0F900FBE0F9036
:1097B0001F9018958091210490912204009731F018
:1097C0004AE050E060E070E00C94AAE360E070E0F2
:1097D000CB010895EFDF97FD0AC0ECDF6F3F710505
:1097E0008105910509F02CF4E5DF862F089580E0CE
:1097F00008958FEF08958091210490912204892B80
:1098000031F0E8DF91E0811103C090E001C091E008
:10981000892F08950F931F93CF93809121049091E6
:109820002204009711F1FC018F01C1912C2F2F7D93
:10983000A9F0C53411F0C536B9F7F801108260E01F
:1098400070E080912104909122040E9457E2F80177
:10985000C083562F472F382F292F0BC060E070E0B0
:10986000CF911F910F910C9457E250E040E030E00F
:1098700020E0652F742F832F922FCF911F910F918E
:10988000089581548A3108F042C0E82FF0E04091F9
:109890000D1850910E1860910F187091101804C097
:1098A00076956795579547958A95D2F7842F81705D
:1098B00040FF2FC0ED50F84E9081992309F1E091BF
:1098C0007210F0917310E90FF11D908120ED290FB6
:1098D0002A3098F09E3211F491810CC09D3211F023
:1098E0009B3271F4918120ED290F2A3030F09E32A5
:1098F00039F4928190539A3018F42E2F9F2F02C082
:1099000020E090E02093210490932204089580E0C9
:1099100008950895B6DF882341F081E02091210465
:1099200030912204232B09F480E0089580E1E2E3E2
:10993000F4E0AEEAB0E101900D928A95E1F7089566
:109940002F923F924F925F926F927F928F929F924F
:10995000AF92BF92CF92DF92EF92FF920F931F933D
:10996000CF93DF9300D01F921F92CDB7DEB77C015B
:109970008B016A0119018090320490903304A09009
:109980003404B0903504A5019401FC01608171811B
:10999000828193810E9456E6F1E0FD83811112C01D
:1099A00020913604309137044091380450913904A5
:1099B000F80160817181828193810E9456E6811154
:1099C00001C01D82F6014080518062807380209129
:1099D0001502309116024091170250911802C301EE
:1099E000B2010E9456E6882309F453C04092150242
:1099F00050921602609217027092180220E030E036
:109A000040E450E46091FB067091FC068091FD06F5
:109A10009091FE060E947EEB69837A838B839C8300
:109A20008092AE109092AF10A092B010B092B11090
:109A30008091360490913704A0913804B091390494
:109A40008093B2109093B310A093B410B093B5105C
:109A5000F60180819181A281B3818093B6109093A9
:109A6000B710A093B810B093B91080913E049091B4
:109A70003F04A0914004B09141048093BA109093A8
:109A8000BB10A093BC10B093BD10CE0101962CDE8C
:109A90004DDFFD81FF2309F16090F7067090F80615
:109AA0008090F9069090FA06A090F306B090F40624
:109AB000C090F506D090F6069501A601B301C40149
:109AC0000E94C8EC181614F05301640120E030E045
:109AD00040E251E4B501C6010CC020E030E040ECAA
:109AE0005FE36091FF0670910007809101079091FC
:109AF00002070E947EEB69837A838B839C8320918B
:109B00002004222349F0AB01BC018BE595E10E94C2
:109B100050C58AE00E94E093F70180819181A28183
:109B2000B3818093AE109093AF10A093B010B09318
:109B3000B110F80180819181A281B3818093B2102C
:109B40009093B310A093B410B093B510F10120819D
:109B50003181428153816091BA107091BB10809124
:109B6000BC109091BD100E94A2EA6093BA1070934D
:109B7000BB108093BC109093BD10CE010196B4DD54
:109B8000D5DE0F900F900F900F900F90DF91CF9137
:109B90001F910F91FF90EF90DF90CF90BF90AF900B
:109BA0009F908F907F906F905F904F903F902F90FD
:109BB000089580E1EEEAF0E1A2E3B4E001900D92B5
:109BC0008A95E1F708959C0197FD0EC084369105B2
:109BD00084F064E670E00E948BEDCB016AE070E0F7
:109BE0000E948BED805D06C03195219531098DE293
:109BF00001C080E280932D042A30310564F0EAE050
:109C0000F0E0C901BF010E948BEDCB01BF010E94B2
:109C10008BED805D01C080E280932E04C9016AE073
:109C200070E00E948BED805D80932F048DE294E0C4
:109C300008958E3691051CF02EE680E002C0282F94
:109C4000892F20934404809345040C94A9762F9285
:109C50003F924F925F926F927F928F929F92AF92BC
:109C6000BF92CF92DF92EF92FF920F931F93CF9309
:109C7000DF93CDB7DEB7C455D1090FB6F894DEBF78
:109C80000FBECDBFEAE1F8E184918F010F5F1F4F56
:109C9000882321F00E94E093F801F6CF0E9485B45A
:109CA00081110C94095880E090E0A0E8BFE3809314
:109CB000A6109093A710A093A810B093A91080E0CD
:109CC00090E0A0E8B0E48093AA109093AB10A0932A
:109CD000AC10B093AD108DEC9CECACE4BEE3809383
:109CE000A2109093A310A093A410B093A51080E0AD
:109CF00090E0A8ECB1E48093240590932505A0930F
:109D00002605B09327058CE390E09093230580937C
:109D1000220588EC90E09093210580932005109215
:109D20001F058FE4F7DD882311F074DD04C060E0C7
:109D300070E080E190E46BAF7CAF8DAF9EAF83E4C9
:109D4000E9DD882311F057DD02C083E49ADD6196D6
:109D50008FAF61978BE4DEDD882311F04CDD02C00C
:109D60008BE48FDD60968FAF609782E4D3DD88232C
:109D7000E9F050DD0E94E6EB709323056093220525
:109D80006115710599F0685271096536710570F0B9
:109D9000E5EEF7E184918F010F5F1F4F882311F4E7
:109DA0000C9409580E94E093F801F4CF8CE4B2DDE2
:109DB000882351F12FDD6B017C016093A210709319
:109DC000A3108093A4109093A51020E030E0A90187
:109DD0000E94C8EC87FD0AC020E030E040E050E47B
:109DE000C701B6010E9456E6181674F4EDEBF7E1D0
:109DF00084918F010F5F1F4F882311F40C94095831
:109E00000E94E093F801F4CF81E53BDD882309F45B
:109E100040C08091210490912204892B19F4E2E939
:109E2000F7E12BC0F7DC6B017C016093AA10709303
:109E3000AB108093AC109093AD102DEC3CEC4CE447
:109E40005DE30E94C8EC87FD0AC020E030E040E7F7
:109E500051E4C701B6010E9456E61816D4F4E1E6B3
:109E6000F7E184918F010F5F1F4F882311F40C9449
:109E700009580E94E093F801F4CF84918F010F5F9D
:109E80001F4F882311F40C9409580E94E093F801A5
:109E9000F4CF83E53FDD882319F1BCDC4B015C0185
:109EA0002DEC3CEC4CEC5DE30E94C8EC87FD0AC055
:109EB00020E030E040E85FE3C501B4010E9456E6CF
:109EC0001816ACF4EAE3F7E184918F010F5F1F4F9E
:109ED000882311F40C9409580E94E093F801F4CF00
:109EE0005DEC852E5CEC952EA92C5EE3B52E80E50D
:109EF000C8DC882309F443C0809121049091220496
:109F0000892B71F4E2E0F7E184918F010F5F1F4F1D
:109F1000882311F40C9409580E94E093F801F4CFBF
:109F200080911F058F5F80931F0574DC6B017C019E
:109F3000609324057093250580932605909327054B
:109F400020E030E0A9010E94C8EC87FD0AC020E0B3
:109F500030E048EC51E4C701B6010E9456E61816FD
:109F600074F4EAEDF6E184918F010F5F1F4F8823AF
:109F700011F40C9409580E94E093F801F4CF86E4A0
:109F8000C9DC882319F146DC6B017C0120E030E05C
:109F900040E85FE30E94C8EC87FD0AC020E030E0A3
:109FA00040E850E4C701B6010E9456E61816A4F432
:109FB000E1EBF6E184918F010F5F1F4F882311F4CD
:109FC0000C9409580E94E093F801F4CFC12CD12CD5
:109FD00040EEE42E4FE3F42EA7019601C701B6012F
:109FE0000E94BBE69B01AC0160E070E084E490E479
:109FF0000E947EEB2091A6103091A7104091A810EE
:10A000005091A9100E94BBE62B013C01A5019401CF
:10A01000C501B4010E94BBE6A70196010E94BBE600
:10A020002CEE31E548EB5DE30E947EEB9B01AC0139
:10A03000C301B2010E94BBE66093A6107093A71003
:10A040008093A8109093A91088E464DC8823C9F059
:10A05000E1DB0E94E6EB7093210560932005655AD1
:10A0600071096437710568F0E3E8F6E184918F01C6
:10A070000F5F1F4F882309F4CCC70E94E093F801BB
:10A08000F5CF85E5FEDB8823E9F00E94F1586115E4
:10A0900071058105910511F00E944EE28091210425
:10A0A00090912204892B11F0B5DB04C060E070E0D0
:10A0B00088E492E460931B0570931C0580931D0552
:10A0C00090931E0582E5DDDB81110DC0EFE4F6E122
:10A0D00084918F010F5F1F4F882309F49AC70E9454
:10A0E000E093F801F5CF8091210490912204892B0F
:10A0F000A9F060DB2F967FAF6EAF2F97161617066D
:10A100009CF0EBE1F6E184918F010F5F1F4F8823F4
:10A1100009F47FC70E94E093F801F5CF8AE190E04F
:10A120002F969FAF8EAF2F9788E5F4DB882361F0E1
:10A1300071DB209114043091150440911604509164
:10A1400017040E94A1EA08C06091320470913304A0
:10A15000809134049091350460931705709318052D
:10A160008093190590931A0589E5D4DB882361F063
:10A1700051DB209118043091190440911A04509138
:10A180001B040E94A1EA08C0609136047091370454
:10A1900080913804909139046093130570931405ED
:10A1A0008093150590931605609117057091180519
:10A1B0008091190590911A0543E155E0B7D98111B5
:10A1C0000DC0E1EFF5E184918F010F5F1F4F8823F0
:10A1D00009F41FC70E94E093F801F5CF84E451DB36
:10A1E00091E089270E9448AC20E030E040EA50E44A
:10A1F00060913A0470913B0480913C0490913D043D
:10A200000E9456E687FF14C0198A1A8A1B8A1C8A84
:10A2100080E090E0A0EAB0E489839A83AB83BC83BA
:10A22000BE016F5E7F4FCE0101960E9467B4C1DC14
:10A23000D8D76B017C01A8E8CA0EA3E1DA1EE11CA5
:10A24000F11C8091220590912305F3DC6091220599
:10A2500070912305072E000C880B990B0E945CE679
:10A260009B01AC01609146047091470480914804C1
:10A27000909149040E94A1EA4B015C0120E030E08A
:10A28000A9010E94C8EC87FF04C0B7FAB094B7F8E0
:10A29000B09420E030E040E450E4C501B4010E94F5
:10A2A000C8EC1816F4F49DD7DC01CB018C199D097C
:10A2B000AE09BF09B7FD0EC094D76B017C01B8E8A9
:10A2C000CB0EB3E1DB1EE11CF11C0E94EF758AE0AE
:10A2D0000E94E0930E941EA1809196188093971887
:10A2E000B5CF80912005909121050E94E65960919B
:10A2F000200570912105072E000C880B990B0E94F8
:10A300005CE69B01AC0160914C0470914D0480911E
:10A310004E0490914F040E94A1EA4B015C0120E0A1
:10A3200030E0A9010E94C8EC87FF04C0B7FAB094DE
:10A33000B7F8B09420E030E040E450E4C501B40147
:10A340000E94C8EC1816F4F44CD7DC01CB018C1930
:10A350009D09AE09BF09B7FD0EC043D76B017C0153
:10A36000E8E8CE0EE3E1DE1EE11CF11C0E94EF7571
:10A370008AE00E94E0930E941EA18091961880932B
:10A380009718B5CF10923E0410923F0410924004EB
:10A39000109241040E9436B380911F05882399F1E1
:10A3A000C5DA20912405309125054091260550916C
:10A3B00027056091BA107091BB108091BC109091EC
:10A3C000BD100E94A2EA6093BA107093BB108093F4
:10A3D000BC109093BD1020E030E040E751E4609164
:10A3E000FF067091000780910107909102070E947B
:10A3F0007EEB69837A838B839C83CE01019674D92B
:10A4000095DA0E9443B180E2E3EFF4E0DF01282F08
:10A410001D922A95E9F7E3EDF4E0DF01282F1D9264
:10A420002A95E9F7E3EBF4E0DF011D928A95E9F75D
:10A430007DDA8091A2109091A310A091A410B09108
:10A44000A5108093B6109093B710A093B810B09356
:10A45000B91019821A821B821C829E012F5F3F4F06
:10A4600046EB50E162EB70E18EEA90E169DA9E0121
:10A47000255C3F4F46EB50E162EB70E18EEA90E1E4
:10A480005FDA6196BFAD6197BB2329F066E374E0A4
:10A4900082E394E004C063E175E087E195E00E9407
:10A4A000A6D8298F3A8F4B8F5C8F6D8F7E8F3FAFF1
:10A4B0002D962FAF2D972D96EFAD2D97E7FD81C4EB
:10A4C000FFADF7FD7EC424E0E202F0011124E35069
:10A4D000F64F40805180628073803FAD84E0380247
:10A4E000F0011124E751F64FD080C18032802380E3
:10A4F0008D2D9C2DA32DB22D8FAB98AFA9AFBAAFE8
:10A50000AE01495C5F4FB201C30110D8882309F442
:10A510005CC420E030E040EA50E4B201C3010E9494
:10A52000A2EAF62E072F182FE92E862F902FA12FA3
:10A53000BE2D8BAB9CABADABBEAB8D2D9C2DA32D9F
:10A54000B22D8FA798ABA9ABBAAB2D969FAD2D9727
:10A55000911152C0AFADA11105C05F2D402F312F19
:10A560002E2D04C0542D452D362D272D852F942FAB
:10A57000A32FB22F8BAB9CABADABBEABBFADB4309A
:10A5800034F4F42C052D162DE72CBB2369F020E0C4
:10A5900030E040EA50E46D2D7C2D832D922D0E94F9
:10A5A000A1EA362F272F03C09601832D922D432F2A
:10A5B000522FBC014FA758AB69AB7AABEFADE4307B
:10A5C0000CF0A7C020E030E040EA50E46D2D7C2D77
:10A5D000832D922D0E94A2EA21966FAF2197239698
:10A5E0007FAF239725968FAF259727969FAF279705
:10A5F000FFADF11185C099C02D962FAD2D97243058
:10A600000CF453C03FAD34305CF020E030E040EA61
:10A6100050E4B201C3010E94A1EA362F272F03C0E4
:10A62000342D252DC301432F522FBC014BAB5CAB06
:10A630006DAB7EAB8FAD8111E3C420E030E040EA2A
:10A6400050E4B201C3010E94A1EAF62E072F182F91
:10A65000E92E20E030E040EA50E46D2D7C2D832D82
:10A66000922D0E94A2EA6FA778AB89AB9AAB9FADFF
:10A67000992309F44EC020E030E040EA50E46D2D0B
:10A680007C2D832D922D0E94A1EA21966FAF2197F8
:10A6900023967FAF239725968FAF259727969FAF59
:10A6A0002797AFADA43064F140C0BFADB1110DC06C
:10A6B00020E030E040EA50E4B201C3010E94A1EA88
:10A6C000F62E072F182FE92E0FC0EFADE430B4F1AE
:10A6D00020E030E040EA50E4B201C3010E94A1EA68
:10A6E0006BAB7CAB8DAB9EAB2196DFAE21972396F7
:10A6F000CFAE239725963FAE259727962FAE279767
:10A7000032ED832E33E5932E3BE7A32E31E4B32EB7
:10A7100029C02196DFAE21972396CFAE23972596A9
:10A720003FAE259727962FAE279722ED822E23E561
:10A73000922E2BEFA22E20E4B22E14C02196DFAE73
:10A7400021972396CFAE239725963FAE2597279640
:10A750002FAE279792ED892E93E5992E9BEFA92E88
:10A7600091E4B92E8BA99CA9ADA9BEA92C968CAF5A
:10A770009DAFAEAFBFAF2C979C01AD01B201C3013D
:10A780000E94A1EA698B7A8B8B8B9C8B4FA458A873
:10A7900069A87AA8A30192016D2D7C2D832D922D9D
:10A7A0000E94A1EA6D8B7E8B8F8B988F2C962CAD9F
:10A7B0003DAD4EAD5FAD2C97609132047091330486
:10A7C00080913404909135040E94A1EA2C966CAFDC
:10A7D0007DAF8EAF9FAF2C97A3019201609136049D
:10A7E0007091370480913804909139040E94A1EA55
:10A7F0002B013C018F2D902FA12FBE2D89839A8391
:10A80000AB83BC8321968FAD219723969FAD239771
:10A810002596AFAD25972796BFAD27978D839E834D
:10A82000AF83B8878091A2109091A310A091A4103B
:10A83000B091A51089879A87AB87BC872DEC3CEC3B
:10A840004CEC5CE3C501B4010E94BBE62091A6106C
:10A850003091A7104091A8105091A9100E94BBE61A
:10A8600020913E0430913F044091400450914104B6
:10A870000E94A2EA6D877E878F87988B2C962CADDD
:10A880003DAD4EAD5FAD2C97CA01B9010E94BBE64C
:10A890006B017C01A3019201C301B2010E94BBE6DE
:10A8A0009B01AC01C701B6010E94A2EA20E030E0A2
:10A8B00040E050E40E94C8EC18160CF046C00E941C
:10A8C00043B11BA21CA21DA21EA220E030E040E06A
:10A8D0005FE360913A0470913B0480913C04909155
:10A8E0003D040E94A2EA6F8F78A389A39AA39E01D8
:10A8F0002D5D3F4FAE01415E5F4F66E374E082E342
:10A9000094E01ED81BA21CA21DA21EA220E030E0D3
:10A9100040E05FE36091A2107091A3108091A410B9
:10A920009091A5100E94A2EA6F8F78A389A39AA3A1
:10A930009E012D5D3F4FAE01415E5F4FBE01615DE7
:10A940007F4FCE01C3960E94A04C1F8E18A219A261
:10A950001AA29E01215E3F4F42EA50E1BE01615DB5
:10A960007F4FCE01C3960E94A04C0E946FB14090D1
:10A970003002509031026090320270903302E090C9
:10A98000F706F090F8060091F9061091FA06A090EB
:10A99000F306B090F406C090F506D090F606950147
:10A9A000A601B701C8010E94C8EC181614F475017D
:10A9B000860120E030E040E251E4B701C8010E9486
:10A9C0007EEB609330027093310280933202909359
:10A9D000330240E0BE016F5E7F4FCE0101960E94C0
:10A9E000EAA4409230025092310260923202709298
:10A9F00033020E94964CADEFB9E02496BFAFAEAFE4
:10AA0000249722961FAE1EAE229701E010E02196F9
:10AA10000FAC219702C0000F111F0A94E2F7229693
:10AA2000EEADFFAD229731962296FFAFEEAF2297A3
:10AA300021E030E021960FAC219702C0220F331F96
:10AA40000A94E2F763963FAF2EAF639783EB282E0D
:10AA500084E0382E83EF94E02A969FAF8EAF2A973A
:10AA6000A3EDB4E02896BFAFAEAF2897E9EEF9E0CA
:10AA70002696FFAFEEAF26972A962EAD3FAD2A97CA
:10AA800065963FAF2EAF6597D9018D919C919C0142
:10AA900020233123232B09F4ADC06396EEADFFAD27
:10AAA00063978E239F23892B09F4A4C02896AEAD0B
:10AAB000BFAD28978D919C9180239123892B09F01C
:10AAC00099C020E030E040E050E42496AEADBFAD48
:10AAD00024976D917D918D919C910E94A2EA6B01CA
:10AAE0007C0120E030E040E050E42496EEADFFAD84
:10AAF000249764817581868197810E94A1EA4B0128
:10AB00005C0120E030E040E850ECC701B6010E9453
:10AB100056E687FD70C120E030E04BE553E4C70105
:10AB2000B6010E94C8EC181634F4C12CD12CBBE538
:10AB3000EB2EB3E4FB2ECBA6DCA6EDA6FEA6269656
:10AB4000AEADBFAD26974D905D906D907C9020E0AE
:10AB500030E040E85FE3C301B2010E9456E687FDA2
:10AB600051C120E030E04BE553E4C301B2010E9443
:10AB7000C8EC181634F4412C512CFBE56F2EF3E48D
:10AB80007F2E4F8E58A269A27AA24FA258A669A61C
:10AB90007AA620E030E040E850ECC501B4010E9404
:10ABA00056E687FD36C120E030E04BE553E4C501B1
:10ABB000B4010E94C8EC181634F4812C912C7BE56A
:10ABC000A72E73E4B72E8BA29CA2ADA2BEA2AE01AB
:10ABD000495D5F4FC701B6010E94964A811120C1AD
:10ABE0002896EEADFFAD289780819181802B912B27
:10ABF000918380832A962EAD3FAD2A972E5F3F4FDB
:10AC00002A963FAF2EAF2A976596AEADBFAD65973A
:10AC10008D919C9180239123892B09F4A6C0F90181
:10AC20008081918180239123892B09F49EC0F101B9
:10AC30008081918180239123892B09F096C020E0A7
:10AC400030E040E050E42696AEADBFAD26976D9162
:10AC50007D918D919C910E94A2EA2B013C0120E004
:10AC600030E040E050E42696EEADFFAD26976481DB
:10AC70007581868197810E94A1EA4B015C0124962F
:10AC8000AEADBFAD2497CD90DD90ED90FC9020E06F
:10AC900030E040E850ECC701B6010E9456E687FD5F
:10ACA000FFC020E030E04BE553E4C701B6010E944D
:10ACB000C8EC181634F4C12CD12C5BE5E52E53E416
:10ACC000F52ECBA2DCA2EDA2FEA2CBA6DCA6EDA6C1
:10ACD000FEA620E030E040E85FE3C301B2010E943D
:10ACE00056E687FDE4C020E030E04BE553E4C301C5
:10ACF000B2010E94C8EC181634F4412C512C3BE5EB
:10AD0000632E33E4732E4FA258A669A67AA620E0DC
:10AD100030E040E85FE3C501B4010E9456E687FDDC
:10AD2000CDC020E030E04BE553E4C501B4010E9402
:10AD3000C8EC181634F4812C912C9BE5A92E93E4D1
:10AD4000B92E8F8E98A2A9A2BAA2AE01495D5F4F1B
:10AD5000C701B6010E94964A8111B7C0F1018081F6
:10AD60009181802B912B91838083F2E02F0E311CF7
:10AD700028962EAD3FAD28972E5F3F4F28963FAFC8
:10AD80002EAF289726968EAD9FAD269704962696D1
:10AD90009FAF8EAF26979DEB291694E0390609F0F8
:10ADA0006BCE2496AEADBFAD249714962496BFAF5C
:10ADB000AEAF24972296EEADFFAD2297359709F0FE
:10ADC00024CE80919618809397182F962EAD3FAD84
:10ADD0002F97215031092F963FAF2EAF2F97232B5E
:10ADE00009F4B3C02D963FAD2D9737FDAEC08FADA2
:10ADF00087FF47CBAAC0C12CD12CA0E8EA2EA0EC3B
:10AE0000FA2E99CE412C512CE0E86E2EEFE37E2EE7
:10AE1000B8CE812C912C60E8A62E60ECB62ED3CE55
:10AE2000AE01415E5F4FC501B4010E94964A88237E
:10AE300009F4D6CE80912004882321F1B701A60120
:10AE40008BEC95E10E9450C54FA158A569A57AA544
:10AE500085EC95E10E9450C54BA15CA16DA17EA13E
:10AE60008BEB95E10E9450C54F8D58A169A17AA145
:10AE700085EB95E10E9450C589E20E94E0938AE04B
:10AE80000E94E0939E01215E3F4FAE014D5D5F4FFA
:10AE9000BE01695D7F4FCE018B960E949FB1A0CE0F
:10AEA000C12CD12C40E8E42E40ECF42E0ACF412CEA
:10AEB000512C20E8622E2FE3722E25CF812C912C6D
:10AEC00080E8A82E8FE3B82E3CCFAE01415E5F4FE5
:10AED000C701B6010E94964A882309F43FCF8091AA
:10AEE0002004882321F1B701A60181E995E10E94A0
:10AEF00050C54FA158A569A57AA58BE895E10E9498
:10AF000050C54BA15CA16DA17EA181E895E10E9495
:10AF100050C54F8D58A169A17AA18BE795E10E9498
:10AF200050C589E20E94E0938AE00E94E0939E016E
:10AF3000215E3F4FAE014D5D5F4FBE01695D7F4FAA
:10AF4000CE018B960E949FB109CF0E9443B180E051
:10AF500090E0A0EAB0E48093B6109093B710A0936D
:10AF6000B810B093B91019821A821B821C829E01FC
:10AF70002F5F3F4F46EB50E162EB70E18EEA90E1CC
:10AF80000E94A04C8091170590911805A091190579
:10AF9000B0911A058093AE109093AF10A093B010AB
:10AFA000B093B1108091130590911405A0911505EF
:10AFB000B09116058093B2109093B310A093B41083
:10AFC000B093B51019821A821B821C829E012F5FDA
:10AFD0003F4F46EB50E162EB70E18EEA90E10E9458
:10AFE000A04C6096FFAD6097F11113C0109245041C
:10AFF000109244040E94A97680E090E0E7D109C055
:10B000002FADF42C052D162DE72C24300CF033CB6E
:10B0100020CBCC5ADF4F0FB6F894DEBF0FBECDBFAA
:10B02000DF91CF911F910F91FF90EF90DF90CF9024
:10B03000BF90AF909F908F907F906F905F904F9058
:10B040003F902F9008951F920F920FB60F921124E8
:10B050000BB60F922F933F938F939F93EF93FF9392
:10B060002091120F3091130F8091140F9091150FB2
:10B070002817390731F4809131018F7D8093310198
:10B0800014C0E091140FF091150FEE56F14F20818E
:10B090008091140F9091150F01968F7799279093B7
:10B0A000150F8093140F20933601FF91EF919F911C
:10B0B0008F913F912F910F900BBE0F900FBE0F906D
:10B0C0001F9018951F920F920FB60F9211240BB676
:10B0D0000F922F934F935F938F939F93EF93FF93D1
:10B0E0008091300182FD1CC0209136018091960F25
:10B0F0009091970F4091980F5091990F01968F77EB
:10B1000099274817590771F0E091960FF091970F22
:10B11000EA5EF04F20839093970F8093960F02C0C2
:10B1200080913601FF91EF919F918F915F914F91A7
:10B130002F910F900BBE0F900FBE0F901F90189580
:10B14000CF92DF92EF92FF920F931F93CF93DF93F3
:10B150006C017A018B01C0E0D0E0CE15DF0581F0F3
:10B16000D8016D918D01D601ED91FC910190F08196
:10B17000E02DC6011995892B11F02196EECF7E01A5
:10B18000C701DF91CF911F910F91FF90EF90DF905A
:10B19000CF9008950E94B2ED3FB7F8948091CF060A
:10B1A0009091D006A091D106B091D20626B5A89B69
:10B1B00005C02F3F19F00196A11DB11D3FBFBA2F49
:10B1C000A92F982F8827820F911DA11DB11DBC01A9
:10B1D000CD0142E0660F771F881F991F4A95D1F76E
:10B1E00008952FB7F8946091CB067091CC068091AA
:10B1F000CD069091CE062FBF08951F920F920FB6E5
:10B200000F9211242F933F938F939F93AF93BF93EC
:10B210008091CB069091CC06A091CD06B091CE0640
:10B220003091CA0623E0230F2D3720F40196A11D8B
:10B23000B11D05C026E8230F0296A11DB11D209364
:10B24000CA068093CB069093CC06A093CD06B0930C
:10B25000CE068091CF069091D006A091D106B091F4
:10B26000D2060196A11DB11D8093CF069093D00602
:10B27000A093D106B093D206BF91AF919F918F91C9
:10B280003F912F910F900FBE0F901F9018951F9216
:10B290000F920FB60F9211240BB60F922F933F937C
:10B2A0004F935F936F937F938F939F93AF93BF93CE
:10B2B000EF93FF9380912B0590912C05A0912D0584
:10B2C000B0912E05892B8A2B8B2B59F190912A0551
:10B2D000E0912805F091290580818927808380915C
:10B2E0002B0590912C05A0912D05B0912E051816D7
:10B2F00019061A061B060CF056C080912B0590917A
:10B300002C05A0912D05B0912E050197A109B10939
:10B3100080932B0590932C05A0932D05B0932E05BB
:10B3200042C080911902E7E4F8E1E4919FEF909325
:10B330001902E230C9F050F4EE2399F0E13081F5C2
:10B3400090916F009D7F90936F002AC0E43019F1B7
:10B35000E0F0E53029F5909173009D7F90937300A4
:10B360001FC010926E001CC0909170009D7F909342
:10B37000700091E09093B0009091B100987F94603C
:10B380009093B1001092B3000BC0909171009D7F1B
:10B390009093710005C0909172009D7F9093720010
:10B3A00060E00E94FBB5FF91EF91BF91AF919F913B
:10B3B0008F917F916F915F914F913F912F910F905E
:10B3C0000BBE0F900FBE0F901F90189590934B04DB
:10B3D00080934A0480E00C94F5762F923F924F922E
:10B3E0005F926F927F928F929F92AF92BF92CF9215
:10B3F000DF92EF92FF920F931F93CF93DF93CDB71E
:10B40000DEB7C857D1090FB6F894DEBF0FBECDBF67
:10B41000E0914A07F0914B07EF2B11F00C94AD62CD
:10B420002896DFAECEAE28976E2C79016A015B01BB
:10B43000FC0120813181428153816C962CAF3DAF5C
:10B440004EAF5FAF6C972091921030919310409166
:10B450009410509195106C966CAD7DAD8EAD9FADF6
:10B460006C970E94BBE60E94D3ECE0966CAF7DAF78
:10B470008EAF9FAFE097D5018D919D910D90BC91BE
:10B48000A02DA0968CAF9DAFAEAFBFAFA09720917F
:10B490009610309197104091981050919910BC01DE
:10B4A000CD010E94BBE60E94D3ECE4966CAF7DAF69
:10B4B0008EAF9FAFE497D6012D913D914D915C9158
:10B4C000A4962CAF3DAF4EAF5FAFA49720919A10DA
:10B4D00030919B1040919C1050919D10A4966CADA2
:10B4E0007DAD8EAD9FADA4970E94BBE60E94D3ECCC
:10B4F000E8966CAF7DAF8EAF9FAFE897D7012D91E7
:10B500003D914D915C9122962CAF3DAF4EAF5FAF18
:10B51000229720919E1030919F104091A010509141
:10B52000A11022966CAD7DAD8EAD9FAD22970E948D
:10B53000BBE60E94D3EC60966CAF7DAF8EAF9FAF41
:10B5400060978091100783FF1CC060962CAD3DADC5
:10B550004EAD5FAD60972093E5093093E6094093C7
:10B56000E7095093E80922968CAD9DADAEADBFAD15
:10B5700022978093D5099093D609A093D709B093C9
:10B58000D809D801BC91B9A7F801F181F9ABD8016C
:10B590001296BC91BEABF801F381FAAF8091B3096A
:10B5A0009091B409891B8F708F3019F40E941EA1ED
:10B5B000F5CF0091B309E9960FAFE9978091B309F0
:10B5C000082F10E01CA30BA38091D9099091DA09F0
:10B5D000A091DB09B091DC09E0968CAC9DACAEACDF
:10B5E000BFACE097881A990AAA0ABB0A8091DD09C4
:10B5F0009091DE09A091DF09B091E009E4962CACAE
:10B600003DAC4EAC5FACE497281A390A4A0A5B0A93
:10B610008091E1099091E209A091E309B091E409D8
:10B62000E8962CAD3DAD4EAD5FADE897281B390BCC
:10B630004A0B5B0B2DA33EA34FA358A78091E509AE
:10B640009091E609A091E709B091E80960960CADE8
:10B650001DAD2EAD3FAD6097081B190B2A0B3B0BA0
:10B660000DA71EA72FA738AB012B022B032B09F424
:10B67000BCC080910F0781114BC060914C04709148
:10B680004D0480914E0490914F040E94E6EB20916E
:10B69000250230912602621773070CF039C06096BC
:10B6A0002CAD3DAD4EAD5FAD60972093E509309375
:10B6B000E6094093E7095093E80922968CAD9DADC9
:10B6C000AEADBFAD22978093D5099093D609A093D4
:10B6D000D709B093D809E4EEFDE184918F010F5FA3
:10B6E0001F4F811103C0EBEBF9E104C00E94E0930E
:10B6F000F801F3CF84918F010F5F1F4F882321F052
:10B700000E94E093F801F6CF1DA61EA61FA618AA58
:10B7100094E0699E800111240F5D1D4F6DA57EA5EB
:10B720008FA598A90E945CE6D8012D913D914D917D
:10B730005C910E94BBE66B017C0120E030E0A90136
:10B740000E94C8EC87FF04C0F7FAF094F7F8F09471
:10B7500060919E1070919F108091A0109091A11007
:10B760000E94E6EB9B01AC01A8ECB0E00E9482EAEB
:10B770000E945CE6A70196010E9456E687FF39C049
:10B7800060960CAD1DAD2EAD3FAD60970093E50901
:10B790001093E6092093E7093093E80922962CAD2F
:10B7A0003DAD4EAD5FAD22972093D5093093D609BC
:10B7B0004093D7095093D809E4EEFDE184918F01BD
:10B7C0000F5F1F4F811103C0ECE9F9E104C00E9433
:10B7D000E093F801F3CF84918F010F5F1F4F88230F
:10B7E00021F00E94E093F801F6CF1DA61EA61FA629
:10B7F00018AAD501C4018827B7FD83959927AA27E0
:10B80000BB27782E57FE03C0382F3260732E8DA1D0
:10B810009EA1AFA1B8A5B7FF03C0972D9460792E64
:10B820000DA51EA52FA538A937FF03C0172D186039
:10B83000712E24E0629E800111240F5D1D4F6DA5C5
:10B840007EA58FA598A90E945CE6D8012D913D9117
:10B850004D915C910E94BBE66B017C0120E030E0E1
:10B86000A9010E94C8EC87FF04C0C701B601905827
:10B8700002C0C701B60120E030E040E05FE30E9473
:10B88000A2EA0E94EBEB6AAB7BAB8CAB9DAB88E68C
:10B890000BA11CA1809FF001819FF00D1124E159A3
:10B8A000FE4E1082EA5BFF4F7082B501A401B7FE25
:10B8B00007C044275527BA01481959096A097B0965
:10B8C00088E60BA11CA1809FF001819FF00D11243F
:10B8D000E159FE4E458B568B678B708F2C962CAEA4
:10B8E0003DAE4EAE5FAE2C9757FE0DC08827992710
:10B8F000DC0182199309A409B5092C968CAF9DAF80
:10B90000AEAFBFAF2C9728E60BA11CA1209FF00182
:10B91000219FF00D1124E159FE4E2C968CAD9DAD6A
:10B92000AEADBFAD2C97818F928FA38FB48F0DA139
:10B930001EA12FA138A537FF07C03095209510957F
:10B9400001951F4F2F4F3F4FE8E67E2EABA1BCA1C4
:10B950007A9EF0017B9EF00D1124E159FE4E058F79
:10B96000168F278F30A38AA99BA9ACA9BDA981A353
:10B9700092A3A3A3B4A323964FAF2397752EF62FBC
:10B98000E72F2C968CAD9DADAEADBFAD2C97481773
:10B9900059076A077B0778F429969FAD2997239664
:10B9A0009FAF23972A967FAC2A972B96FFAD2B97B4
:10B9B0002C96EFAD2C9723968FAD2397972DAF2F15
:10B9C000BE2F80179107A207B30710F4D901C80151
:10B9D0000AA91BA92CA93DA980179107A207B307A3
:10B9E00010F4D901C80128E60BA11CA1209FF00189
:10B9F000219FF00D1124E159FE4E85A396A3A7A324
:10BA0000B0A70697A105B10508F4A0C5DF01AE599E
:10BA1000BF4F80914204909143048D939C9361A603
:10BA2000452B462B472B09F05F9888E60BA11CA1FC
:10BA3000809FF001819FF00D1124E159FE4E818D10
:10BA4000928DA38DB48D892B8A2B8B2B11F08A9824
:10BA5000479888E60BA11CA1809FF001819FF00D03
:10BA60001124E159FE4E858D968DA78DB0A1892BAD
:10BA70008A2B8B2B31F08091080181708093060115
:10BA800047982AA93BA94CA95DA9232B242B252B38
:10BA900009F465C580911507882319F081508093BA
:10BAA0001507611004C0129880E28093150760901A
:10BAB0000B0770900C0700910D0710910E07930172
:10BAC000A80169A579A98EA99AAD0E9456E687FFBB
:10BAD00004C069A679AA0EAB1AAFC501B4010E94D1
:10BAE0005CE620915F11309160114091611150919D
:10BAF00062110E94BBE626966CAF7DAF8EAF9FAF02
:10BB00002697698B7A8B8B8B9C8BC201B1010E942B
:10BB10005CE6209163113091641140916511509160
:10BB200066110E94BBE62B013C016D8B7E8B8F8BD7
:10BB3000988F6DA17EA18FA198A50E945CE62091AF
:10BB40006711309168114091691150916A110E94FA
:10BB5000BBE64B015C01698F7A8F8B8F9C8F2091A4
:10BB60006B1130916C1140916D1150916E11C701A4
:10BB7000B6010E94BBE66B017C016D8F7E8F8F8FBB
:10BB800098A388E60BA11CA1809FF001819FF00D76
:10BB90001124E159FE4E258936894789508D2DA300
:10BBA0003EA34FA358A7263031054105510508F49F
:10BBB000DFC42896AEADBFAD2897CD90DD90ED9057
:10BBC000FC9020E030E0A901C701B6010E9456E6D2
:10BBD0008111EDC426962CAD3DAD4EAD5FAD2697DF
:10BBE000CA01B9010E94BBE66B017C01A30192016D
:10BBF000C301B2010E94BBE69B01AC01C701B601C3
:10BC00000E94A2EA6B017C01A5019401C501B40167
:10BC10000E94BBE69B01AC01C701B6010E94A2EAEB
:10BC20000E940DED28E60BA11CA1209FF001219F91
:10BC3000F00D1124E159FE4E658776878787908B3A
:10BC400088E60BA11CA1809FF001819FF00D1124BB
:10BC5000E159FE4E4584568467847088A3019201A1
:10BC600060E070E080E89FE30E947EEB64966CAF3A
:10BC70007DAF8EAF9FAF649729A539A94EA95AAD64
:10BC80000E94BBE64B015C018091B3099091B10920
:10BC9000891B8F7027968FAF2797A501940160E0CD
:10BCA00074E284E799E40E947EEB0E94D3EC6B017E
:10BCB0007C0127968FAD27978250863008F486C482
:10BCC000A5019401C301B2010E94BBE69B01AC0136
:10BCD0000E94BBE668966CAF7DAF8EAF9FAF689752
:10BCE00088E6ABA1BCA18A9F80018B9F100D112417
:10BCF00001591E4E68962CAD3DAD4EAD5FAD6897B7
:10BD0000D80111962D933D934D935C93149795967E
:10BD10002D913D914D915C9198972EAB3FAB48AFE3
:10BD200059AFCA01B9010E945AE66AAF7BAF8CAF26
:10BD30009DAF9B01AC01C501B4010E94BBE60E940E
:10BD400068EB0E94EBEBA8966CAF7DAF8EAF9FAF18
:10BD5000A897F801EE5AFF4F608371838283938323
:10BD60008E010F5E1F4F2A961FAF0EAF2A9700510C
:10BD7000110924961FAF0EAF249703EF16E0AC967F
:10BD80001FAF0EAFAC978E010F5D1F4F1AA309A313
:10BD900024960EAD1FAD2497AA961FAF0EAFAA979B
:10BDA000312C212C10E819A70FE309AB2A96AEAD70
:10BDB000BFAD2A972D913D914D915D912A96BFAFD0
:10BDC000AEAF2A97C501B4010E94BBE66B017C01AE
:10BDD000AA96EEADFFADAA9761937193819391936B
:10BDE000AA96FFAFEEAFAA9720E030E0A9010E942B
:10BDF000C8EC87FF04C0F7FAF094F7F8F094AC961B
:10BE0000AEADBFADAC974D905D906D907D90AC9612
:10BE1000BFAFAEAFAC97A7019601C301B2010E94BC
:10BE200056E687FD0DC409A11AA12A962EAD3FAD95
:10BE30002A970217130709F0B9CF20E030E040E855
:10BE40005FE3632D722D89A599A90E9456E687FFAD
:10BE500058C07E0131E1E30EF11C24960EAD1FADFA
:10BE60002497232D322D49A559A9D8016D917D9193
:10BE70008D919C910E94BBE6F8016193719381932F
:10BE800091938F01EE16FF0661F728E60BA11CA126
:10BE9000209FC001219F900D11249C0121593E4EED
:10BEA000790189010E5A1F4FA8966CAD7DAD8EADFC
:10BEB0009FADA8970E945AE6232D322D49A559A976
:10BEC0000E94BBE60E94EBEBD8016D937D938D93AE
:10BED0009C931397232D322D49A559A9632D722DBB
:10BEE00089A599A90E94BBE668962CAD3DAD4EADE3
:10BEF0005FAD68970E94BBE6F7016183728383831D
:10BF000094832AAD3BAD4CAD5DAD64966CAD7DAD1B
:10BF10008EAD9FAD64970E94BBE669A77AA78BA7F9
:10BF20009CA70DA11EA12FA138A5012B022B032B2D
:10BF300009F09EC388E62BA13CA1829F8001839FCC
:10BF4000100D112401591E4EF801818D928DA38D83
:10BF5000B48D892B8A2B8B2B09F08AC3858D968D06
:10BF6000A78DB0A1892B8A2B8B2B09F081C320913F
:10BF7000EF063091F0064091F1065091F20669A566
:10BF80007AA58BA59CA50E94BBE60E9468EB0E9447
:10BF9000EBEB2B013C01F801E95BFF4F108288E6D7
:10BFA0002BA13CA1829F8001839F100D1124015978
:10BFB0001E4EF801E25AFF4F408251826282738224
:10BFC000C301B2010E945AE629A53AA54BA55CA57A
:10BFD0000E947EEB6AAF7BAF8CAF9DAFD8015196CC
:10BFE0006D937D938D939C935497F801E95BFF4F7C
:10BFF0008081882381F17801B8E4EB0EF11C37963B
:10C000002091E3063091E4064091E5065091E60662
:10C0100060817181828193810E94BBE62AAD3BAD34
:10C020004CAD5DAD0E94BBE620919E1030919F10FB
:10C030004091A0105091A1100E94BBE69B01AC0161
:10C0400060E074E284EF99E40E947EEB0E94EBEBE7
:10C05000F7017183608388E60BA11CA1809FF0012A
:10C06000819FF00D1124E159FE4E218132814381DF
:10C0700054812C962CAF3DAF4EAF5FAF2C97CA01C9
:10C08000B9010E940DED362E272E8C0143ED56E0AE
:10C0900062965FAF4EAF62973E0151E1650E711C33
:10C0A00083ED96E09FAB8EAB24964EAC5FAC2497AD
:10C0B0003DA62DA209A719AB1AAAD201CD90DD90F9
:10C0C000ED90FD902D0120E030E0A901C701B601FF
:10C0D0000E94C8EC87FF04C0F7FAF094F7F8F094D8
:10C0E000EEA9FFA981909190A190B190FFABEEAB2A
:10C0F000A7019601C501B4010E9456E687FDD8C587
:10C1000064147504D1F627965FAD2797552309F47B
:10C1100048C6C090B509D090B609E090B709F09034
:10C12000B8092DEB37E346E855E3C701B6010E9495
:10C1300056E687FD36C6C701B6010E940DED6B01BC
:10C140007C019B01AC01632D722DC8010E9456E653
:10C1500087FD03C03C2C2D2C87019601A701632D80
:10C16000722DC8010E947EEB68966CAF7DAF8EAFDA
:10C170009FAF689789EB99E028969FAF8EAF28977D
:10C1800020E030E040E85FE32AAB3BAB4CAB5DAB7B
:10C190001EAA2896AEADBFAD28972D913D914D9129
:10C1A0005D912896BFAFAEAF289768966CAD7DAD18
:10C1B0008EAD9FAD68970E94BBE64B015C01249653
:10C1C000EEADFFAD2497C190D190E190F19024960F
:10C1D000FFAFEEAF2497FEA9FF2391F02AA93BA958
:10C1E0004CA95DA90E94BBE64B015C012AA93BA9B1
:10C1F0004CA95DA9C701B6010E94BBE66B017C0199
:10C20000A7019601C501B4010E94C8EC20E030E00E
:10C21000A90118160CF092C5C701B6010E94C8EC1E
:10C2200018160CF486C520E030E0A901C501B40160
:10C230000E9456E687FD7DC52601370177FA709486
:10C2400077F87094A3019201C501B4010E94C8EC73
:10C25000181614F4240135016296AEADBFAD629795
:10C26000CD90DD90ED90FD906296BFAFAEAF62973E
:10C27000A3019201C701B6010E9456E687FF15C0CF
:10C28000A3019201C701B6010E947EEB9B01AC01A4
:10C290006AA97BA98CA99DA90E94BBE66AAB7BAB6E
:10C2A0008CAB9DABBEA9BF5FBEABE9ECF9E02896B5
:10C2B0002EAD3FAD2897E217F30709F06ACF3EA9EC
:10C2C000332361F02AA93BA94CA95DA9632D722DE6
:10C2D000C8010E94BBE6362E272E8C0124EA30E7E7
:10C2E0004DE75FE3632D722DC8010E94BBE66B0131
:10C2F0007C01209111073091120740911307509152
:10C3000014070E9456E687FD42C58DA59DA1A9A5EB
:10C31000B9A98093110790931207A0931307B093C4
:10C32000140728E64BA15CA1249FC001259F900D16
:10C330001124DC01A159BE4E7D01232D322DA8010F
:10C34000632D722DC8010E94BBE6F70161877287D9
:10C35000838794876AAD7BAD8CAD9DAD90589B0172
:10C36000AC010E94A2EAD7011D962D913D914D91FD
:10C370005C9150970E94BBE69B01AC016BE077EDAE
:10C3800083E29BE30E94A1EA9B01AC018BE097ED65
:10C39000A3E2BBE3F70185839683A783B08710816F
:10C3A0002C966CAD7DAD8EAD9FAD2C970E9456E660
:10C3B00018160CF4FBC483E0182B88E62BA13CA1D3
:10C3C000829FF001839FF00D1124E159FE4E1083EE
:10C3D00080E1FE013196A9EBB9E001900D928A95BA
:10C3E000E1F72C968CAD9DADAEADBFAD2C97809393
:10C3F000B5099093B609A093B709B093B809E09630
:10C400000CAD1DAD2EAD3FADE0970093D909109353
:10C41000DA092093DB093093DC09E4962CAD3DADBD
:10C420004EAD5FADE4972093DD093093DE09409374
:10C43000DF095093E009E8968CAD9DADAEADBFAD80
:10C44000E8978093E1099093E209A093E309B09300
:10C45000E40960960CAD1DAD2EAD3FAD6097009325
:10C46000E5091093E6092093E7093093E8096C96F3
:10C470002CAD3DAD4EAD5FAD6C972093C9093093A7
:10C48000CA094093CB095093CC09A0968CAD9DADC1
:10C49000AEADBFADA0978093CD099093CE09A09388
:10C4A000CF09B093D009A4960CAD1DAD2EAD3FAD14
:10C4B000A4970093D1091093D2092093D309309304
:10C4C000D40922962CAD3DAD4EAD5FAD22972093A1
:10C4D000D5093093D6094093D7095093D809909144
:10C4E000B3098091B409981303C084E68093B0091E
:10C4F000E9968FADE9978F5F8F708093B309809134
:10C50000B3099091B20981508F70891351C4109171
:10C51000B4091BA30091B3090DA728E61BA10DA523
:10C520001013D1C4812C912CA12CB12C1DA219A6C1
:10C5300019AA1EAE212C312C00E010E02DA53BA144
:10C540002313CEC42114310409F07FC580916F00FC
:10C55000826080936F0081E0ECC680E0EAC6609064
:10C560000707709008070091090710910A07A7CAEA
:10C57000818D928DA38DB48D0697A105B10508F02C
:10C5800018CB858D968DA78DB0A10697A105B10515
:10C5900008F00FCB20E030E0A901C701B6010E94EE
:10C5A000C8EC87FF04C0F7FAF094F7F8F09488E637
:10C5B0000BA11CA1809FF001819FF00D1124E15976
:10C5C000FE4EC586D686E786F08A3ACB8091030771
:10C5D00090910407A0910507B0910607C816D906E7
:10C5E000EA06FB0608F06CCB8C199D09AE09BF0961
:10C5F000BC01CD01660F771F881F991F27964FAD8D
:10C600002797042F10E020E030E0A90198010E9454
:10C6100044EACA01B9010E945AE60E94D3EC6C0DAB
:10C620007D1D8E1D9F1D0E945AE69B01AC0160E09E
:10C6300074E284E799E40E947EEB4B015C0140CBFD
:10C64000A7019601C301B2010E947EEB7B018C0120
:10C650009B01AC01632D722D89A599A90E94C8EC9C
:10C6600018160CF0E0CB3E2C2F2C09A719ABDBCB16
:10C670000AA91BA92CA93DA9012B022B032B49F0C8
:10C680002091EB063091EC064091ED065091EE06BC
:10C6900008C02091E7063091E8064091E9065091E4
:10C6A000EA0669A57AA58BA59CA50E94BBE60E9417
:10C6B00068EB0E94EBEB2B013C012AA93BA94CA99A
:10C6C0005DA9232B242B252BC9F020E030E0A90104
:10C6D0006091E3067091E4068091E5069091E6068C
:10C6E0000E9456E6882351F081E00DA51EA52FA5D6
:10C6F00038A910161106120613060CF080E098E611
:10C700002BA13CA1929F8001939F100D11240159F0
:10C710001E4E180137E4230E311CD1018C9388235F
:10C7200009F4B3C02091C9093091CA094091CB09DD
:10C730005091CC096C966CAD7DAD8EAD9FAD6C9774
:10C740000E94A1EA6DA77EA78FA798AB2091CD0983
:10C750003091CE094091CF095091D009A0966CAD8F
:10C760007DAD8EAD9FADA0970E94A1EA4B015C010B
:10C770002091D1093091D2094091D3095091D40927
:10C78000A4966CAD7DAD8EAD9FADA4970E94A1EA3D
:10C790006B017C012DA53EA54FA558A9CA01B90181
:10C7A0000E94BBE66DA77EA78FA798ABA501940159
:10C7B000C501B4010E94BBE69B01AC016DA57EA53D
:10C7C0008FA598A90E94A2EA4B015C01A7019601DE
:10C7D000C701B6010E94BBE69B01AC01C501B401D3
:10C7E0000E94A2EA0E940DED6B017C012091D50907
:10C7F0003091D6094091D7095091D80922966CAD55
:10C800007DAD8EAD9FAD22970E94A1EAA701960152
:10C810000E947EEB6B017C01F801E25BFF4F6083BD
:10C8200071838283938320E030E040E450E40E94EF
:10C83000C8EC18161CF4F101108227C02091E30601
:10C840003091E4064091E5065091E606C701B60135
:10C850000E94BBE69B01AC016091DF067091E0068F
:10C860008091E1069091E2060E947EEB29A53AA50F
:10C870004BA55CA50E94BBE60E94EBEB6415750519
:10C880008605970510F42B013C0180913B11909196
:10C890003C11A0913D11B0913E110EA91FA928ADE8
:10C8A00039AD80179107A207B30708F4DFC02DA1A7
:10C8B0003EA14FA158A5232B242B252B41F160919C
:10C8C0003F11709140118091411190914211641576
:10C8D000750586059705D8F42EA93FA948AD59AD31
:10C8E0000E9435EA6B017C012DA13EA14FA158A504
:10C8F000C301B2010E9435EAC616D706E806F9065A
:10C9000030F4C701B6010E9444EA29013A0188E6E1
:10C910000BA11CA1809FF001819FF00D1124E15912
:10C92000FE4EC18CD28CE38CF48CC114D104E10492
:10C93000F10431F1609143117091441180914511DE
:10C94000909146116415750586059705C8F42EA9C2
:10C950003FA948AD59AD0E9435EA4B015C01A701E2
:10C960009601C301B2010E9435EA86169706A80611
:10C97000B90630F4C501B4010E9444EA29013A0124
:10C9800088E60BA11CA1809FF001819FF00D11246E
:10C99000E159FE4EC58CD68CE78CF0A0C114D104B1
:10C9A000E104F10431F160914711709148118091D7
:10C9B000491190914A116415750586059705C8F4CB
:10C9C0002EA93FA948AD59AD0E9435EA4B015C0143
:10C9D000A7019601C301B2010E9435EA86169706A7
:10C9E000A806B90630F4C501B4010E9444EA290141
:10C9F0003A0188E60BA11CA1809FF001819FF00DF8
:10CA00001124E159FE4EC1A0D2A0E3A0F4A0C114AC
:10CA1000D104E104F10409F4C2CA60914B11709190
:10CA20004C1180914D1190914E116415750586053C
:10CA3000970508F0B4CA2EA93FA948AD59AD0E9488
:10CA400035EA4B015C01A7019601C301B2010E94C6
:10CA500035EA86169706A806B90608F0A0CAC501E9
:10CA6000B4010E9444EA29013A0199CA2DA13EA1CC
:10CA70004FA158A5232B242B252BC9F160913F11E1
:10CA8000709140118091411190914211641575058A
:10CA90008605970560F50E945AE62AAD3BAD4CAD80
:10CAA0005DAD0E94BBE66B017C016DA17EA18FA1F3
:10CAB00098A50E945AE64B015C01C301B2010E9495
:10CAC0005AE6A50194010E94BBE69B01AC01C70197
:10CAD000B6010E9456E687FF0AC0A5019401C7016E
:10CAE000B6010E947EEB0E94EBEB2B013C0188E635
:10CAF0000BA11CA1809FF001819FF00D1124E15931
:10CB0000FE4E818C928CA38CB48C81149104A10470
:10CB1000B104B9F1609143117091441180914511B4
:10CB200090914611641575058605970550F50E948C
:10CB30005AE62AAD3BAD4CAD5DAD0E94BBE66B0144
:10CB40007C01C501B4010E945AE64B015C01C3019E
:10CB5000B2010E945AE6A50194010E94BBE69B0126
:10CB6000AC01C701B6010E9456E687FF0AC0A501C5
:10CB70009401C701B6010E947EEB0E94EBEB2B01F2
:10CB80003C0188E60BA11CA1809FF001819FF00D64
:10CB90001124E159FE4E858C968CA78CB0A081148F
:10CBA0009104A104B104B9F1609147117091481149
:10CBB0008091491190914A11641575058605970574
:10CBC00050F50E945AE62AAD3BAD4CAD5DAD0E94DA
:10CBD000BBE66B017C01C501B4010E945AE64B0122
:10CBE0005C01C301B2010E945AE6A50194010E94B2
:10CBF000BBE69B01AC01C701B6010E9456E687FF68
:10CC00000AC0A5019401C701B6010E947EEB0E94F3
:10CC1000EBEB2B013C0188E60BA11CA1809FF001EE
:10CC2000819FF00D1124E159FE4EC1A0D2A0E3A0D6
:10CC3000F4A0C114D104E104F10409F4B0C9609175
:10CC40004B1170914C1180914D1190914E116415C2
:10CC500075058605970508F0A2C90E945AE62AAD17
:10CC60003BAD4CAD5DAD0E94BBE64B015C01C70125
:10CC7000B6010E945AE66B017C01C301B2010E9419
:10CC80005AE6A70196010E94BBE69B01AC01C501D3
:10CC9000B4010E9456E687FF82C9A7019601C5012B
:10CCA000B4010E947EEB0E94EBEB2B013C0177C9A3
:10CCB000FAA9FF2331F1A5019401632D722DC8015A
:10CCC0000E94BBE64B015C012DA53DA149A559A9D8
:10CCD000C701B6010E94BBE69B01AC01C501B401CE
:10CCE0000E9456E687FF22C0A7019601C501B40144
:10CCF0000E947EEB6DA77DA389A799AB21E02AABAB
:10CD0000FFC9A7019601C501B4010E947EEB9B01FA
:10CD1000AC016DA57DA189A599A90E94BBE66DA76F
:10CD20007DA389A799AB31E03AABEAC941E04AABB0
:10CD3000E7C9A7019601C501B40113C0C701B60137
:10CD40000E9456E687FD09C020E030E0A901C50138
:10CD5000B4010E94C8EC18164CF4A5019401C70157
:10CD6000B6010E94A1EA2B013C0176CA24013501DB
:10CD700077FA709477F87094A3019201C701B60115
:10CD80000E9456E687FD68CA2601370165CA2DA5AF
:10CD90003DA149A559A9C701B6010E9456E687FFE2
:10CDA000B4CA3DA42DA009A519A9AFCA81E004CB3E
:10CDB000F090B3098FEF8F0D8F708BA3B090B209F5
:10CDC0008091B309B81609F454C0C12CD12C0BA121
:10CDD0000B1509F44EC0602E712C28E6269D8001AB
:10CDE000279D100D112401591E4ED8018C9183FDF1
:10CDF0002BC00EAF1AAB0115110541F11996BC916C
:10CE0000BDA7F801F285FDA3D8011B96BC91B9A777
:10CE1000F801F485F9ABD80115962D903D904D9011
:10CE20005C901897A20191016DA57DA189A59F2F06
:10CE30000E9456E6811186C1C114D10439F0F60171
:10CE4000808180FD7FC102C0CEAEDAAA8BA1815065
:10CE50008F708BA38091B2098B1103C0CEACDAA87E
:10CE6000B6CF0BA10B1529F081E08B0D8F70B82E7A
:10CE7000F1CF1091B2091BA3C12CD12C8091B30921
:10CE80000BA1801709F443CB802E912C28E6289D16
:10CE90008001299D100D112401591E4ED8018C913D
:10CEA00083FD0AC05801C114D10439F0C6010E94A3
:10CEB0003A7F811102C0C5C156018BA18F5F8F706F
:10CEC0008BA36501DBCF802F81508F70289FF001ED
:10CED0001124E159FE4E908193FF24CB8DA71ECBE8
:10CEE00048E6439FC0011124DC01A159BE4E1D013B
:10CEF0008C9183FD19C015966D917D918D919C91BA
:10CF000018970E940DEDF62EE72ED82EC92E01158A
:10CF1000110509F48CC0F801808180FD0AC0D1019F
:10CF20008C9180FD06C083C0FDA0E9A4D9A8CEAC39
:10CF300083C0F801808181608083C8010E943A7FAC
:10CF4000811171C0F80161817281838194810E9495
:10CF50000DED2B013C019B01AC0160E070E080E82D
:10CF60009FE30E947EEB4B015C019B01AC016F2DA6
:10CF70007E2D8D2D9C2D0E94BBE669837A838B8349
:10CF80009C832DA139A549A95EADC501B4010E94BC
:10CF9000BBE6698B7A8B8B8B9C8BAE014F5F5F4FAF
:10CFA000BE016F5E7F4FC8010E9469B8F801E95B5E
:10CFB000FF4F80818823B9F12091E3063091E40688
:10CFC0004091E5065091E606379660817181828135
:10CFD00093810E94BBE620919E1030919F1040915A
:10CFE000A0105091A1100E94BBE64B015C019B0177
:10CFF000AC01C301B2010E94BBE60E94EBEBF80159
:10D00000E65BFF4F71836083A50194016F2D7E2D38
:10D010008D2D9C2D0E94BBE60E94EBEBF801E45B9A
:10D02000FF4F71836083D8018C918E7F8C938F2CFE
:10D030009E2CAD2CBC2C81018BA18F5F8F708BA39C
:10D04000FDA2E9A6D9AACEAE79CAF101808181609C
:10D050008083C8010E943A7F81116FC0D10111966F
:10D060006D917D918D919C9114970E940DED6B01B6
:10D070007C019B01AC0160E070E080E89FE30E94CE
:10D080007EEB2B013C012DEC3CEC4CE45DE30E947B
:10D09000BBE669837A838B839C839401A501C301DA
:10D0A000B2010E94BBE6698B7A8B8B8B9C8BAE01A5
:10D0B0004F5F5F4FBE016F5E7F4FC1010E9469B835
:10D0C000F101E95BFF4F80818823B9F12091E306EC
:10D0D0003091E4064091E5065091E606379660816E
:10D0E0007181828193810E94BBE620919E103091D4
:10D0F0009F104091A0105091A1100E94BBE64B01DF
:10D100005C019B01AC01C701B6010E94BBE60E9415
:10D11000EBEBF101E65BFF4F718360832DEC3CECA0
:10D120004CE45DE3C501B4010E94BBE60E94EBEB59
:10D13000F101E45BFF4F71836083F10180818E7F99
:10D14000808304CA28E6269DF001279DF00D112456
:10D15000E159FE4E808181FD43C0C114D10441F0EC
:10D16000D6011596CD90DD90ED90FC90189708C0F3
:10D170008BE0C82E87EDD82E83E2E82E8BE3F82EC5
:10D18000B8E6B69DF001B79DF00D1124E159FE4EB1
:10D1900081899289A389B489BC01CD0190589B01F2
:10D1A000AC010E94A2EAF8012585368547855089A1
:10D1B0000E94BBE69B01AC01C701B6010E94A1EA37
:10D1C000E62E872E982EA92E262F372F482F592F3F
:10D1D0006DA57DA189A599A90E9456E687FF04C087
:10D1E000EDA48DA099A4A9A82E2D382D492D5A2D36
:10D1F000C201B1010E9456E6882309F427CEF8E661
:10D20000F69DC001F79D900D11249C0121593E4EC1
:10D210006901D9018C9181608C93C8010E943A7F89
:10D22000882329F0F60180818E7F80830FCE8E2D9A
:10D23000982DA92DBA2DF60185839683A783B087F3
:10D2400005CED6018C9181FD52C0D60115962D9147
:10D250003D914D915C9118972DA73EA74FA758ABD4
:10D260001501B5E02B0E311CF80145805680678012
:10D270007084A30192016DA57EA58FA598A90E9437
:10D2800056E687FF34C0F60181899289A389B48963
:10D29000BC01CD0190589B01AC010E94A2EAD601CD
:10D2A0001D962D913D914D915C9150970E94BBE64A
:10D2B0009B01AC016DA57EA58FA598A90E94A1EA4E
:10D2C0006B017C019B01AC01C301B2010E94C8EC5F
:10D2D00018166CF4D8018C9181608C93C5010E9462
:10D2E0003A7F8823E1F0F80180818E7F808318E601
:10D2F000189DF001199DF00D1124E159FE4E218574
:10D3000032854385548565817681878190850E9429
:10D3100056E68111D2CD0BA10093B209CECDD10139
:10D32000CD92DD92ED92FC9213970BA10093B2097E
:10D33000DECFC858DF4F0FB6F894DEBF0FBECDBFAB
:10D34000DF91CF911F910F91FF90EF90DF90CF90E1
:10D35000BF90AF909F908F907F906F905F904F9015
:10D360003F902F9008958091B3099091B409891B43
:10D370008F708F3019F40E941EA1F5CF8091B309F0
:10D380008F5F8F70E091B30998E69E9FF0011124A2
:10D39000E159FE4EDF011D929A95E9F798E09083DE
:10D3A0004091D9095091DA096091DB097091DC094B
:10D3B000458B568B678B708F4091DD095091DE094C
:10D3C0006091DF097091E009418F528F638F748FF4
:10D3D0004091E1095091E2096091E3097091E409FB
:10D3E000458F568F678F70A34091E5095091E609EC
:10D3F0006091E7097091E80941A352A363A374A364
:10D400002091B3099091B409291303C094E6909335
:10D41000B0098093B30980916F00826080936F00A0
:10D4200008959091B3098091B409981306C0809132
:10D430004A0790914B07892B19F00E941EA1F1CF4A
:10D440000895CF93DF938B3D9240B1F0EFECFDE177
:10D450008491EF012196882321F00E94E093FE0140
:10D46000F7CFE6EDF9E18491EF012196882331F0C1
:10D470000E94E093FE01F7CF80E001C081E0DF91E0
:10D48000CF9108952F923F924F925F926F927F9229
:10D490008F929F92AF92BF92CF92DF92EF92FF92C4
:10D4A0000F931F93CF93DF93CDB7DEB7C757D10943
:10D4B0000FB6F894DEBF0FBECDBF2DB63EB6A79611
:10D4C0001FAE1EAEA79784E690E0A9969FAF8EAFE1
:10D4D000A99701E09E012B593F4F44E050E0BE0167
:10D4E000655A7F4FCE0189599F4F0E9411D09E01EE
:10D4F0002B593F4F42E050E0BE0167597F4FCE01AC
:10D5000089599F4F0E9411D043E050E0BE01655AF7
:10D510007F4F8FED92E00E940DEE892B09F43FC002
:10D520006F968FAD6F97882339F08FE36C968FAF2E
:10D530006C976D961FAE6D97E4EEFDE184917F01CF
:10D540002FEFE21AF20A811103C0E9E9FAE104C0FF
:10D550000E94E093F701F2CF84917F013FEFE31A3D
:10D56000F30A882321F00E94E093F701F5CFBE0172
:10D57000655A7F4F80E99AE10E9486C5E2E8FAE1A8
:10D5800084917F019FEFE91AF90A882321F00E9414
:10D59000E093F701F5CF81E08093160754C5EDB70E
:10D5A000FEB7E696FFAFEEAFE6976B961CAE1DAEEC
:10D5B0001EAE1FAE6B97A7961FAE1EAEA79701E0DB
:10D5C0009E012B593F4F41E050E0BE0160597F4F13
:10D5D000CE0189599F4F0E9411D080E1EBE5F2E026
:10D5E000DE01919601900D928A95E1F780E1EBE6DC
:10D5F000F2E0DE01519601900D928A95E1F780E10B
:10D60000EBE7F2E0DE01119601900D928A95E1F7C9
:10D61000E1964FADE19750E04D5F5F4F440F551FCE
:10D62000440F551F2DB73EB7241B350B0FB6F8948A
:10D630003EBF0FBE2DBF8DB79EB701967C0100E0A7
:10D640009E012B593F4FBC01CE0189599F4F0E942B
:10D6500011D09E012B593F4F44E050E063E077E04A
:10D66000CE0189599F4F0E9411D0E1968FACE1976E
:10D67000912C93E0890E911C880C991C880C991CA4
:10D68000EDB7FEB7E819F9090FB6F894FEBF0FBE63
:10D69000EDBF2DB73EB72F5F3F4F69018DB79EB7E6
:10D6A000881999090FB6F8949EBF0FBE8DBFEDB7CC
:10D6B000FEB731965F019E012B593F4FA401B60181
:10D6C000CE0189599F4F0E9411D09E012B593F4F87
:10D6D000A401B501CE0189599F4F0E9411D010912C
:10D6E0001707112309F4A7C000E09E012B593F4FF3
:10D6F00044E050E06BEE76E0CE0189599F4F0E94E6
:10D7000011D09E012B593F4F44E050E06FEE76E080
:10D71000CE0189599F4F0E9411D09E012B593F4F36
:10D7200044E050E067EE76E0CE0189599F4F0E94B9
:10D7300011D09E012B593F4F44E050E06BE077E061
:10D74000CE0189599F4F0E9411D09E012B593F4F06
:10D7500044E050E067E077E0CE0189599F4F0E9496
:10D7600011D09E012B593F4F40E150E063ED76E030
:10D77000CE0189599F4F0E9411D09E012B593F4FD6
:10D7800044E050E0BE01695A7F4FCE0189599F4F56
:10D790000E9411D09E012B593F4F4CE050E068E3AE
:10D7A00075E0CE0189599F4F0E9411D09E012B59DF
:10D7B0003F4F44E050E063E371E1CE0189599F4F50
:10D7C0000E9411D09E012B593F4F44E050E0BE0112
:10D7D000695A7F4FCE0189599F4F0E9411D001E0B5
:10D7E0009E012B593F4F41E050E0BE0161597F4FF0
:10D7F000CE0189599F4F0E9411D09E012B593F4F56
:10D8000041E050E0BE0162597F4FCE0189599F4FE0
:10D810000E9411D011118AC06B968CAD9DADAEAD3A
:10D82000BFAD6B978093C2109093C310A093C410A8
:10D83000B093C5107BC0E1968FADE19790E0029662
:10D8400023EF36E0E4963FAF2EAFE497B501DE015B
:10D850001196E2E98E2EE0E19E2EAE014F5E5F4F03
:10D86000FFE4AF2EF1E1BF2EE896FFAEEEAEE897F3
:10D870007E0131E2E30EF11C20E030E082179307D5
:10D880002CF0E896EEADFFADE89701C0F7014080BF
:10D89000518062807380F501419251926192719240
:10D8A0005F018217930714F0F60101C0FA0140806E
:10D8B000518062807380F401419251926192719221
:10D8C0004F018217930734F0FB0140805180628042
:10D8D000738005C04D905D906D907C901397E49699
:10D8E000EEADFFADE4974192519261927192E49650
:10D8F000FFAFEEAFE4972F5F3F4F6C5F7F4F149603
:10D90000F4E0CF0ED11C4C5F5F4FE896EEADFFAD5B
:10D91000E8973496E896FFAFEEAFE897F4E0EF0EA5
:10D92000F11C2430310509F0A9CFDECEE0968FAD91
:10D93000E097853099F4AF968FADAF97853071F44D
:10D9400000E09E012B593F4F44E650E066EC70E149
:10D95000CE0189599F4F0E9411D024C0111102C0DD
:10D960000E94D1BDE0968FADE097AF96CFACAF9758
:10D970008C9D60011124E12CF12CEC14FD0491F03C
:10D9800000E09E012B593F4F44E050E0BE01695A30
:10D990007F4FCE0189599F4F0E9411D02FEFE21A7D
:10D9A000F20AEBCF00E09E012B593F4F44E050E0DC
:10D9B000BE016D5A7F4FCE0189599F4F0E9411D0F1
:10D9C0001AE0115079F000E09E012B593F4F44E0DE
:10D9D00050E0BE01695A7F4FCE0189599F4F0E9486
:10D9E00011D0EFCF01E09E012B593F4F41E050E0B5
:10D9F000BE0163597F4FCE0189599F4F0E9411D0BC
:10DA00009E012B593F4F41E050E0BE0164597F4FCA
:10DA1000CE0189599F4F0E9411D000E09E012B59E1
:10DA20003F4F44E050E0BE01635C7F4FCE01895917
:10DA30009F4F0E9411D09E012B593F4F44E050E070
:10DA4000BE016F5C7F4FCE0189599F4F0E9411D05C
:10DA5000AE968FADAE97AD96CFACAD978C9D600175
:10DA60001124E12CF12C00E09E012B593F4FCE14E4
:10DA7000DF0471F044E050E0BE01695A7F4FCE01EF
:10DA800089599F4F0E9411D03FEFE31AF30AEBCF61
:10DA900041E050E0BE016F587F4FCE0189599F4F42
:10DAA0000E9411D09E012B593F4F41E050E0BE0132
:10DAB00065597F4FCE0189599F4F0E9411D09E0119
:10DAC0002B593F4F44E050E0BE01695A7F4FCE01D1
:10DAD00089599F4F0E9411D09E012B593F4F44E01E
:10DAE00050E0BE01695A7F4FCE0189599F4F0E9475
:10DAF00011D09E012B593F4F44E050E067E371E1A4
:10DB0000CE0189599F4F0E9411D09E012B593F4F42
:10DB100044E050E0BE01615B7F4FCE0189599F4FC9
:10DB20000E9411D09E012B593F4F44E050E0BE01AE
:10DB3000655B7F4FCE0189599F4F0E9411D09E0196
:10DB40002B593F4F44E050E0BE01695B7F4FCE014F
:10DB500089599F4F0E9411D010E000E09E012B597F
:10DB60003F4F44E050E0BE01695A7F4FCE018959D2
:10DB70009F4F0E9411D0111110C06B96CCACDDAC40
:10DB8000EEACFFAC6B9720E030E84BE355E4C70107
:10DB9000B6010E9456E6811103C054E0F52E33C051
:10DBA00080911707811108C0C0923C07D0923D07B1
:10DBB000E0923E07F0923F0700E09E012B593F4F55
:10DBC00044E050E068E377E0CE0189599F4F0E941E
:10DBD00011D09E012B593F4F44E050E060E477E0C4
:10DBE000CE0189599F4F0E9411D09E012B593F4F62
:10DBF00044E050E0BE01695A7F4FCE0189599F4FE2
:10DC00000E9411D012C0FA94FF2079F000E09E012A
:10DC10002B593F4F44E050E0BE01695A7F4FCE017F
:10DC200089599F4F0E9411D0EECF1F5F153009F028
:10DC300094CF00E09E012B593F4F42E050E0BE01DF
:10DC40006D597F4FCE0189599F4F0E9411D09E017F
:10DC50002B593F4F44E050E0BE01695A7F4FCE013F
:10DC600089599F4F0E9411D06B96CCACDDACEEACC5
:10DC7000FFAC6B9720E030E84BE355E4C701B601F9
:10DC80000E9456E6882329F180911707811108C068
:10DC9000C0923407D0923507E0923607F0923707EA
:10DCA00000E09E012B593F4F44E050E060E377E0F5
:10DCB000CE0189599F4F0E9411D09E012B593F4F91
:10DCC00044E050E06CE277E0CE0189599F4F0E941A
:10DCD00011D000E09E012B593F4F42E050E0BE01C1
:10DCE0006F597F4FCE0189599F4F0E9411D09E01DD
:10DCF0002B593F4F41E050E0BE016F587F4FCE019E
:10DD000089599F4F0E9411D019E0115000E09E01E7
:10DD10002B593F4F112359F044E050E0BE01695A9E
:10DD20007F4FCE0189599F4F0E9411D0EECF41E025
:10DD300050E06AE271E1CE0189599F4F0E9411D0F3
:10DD4000F12C00E09E012B593F4F44E050E0BE0112
:10DD5000695A7F4FCE0189599F4F0E9411D010916F
:10DD60001707111110C0F1100EC06B968CAD9DAD50
:10DD7000AEADBFAD6B9780932F1190933011A093F0
:10DD80003111B0933211F39485E0F812DACF11110A
:10DD900002C00E94D1C44CE0F42EFA94F11003C0EA
:10DDA0003CE0F32E0FC000E09E012B593F4F42E0B4
:10DDB00050E0BE01615A7F4FCE0189599F4F0E94AA
:10DDC00011D0EBCFFA9400E09E012B593F4FFF207A
:10DDD00059F044E050E0BE016D5B7F4FCE018959A0
:10DDE0009F4F0E9411D0EECF46E050E0BE01635C31
:10DDF0007F4FCE0189599F4F0E9411D09E012B5910
:10DE00003F4F44E050E063EE76E0CE0189599F4FEA
:10DE10000E9411D09E012B593F4F4CE050E0BE01B3
:10DE20006F5C7F4FCE0189599F4F0E9411D02CE12A
:10DE3000F22EFA94F11003C094E0F92E1DC000E018
:10DE40009E012B593F4F44E050E0BE01695A7F4F7D
:10DE5000CE0189599F4F0E9411D0EBCF00E09E0167
:10DE60002B593F4F44E050E0BE01695A7F4FCE012D
:10DE700089599F4F0E9411D0FA94F110EFCF8BE097
:10DE8000F82EFA94FF2079F000E09E012B593F4FC5
:10DE900044E050E0BE01695A7F4FCE0189599F4F3F
:10DEA0000E9411D0EECFA9968EAD9FADA997845652
:10DEB0009109C7DA80931607882309F1E4EEFDE1A2
:10DEC00084917F019FEFE91AF90A882321F00E94CB
:10DED000E093F701F5CFA9966EAD7FADA997645693
:10DEE00071098AE79AE10E946DC56BED72E082E7E5
:10DEF0009AE10E946DC58AE00E94E09399C0A796BE
:10DF00002EAD3FADA797AB968EAD9FADAB972817C3
:10DF1000390709F44BC081E080931607EFECFDE16F
:10DF200084917F012FEFE21AF20A811103C0E2E52A
:10DF3000FAE104C00E94E093F701F2CF84917F01DF
:10DF40003FEFE31AF30A882321F00E94E093F701E0
:10DF5000F5CFAB966EAD7FADAB9780E090E04AE039
:10DF60000E940197EDE4FAE184917F019FEFE91AA5
:10DF7000F90A882321F00E94E093F701F5CFA796D4
:10DF80006EAD7FADA79780E090E04AE00E940197D8
:10DF9000EDE3FAE184917F012FEFE21AF20A882380
:10DFA00009F446C00E94E093F701F4CF111142C07A
:10DFB000E4EEFDE184917F013FEFE31AF30A811162
:10DFC00003C00FED12E004C00E94E093F701F2CF0E
:10DFD000F80181918F01882319F00E94E093F8CF16
:10DFE000A9966EAD7FADA9976456710980E29AE15A
:10DFF0000E946DC5A7964EAD5FADA79760E070E03B
:10E0000083E19AE10E9433C5E0E1FAE184917F0166
:10E010002FEFE21AF20A811107C0809116078111D1
:10E0200009C00E94D2D006C00E94E093F701EECF53
:10E03000112399F3E6968EAD9FADE6970FB6F8944F
:10E040009EBF0FBE8DBF80911707811102C00E9435
:10E050009EBE9091160781E089270FB6F8943EBEC8
:10E060000FBE2DBEC958DF4F0FB6F894DEBF0FBEEE
:10E07000CDBFDF91CF911F910F91FF90EF90DF9077
:10E08000CF90BF90AF909F908F907F906F905F9058
:10E090004F903F902F90089581E080931707F2D919
:10E0A000109217078111EEC90E940DC381E00895F7
:10E0B0008F929F92AF92BF92CF92DF92EF92FF9298
:10E0C0000F931F93CF93DF93CDB7DEB7CA5AD10911
:10E0D0000FB6F894DEBF0FBECDBFE9961CAE1DAEE5
:10E0E0001EAE1FAEE9978091EC039091ED03A091D5
:10E0F000EE03B091EF03ED968CAF9DAFAEAFBFAF27
:10E10000ED97C556DF4F19821882CB59D04084E66F
:10E1100090E0C356DF4F99838883CD59D040109249
:10E1200016079E0125563F4F44E050E0BE01675858
:10E130007F4FCE0183569F4F0E945ED0C356DF4F64
:10E1400088819981CD59D0400296C356DF4F99837B
:10E150008883CD59D040C556DF4F19821882CB59DC
:10E16000D04081E0CD55DF4F8883C35AD0409E0117
:10E1700025563F4F41E050E0BE016D557F4FCE0127
:10E1800083569F4F0E945ED09E0125563F4F40E12F
:10E1900050E06FE471E1CE0183569F4F0E945ED044
:10E1A0009E0125563F4F44E050E063E077E0CE010A
:10E1B00083569F4F0E945ED09E0125563F4F40E1FF
:10E1C00050E062E970E1CE0183569F4F0E945ED01D
:10E1D0009E0125563F4F40E150E063EF76E0CE01CF
:10E1E00083569F4F0E945ED09E0125563F4F44E0CC
:10E1F00050E06BEE76E0CE0183569F4F0E945ED0DA
:10E200009E0125563F4F44E050E06FEE76E0CE0190
:10E2100083569F4F0E945ED09E0125563F4F44E09B
:10E2200050E067EE76E0CE0183569F4F0E945ED0AD
:10E230009E0125563F4F44E050E06BE077E0CE0171
:10E2400083569F4F0E945ED09E0125563F4F44E06B
:10E2500050E067E077E0CE0183569F4F0E945ED08A
:10E260009E0125563F4F40E150E063ED76E0CE0140
:10E2700083569F4F0E945ED08AE097EDA3EABCE3ED
:10E28000E9968CAF9DAFAEAFBFAFE9979E01255623
:10E290003F4F44E050E0BE016B587F4FCE018356A4
:10E2A0009F4F0E945ED09E0125563F4F4CE050E0AC
:10E2B00068E375E0CE0183569F4F0E945ED0809147
:10E2C0007D1090917E10A0917F10B0918010C35866
:10E2D000DF4F88839983AA83BB83CD57D0409E01AB
:10E2E00025563F4F44E050E0BE0163587F4FCE01BA
:10E2F00083569F4F0E945ED085E0CC55DF4F8883C8
:10E30000C45AD040CB55DF4F8883C55AD0409E01B8
:10E3100025563F4F44E050E062EC70E1CE01835659
:10E320009F4F0E945ED09E0125563F4F41E050E036
:10E33000BE016C557F4FCE0183569F4F0E945ED029
:10E340009E0125563F4F41E050E0BE016B557F4F87
:10E35000CE0183569F4F0E945ED09E0125563F4FAF
:10E3600044E650E066EC70E1CE0183569F4F0E9478
:10E370005ED0CF57DF4F188219821A821B82C15894
:10E38000D0409E0125563F4F44E050E0BE016F57FC
:10E390007F4FCE0183569F4F0E945ED0E9961CAE00
:10E3A0001DAE1EAE1FAEE9971AE0115071F09E012E
:10E3B00025563F4F44E050E0BE016B587F4FCE01E1
:10E3C00083569F4F0E945ED0F0CF83E0CA55DF4F47
:10E3D0008883C65AD040C955DF4F8883C75AD0407A
:10E3E000CB57DF4F188219821A821B82C558D04042
:10E3F000C757DF4F188219821A821B82C958D04032
:10E40000E9961CAE1DAE1EAE1FAEE9979E012556C5
:10E410003F4F41E050E0BE016A557F4FCE01835629
:10E420009F4F0E945ED09E0125563F4F41E050E035
:10E43000BE0169557F4FCE0183569F4F0E945ED02B
:10E440009E0125563F4F44E050E0BE0167577F4F85
:10E45000CE0183569F4F0E945ED09E0125563F4FAE
:10E4600044E050E0BE016B577F4FCE0183569F4F73
:10E470000E945ED00AE010E00150110971F09E0187
:10E4800025563F4F44E050E0BE016B587F4FCE0110
:10E4900083569F4F0E945ED0EFCFC855DF4F188242
:10E4A000C85AD0408FEFC755DF4F8883C95AD04034
:10E4B0009E0125563F4F41E050E0BE0168557F4F19
:10E4C000CE0183569F4F0E945ED09E0125563F4F3E
:10E4D00041E050E0BE0167557F4FCE0183569F4F0C
:10E4E0000E945ED0E9961CAE1DAE1EAE1FAEE9972F
:10E4F0009E0125563F4F44E050E0BE016B587F4FD0
:10E50000CE0183569F4F0E945ED09E0125563F4FFD
:10E5100044E050E0BE016B587F4FCE0183569F4FC1
:10E520000E945ED09E0125563F4F44E050E067E3D5
:10E5300071E1CE0183569F4F0E945ED080918B0285
:10E5400090918C02A0918D02B0918E02C357DF4F43
:10E5500088839983AA83BB83CD58D04080918F0252
:10E5600090919002A0919102B0919202CF56DF4F0C
:10E5700088839983AA83BB83C159D040CB56DF4F90
:10E5800019821882C559D040C956DF4F19821882A6
:10E59000C759D0409E0125563F4F44E050E0BE0190
:10E5A00063577F4FCE0183569F4F0E945ED09E01DE
:10E5B00025563F4F44E050E0BE016F567F4FCE01DD
:10E5C00083569F4F0E945ED09E0125563F4F44E0E8
:10E5D00050E0BE016B567F4FCE0183569F4F0E9485
:10E5E0005ED010E0C12C80E8D82E8BE3E82E85E4C5
:10E5F000F82E812C912C90E8A92E9FE3B92E1111B1
:10E6000038C09E0125563F4F44E050E06CE377E070
:10E61000CE0183569F4F0E945ED09E0125563F4FEC
:10E6200044E050E068E377E0CE0183569F4F0E94BC
:10E630005ED09E0125563F4F44E050E060E477E015
:10E64000CE0183569F4F0E945ED0E9968CAE9DAE60
:10E65000AEAEBFAEE9979E0125563F4F44E050E075
:10E66000BE016B587F4FCE0183569F4F0E945ED0F4
:10E670002AC0E996CCAEDDAEEEAEFFAEE9979E01C4
:10E6800025563F4F44E050E0BE016B587F4FCE010E
:10E6900083569F4F0E945ED0E9961CAE1DAE1EAE03
:10E6A0001FAEE99704E0015071F09E0125563F4FDF
:10E6B00044E050E0BE016B587F4FCE0183569F4F20
:10E6C0000E945ED0F0CF1F5F153009F098CF84E133
:10E6D00090E0C156DF4F99838883CF59D0409E0187
:10E6E00025563F4F42E050E0BE0161567F4FCE01BC
:10E6F00083569F4F0E945ED09E0125563F4F44E0B7
:10E7000050E064E377E0CE0183569F4F0E945ED0D5
:10E710009E0125563F4F44E050E060E377E0CE0194
:10E7200083569F4F0E945ED09E0125563F4F44E086
:10E7300050E06CE277E0CE0183569F4F0E945ED09E
:10E7400080E290E0CF55DF4F99838883C15AD04053
:10E750009E0125563F4F42E050E0BE016F557F4F6E
:10E76000CE0183569F4F0E945ED0C655DF4F188260
:10E77000CA5AD04080E2E3E9F2E0DE019D960190C2
:10E780000D928A95E1F79E0125563F4F41E050E0FA
:10E79000BE0166557F4FCE0183569F4F0E945ED0CB
:10E7A0009E0125563F4F40E250E0BE01635D7F4F22
:10E7B000CE0183569F4F0E945ED09E0125563F4F4B
:10E7C00041E050E06AE271E1CE0183569F4F0E9422
:10E7D0005ED010E011110EC080912F119091301178
:10E7E000A0913111B0913211E9968CAF9DAFAEAFCF
:10E7F000BFAFE9979E0125563F4F44E050E0BE0170
:10E800006B587F4FCE0183569F4F0E945ED01F5F93
:10E81000153001F7BE01635B7F4F86E1FB0111926A
:10E820008A95E9F79E0125563F4F46E150E0CE011B
:10E8300083569F4F0E945ED08CE2E3EBF2E0DE0154
:10E84000119601900D928A95E1F79E0125563F4F52
:10E850004CE250E0BE016F5F7F4FCE0183569F4F69
:10E860000E945ED0BE0161597F4F86E0FB0111928C
:10E870008A95E9F79E0125563F4F46E050E0CE01CC
:10E8800083569F4F0E945ED09E0125563F4F44E025
:10E8900050E063EE76E0CE0183569F4F0E945ED03B
:10E8A000BE016D597F4F8CE0FB0111928A95E9F70B
:10E8B0009E0125563F4F4CE050E0CE0183569F4FBE
:10E8C0000E945ED0E9961CAE1DAE1EAE1FAEE9974B
:10E8D0001CE1115071F09E0125563F4F44E050E07D
:10E8E000BE016B587F4FCE0183569F4F0E945ED072
:10E8F000F0CFE9961CAE1DAE1EAE1FAEE99714E038
:10E90000115071F09E0125563F4F44E050E0BE018A
:10E910006B587F4FCE0183569F4F0E945ED0F0CF41
:10E92000E9961CAE1DAE1EAE1FAEE9971BE011505E
:10E9300071F09E0125563F4F44E050E0BE016B58F8
:10E940007F4FCE0183569F4F0E945ED0F0CF8091C3
:10E950001607811167C0C356DF4FE880F980CD5993
:10E96000D040F4E6EF1AF108C556DF4F888199814F
:10E97000CB59D040C756DF4F99838883C959D040BF
:10E9800084E690E0C356DF4F99838883CD59D04009
:10E990009E0125563F4F44E050E06FED72E0CE01FE
:10E9A00083569F4F0E945ED09E0125563F4F42E006
:10E9B00050E0BE0167567F4FCE0183569F4F0E94A5
:10E9C0005ED0E4EEFDE184918F010F5F1F4F88233D
:10E9D00021F00E94E093F801F6CFB7018EEF99E1A4
:10E9E0000E946DC5C756DF4F48815981C959D04033
:10E9F00060E070E081EF99E10E9433C5EEEEF9E14D
:10EA000084918F010F5F1F4F882321F00E94E093B4
:10EA1000F801F6CFC7010E94216A90911607892B51
:10EA2000809316079091160781E08927C655DF4F1E
:10EA30000FB6F894DEBF0FBECDBFDF91CF911F910F
:10EA40000F91FF90EF90DF90CF90BF90AF909F908D
:10EA50008F900895FF920F931F93CF93DF938C01B4
:10EA6000EB01F42E80E20E94E0938FEFF81611F094
:10EA700084E501C082E40E94E0938AE30E94E0936F
:10EA8000F801608171818281938142E00E948697C2
:10EA9000488159816A817B818DE49DE10E9450C546
:10EAA00062E070E080E090E0DF91CF911F910F91E4
:10EAB000FF900C942CB78F929F92AF92BF92CF92FF
:10EAC000DF92EF92FF920F931F93CF93DF93F0E2C9
:10EAD000FF2EE12CAE2DB0E0BD016F0D711D7595BF
:10EAE00067956E1511F0F6120BC0E0E3FBE165913E
:10EAF0007491072E000C880B990B0E945CE662C093
:10EB00009B0121503109220F331F220F331FF901BE
:10EB1000EE54F54E05911491AB01440F551F440F6F
:10EB2000551FFA01EE54F54EC591D4918017910707
:10EB300014F4F62ED1CFC817D90714F4E62ECACF95
:10EB4000F901EC54F54EE590F490FA01EC54F54ED1
:10EB5000C590D490BC01601B710B072E000C880B74
:10EB6000990B0E945CE64B015C01B6016E197F09AE
:10EB7000072E000C880B990B0E945CE69B01AC01F0
:10EB8000C501B4010E94BBE64B015C01C01BD10B67
:10EB9000BE01DD0F880B990B0E945CE69B01AC0166
:10EBA000C501B4010E947EEB4B015C01B701FF0C73
:10EBB000880B990B0E945CE69B01AC01C501B40176
:10EBC0000E94A2EADF91CF911F910F91FF90EF90E9
:10EBD000DF90CF90BF90AF909F908F9008950F934C
:10EBE0001F93CF93DF93CDB7DEB728970FB6F89476
:10EBF000DEBF0FBECDBF60914A0470914B04072E5B
:10EC0000000C880B990B0E945CE66D837E838F83DA
:10EC1000988780914C0490914D04A0914E04B0913E
:10EC20004F0489839A83AB83BC834DEFBE016B5F36
:10EC30007F4FCE0101960EDF609144047091450430
:10EC4000072E000C880B990B0E945CE66D837E8377
:10EC50008F8398878091460490914704A09148043F
:10EC6000B091490489839A83AB83BC834FEFBE0183
:10EC70006B5F7F4FCE010196EDDEE5E5FDE184910E
:10EC80008F010F5F1F4F882321F00E94E093F8014E
:10EC9000F6CFE0914E07F0E0E45BF84F608170E062
:10ECA00080E090E00E946C97E0E5FDE184918F01A7
:10ECB0000F5F1F4F882321F00E94E093F801F6CFE9
:10ECC00060914D0770E080E090E00E946C9728967C
:10ECD0000FB6F894DEBF0FBECDBFDF91CF911F916D
:10ECE0000F9108950F930FB70F9300916E000B7F54
:10ECF00000936E0078940F930BB70F930CB70F929D
:10ED00001F922F933F934F935F936F937F938F93B4
:10ED10009F93AF93BF93EF93FF931124EFD2FF9193
:10ED2000EF91BF91AF919F918F917F916F915F9183
:10ED30004F913F912F911F900F900CBF0F910BBFE0
:10ED40000F910460F89400936E000F910FBF0F9124
:10ED50001895CF92DF92EF92FF92C0904604D09028
:10ED60004704E0904804F090490460914404709195
:10ED7000450466507109072E000C880B990B0E9400
:10ED80005CE69B01AC01C701B6010E9456E687FF15
:10ED90001FC020E030E040E050E4C701B6010E940F
:10EDA000A2EA0E94EBEB70938607609385070E94AE
:10EDB000F158DC01CB01805A9541AF4FBF4F809392
:10EDC000810790938207A0938307B093840708C0BC
:10EDD0001092810710928207109283071092840785
:10EDE000FF90EF90DF90CF900895CF92DF92EF9257
:10EDF000FF92C0904C04D0904D04E0904E04F090EF
:10EE00004F0460914A0470914B0469507109072EB8
:10EE1000000C880B990B0E945CE69B01AC01C701BA
:10EE2000B6010E9456E687FF1FC020E030E040EAAE
:10EE300050E4C701B6010E94A2EA0E94EBEB709376
:10EE4000800760937F070E94F158DC01CB01885452
:10EE50009747AF4FBF4F80937B0790937C07A0935A
:10EE60007D07B0937E0708C010927B0710927C0745
:10EE700010927D0710927E07FF90EF90DF90CF9069
:10EE800008958F929F92AF92BF92CF92DF92EF92AE
:10EE9000FF920F931F93CF93DF93F0E4FF2EE12CAB
:10EEA000AE2DB0E0BD016F0D711D759567956E15A6
:10EEB00011F0F6120BC0E2EAFCE165917491072EA5
:10EEC000000C880B990B0E945CE662C09B012150EC
:10EED0003109220F331F220F331FF901EC55F44E75
:10EEE00005911491AB01440F551F440F551FFA01B2
:10EEF000EC55F44EC591D4918017910714F4F62E79
:10EF0000D1CFC817D90714F4E62ECACFF901EA55B4
:10EF1000F44EE590F490FA01EA55F44EC590D49081
:10EF2000BC01601B710B072E000C880B990B0E9413
:10EF30005CE64B015C01B6016E197F09072E000CDF
:10EF4000880B990B0E945CE69B01AC01C501B401E2
:10EF50000E94BBE64B015C01C01BD10BBE01DD0F63
:10EF6000880B990B0E945CE69B01AC01C501B401C2
:10EF70000E947EEB4B015C01B701FF0C880B990BE3
:10EF80000E945CE69B01AC01C501B4010E94A2EAAB
:10EF9000DF91CF911F910F91FF90EF90DF90CF9075
:10EFA000BF90AF909F908F90089560E080919107FF
:10EFB0009091920780DD60934C0470934D04809390
:10EFC0004E0490934F0480918F079091900759DFE2
:10EFD00060934604709347048093480490934904D7
:10EFE000A8951092490708957F928F929F92AF92B1
:10EFF000BF92CF92DF92EF92FF920F931F93CF9326
:10F00000DF9320E030E048E452E460914C047091DA
:10F010004D0480914E0490914F040E94C8EC181644
:10F020004CF4E8E3FBE1E491C1E001C0CC0FEA95C8
:10F03000EAF701C0C0E082E3E82E8BE1F82E08E396
:10F040001BE196E0A92E912CD0E0CC24C394D12CC6
:10F05000F7017490F801849077FC23C0892D90E02B
:10F06000082C02C0959587950A94E2F780FD19C097
:10F07000BE01082C02C0759567950A94E2F761708D
:10F08000B62EB1946B2D872D0E94FBB56B2D70E0D1
:10F09000872D0E9465B6C60101C0880F8A94EAF7E1
:10F0A000982AAA94FFEFEF1AFF0A0F5F1F4FA110D3
:10F0B000CFCFDF91CF911F910F91FF90EF90DF9015
:10F0C000CF90BF90AF909F908F907F9008950F93B7
:10F0D0001F9380912B07813019F40E94F15808C0CA
:10F0E00060912707709128078091290790912A073E
:10F0F00000915307109154072091550730915607FE
:10F10000601B710B820B930B28EE33E040E050E064
:10F110000E9444EA80914F0790915007A0915107B7
:10F12000B0915207BC01CD01620F731F841F951F60
:10F130001F910F91089510922B0710925307109270
:10F1400054071092550710925607109227071092F5
:10F1500028071092290710922A0710924F07109241
:10F1600050071092510710925207089580912B0773
:10F170008130E1F0823051F4AADF60934F07709341
:10F180005007809351079093520701C0D4DF81E06C
:10F1900080932B070E94F158609353077093540794
:10F1A000809355079093560781E0089580E0089575
:10F1B00080912B07813079F482E080932B070E94A5
:10F1C000F15860932707709328078093290790933D
:10F1D0002A0781E0089580E0089580912B078150EF
:10F1E000823010F080E0089510922B070E94F158B1
:10F1F00060932707709328078093290790932A0725
:10F2000081E008951092480780E090E00E94E6595E
:10F2100010924504109244049CDDDFDF80E090E012
:10F220000E94E65910924C072C98109245041092B7
:10F23000440410924D078091020180728093000176
:10F240000895DF92EF92FF920F931F93CF93DF9376
:10F25000F82ED62EE72E8A0180912702882309F402
:10F2600039C0EFECFDE18491EF012196882321F074
:10F270000E94E093FE01F7CFED2DFE2D8491EF016A
:10F280002196882321F00E94E093FE01F7CFE3E46A
:10F29000FBE18491EF012196882321F00E94E09305
:10F2A000FE01F7CFF7FC0BC06F2DFF0C770B880B1F
:10F2B000990B0E946C978AE00E94E0930BC0EEE3EA
:10F2C000FBE18491EF012196882321F00E94E093D5
:10F2D000FE01F7CF80915707811108C010922702D5
:10F2E00081E080935707C8010E94D7A0DF91CF919A
:10F2F0001F910F91FF90EF90DF9084CFEF92FF92DC
:10F300000F931F93CF93DF9380912A028F37A0F042
:10F310008F5790914C079093A207992311F02C9A44
:10F3200001C02C9820914D072093A10790910201D4
:10F33000222369F090950BC09091A207891708F0DD
:10F340002C989091A107891728F090910201907252
:10F35000909300018F5F80932A029091A00781E033
:10F3600089278093A0078091290285301CF4C1E091
:10F37000C80F01C0C0E0823009F4B4C054F488233F
:10F3800001F1813009F0E3C088E080937B0085E4DF
:10F39000C0C0843009F4C5C00CF4B7C0853009F092
:10F3A000D6C090919F07911102C080939F078091D2
:10F3B0009F07815080939F07882309F4C8C0C5E048
:10F3C000C6C0809128028F5F80311CF48093280290
:10F3D000BEC01092280280914907811113C080910C
:10F3E000950790919607909392078093910780914B
:10F3F0009307909194079093900780938F0781E0F3
:10F40000809349078AE0E5E9F7E0DF011D928A95DC
:10F41000E9F71092940710929307009191071091C9
:10F42000920711950195110980914A0490914B041E
:10F43000D1E0181619062CF080914C07811101C0FB
:10F44000D0E0809132059091330591958195910995
:10F450008017910734F44BED5CE16CEF7CE180E0C8
:10F46000F0DE80911C0290911D0291958195910989
:10F470000817190744F4DD2331F04EE05DE16FE237
:10F480007DE180E0DEDE809144049091450411E04E
:10F49000181619062CF080914D07811101C010E05B
:10F4A000E0908F07F09090078091300590913105A2
:10F4B0008E159F0534F04BEE5CE16CEF7CE18FEF35
:10F4C000C0DE80911A0290911B02E816F9060CF436
:10F4D0003EC01123E1F14EE15DE16FE27DE18FEF8E
:10F4E000B0DE35C080917A0086FD2EC08091780014
:10F4F000909179002091950730919607820F931F84
:10F50000909396078093950722C088E080937B00B4
:10F5100086E480937C0080917A00806480937A00F6
:10F5200016C080917A0086FD11C08091780090917C
:10F5300079002091930730919407820F931F909345
:10F5400094078093930703C0C2E001C0C4E0C09356
:10F5500029028091370581110E94E1BD80914A07FF
:10F5600090914B070097A9F0019790934B078093D8
:10F570004A07892B71F481E49DE19093A40780935D
:10F58000A307DF91CF911F910F91FF90EF900C9403
:10F590000C94DF91CF911F910F91FF90EF90089500
:10F5A0002F923F924F925F926F927F928F929F9293
:10F5B000AF92BF92CF92DF92EF92FF920F931F9381
:10F5C000CF93DF9300D01F92CDB7DEB75C017A8373
:10F5D00069834A01170107FD07C0802F002E000C28
:10F5E000990B9C838B8304C0E1E0F0E0FC83EB8308
:10F5F000F90140805180628073808B819C81880FEB
:10F60000991F880F991F9C838B838957984F7C0182
:10F61000A3019201FC0160817181828193810E942A
:10F6200056E6882391F0F70140825182628273820C
:10F6300011E020E030E0A901C301B2010E94C8EC52
:10F6400018160CF010E0F5011083F501808182306E
:10F65000D1F0833009F45EC0813009F07CC0EB81C9
:10F66000FC81E957F84F2081318142815381F401B7
:10F6700060817181828193810E9456E687FD6BC013
:10F6800082E0F50180838B819C818957984F9C8310
:10F690008B83B60180E090E00E945AE69B01AC01AA
:10F6A000EB81FC8160817181828193810E94A1EA5A
:10F6B0009B01AC01F40160817181828193810E9480
:10F6C000C8EC87FD14C00E94F1586B017C019101C8
:10F6D000A8EEB3E00E9492EAC60ED71EE81EF91EFD
:10F6E000E981FA81C082D182E282F38234C00E9431
:10F6F000F158E981FA81C080D180E280F380DC0199
:10F70000CB018C199D09AE09BF09B7FD24C083E068
:10F71000F50180830F3F19F044EA5CE102C047EB3A
:10F720005CE16BEC7CE1802F0F900F900F900F90BD
:10F73000DF91CF911F910F91FF90EF90DF90CF90CD
:10F74000BF90AF909F908F907F906F905F904F9001
:10F750003F902F9076CD0F900F900F900F90DF91EC
:10F76000CF911F910F91FF90EF90DF90CF90BF90BE
:10F77000AF909F908F907F906F905F904F903F9051
:10F780002F9008954F925F926F927F928F929F92E7
:10F79000AF92BF92CF92DF92EF92FF920F931F939F
:10F7A000CF93DF93CDB7DEB760970FB6F894DEBF87
:10F7B0000FBECDBF80914907811117C060960FB66B
:10F7C000F894DEBF0FBECDBFDF91CF911F910F9197
:10F7D000FF90EF90DF90CF90BF90AF909F908F9071
:10F7E0007F906F905F904F900895DFDB0E94F158FB
:10F7F0004B015C0160914A0470914B04072E000C90
:10F80000880B990B0E945CE669837A838B839C83C7
:10F8100044E1C42ED12C5CE3E52EF12C00E09E01E6
:10F820002F5F3F4F4CE454E067E777E086E797E0CF
:10F83000B7DEC0904C04D0904D04E0904E04F090A0
:10F840004F046091340570913505072E000C880B2C
:10F85000990B0E945CE69B01AC01C701B6010E94B6
:10F86000C8EC18160CF009C160911E0270911F02BD
:10F87000072E000C880B990B0E945CE69B01AC01E3
:10F88000C701B6010E9456E687FFF7C000914A04FF
:10F8900010914B04B801012E000C880B990B0E94AB
:10F8A0005CE6A70196010E94A1EA2B013C0120ED34
:10F8B0003CEC4CE45DE3609140077091410780911E
:10F8C0004207909143070E94BBE66D837E838F833E
:10F8D000988720916D0730916E0740916F07509186
:10F8E0007007C701B6010E94A1EA9B01AC016D81BE
:10F8F0007E818F8198850E94BBE66D837E838F8396
:10F90000988723E333E343E75FE3609169077091EE
:10F910006A0780916B0790916C070E94BBE69B0180
:10F92000AC016D817E818F8198850E94A2EA6D83F2
:10F930007E838F8398876093690770936A078093AB
:10F940006B0790936C07C0926D07D0926E07E092A0
:10F950006F07F092700720E030E040E251E4C3010D
:10F96000B2010E94C8EC18160CF431C220E030E05D
:10F9700040E251ECC301B2010E9456E687FD2FC25E
:10F98000012B09F42CC28091680781112CC22091AF
:10F990006407309165074091660750916707298792
:10F9A0003A874B875C8720913C0730913D07409117
:10F9B0003E0750913F07C301B2010E94BBE66B01B5
:10F9C0007C01A301920169857A858B859C850E94C3
:10F9D000A2EA69877A878B879C8760936407709314
:10F9E00065078093660790936707209138073091E9
:10F9F000390740913A0750913B070E94BBE6A701A7
:10FA000096010E94A2EA2D813E814F8158850E9475
:10FA1000A1EA6B017C0120E030E04FE753E40E9453
:10FA2000C8EC20E030E0A90118160CF4E3C1C701CE
:10FA3000B6010E9456E687FD07C0C701B6010E94C5
:10FA4000E6EB759567951AC020E030E0A901C30187
:10FA5000B2010E9456E687FF10C0A301920169859A
:10FA60007A858B859C850E94A1EA609364077093D8
:10FA70006507809366079093670760E060934C0783
:10FA800080917B0790917C07A0917D07B0917E07C4
:10FA90000097A105B10521F1A5019401281B390B9F
:10FAA0004A0B5B0B57FD1CC060917F07709180076C
:10FAB00080E090E00E945AE69B01AC0160914C040A
:10FAC00070914D0480914E0490914F040E9456E62F
:10FAD00087FF82C143E85BE165E97BE180E0B1DB60
:10FAE0008091440790914507A0914607B091470740
:10FAF000A5019401281B390B4A0B5B0B57FD0FC066
:10FB000073DAD501C4018C53964FAF4FBF4F80932A
:10FB1000440790934507A0934607B0934707809109
:10FB2000810790918207A0918307B0918407009785
:10FB3000A105B10511F1881A990AAA0ABB0AB7FCF6
:10FB40001CC0609185077091860780E090E00E945C
:10FB50005AE69B01AC016091460470914704809184
:10FB60004804909149040E9456E687FF20C141E66F
:10FB70005BE164E77BE18FEF64DB609144047091AB
:10FB80004504072E000C880B990B0E945CE66983E4
:10FB90007A838B839C8395E0C92ED12C24E1E22EBD
:10FBA000F12C0FEF9E012F5F3F4F46E454E061E7D9
:10FBB00077E085E797E0F4DCC0904604D0904704F6
:10FBC000E0904804F090490420E030E040EA50E43E
:10FBD000C701B6010E94C8EC87FDE5C020E030E017
:10FBE0004CED52E4C701B6010E9456E618160CF41B
:10FBF000DAC06091440470914504072E000C880B14
:10FC0000990B0E945CE6A70196010E94A1EA4B01B4
:10FC10005C012091340730913507409136075091AF
:10FC200037070E94BBE669877A878B879C8720917C
:10FC30006007309161074091620750916307C501E9
:10FC4000B4010E94A2EA6D837E838F8398876093BC
:10FC50006007709361078093620790936307209118
:10FC600030073091310740913207509133070E949D
:10FC7000BBE66D877E878F87988B20ED3CEC4CE44C
:10FC80005DE360912C0770912D0780912E07909174
:10FC90002F070E94BBE62B013C0120915C073091AD
:10FCA0005D0740915E0750915F07C701B6010E9452
:10FCB000A1EA9B01AC01C301B2010E94BBE62B018A
:10FCC0003C0123E333E343E75FE36091580770911E
:10FCD000590780915A0790915B070E94BBE69B01F0
:10FCE000AC01C301B2010E94A2EA2B013C01609366
:10FCF00058077093590780935A0790935B07C092F7
:10FD00005C07D0925D07E0925E07F0925F072D8559
:10FD10003E854F85588969857A858B859C850E94AB
:10FD2000A2EAA30192010E94A1EA6B017C0120E0FA
:10FD300030E04FE753E40E94C8EC20E030E0A90136
:10FD40001816C4F5C501B4010E94C8EC181684F455
:10FD5000A50194016D817E818F8198850E94A1EA21
:10FD600060936007709361078093620790936307C5
:10FD70006FE71AC020E030E0A901C501B4010E947C
:10FD800056E687FF10C0A50194016D817E818F81A9
:10FD900098850E94A1EA6093600770936107809341
:10FDA00062079093630760E060934D0707CD0E9460
:10FDB000A976E3CEC701B6010E9456E687FDDACFE9
:10FDC000C701B6010E94E6EB75956795EDCF81E01E
:10FDD000809368076FE752CE80E007D881CE81E03C
:10FDE000809368074ACE1092680719861A861B8688
:10FDF0001C86D9CDC301B2010E94C8EC181654F775
:10FE0000A301920169857A858B859C850E94A1EA70
:10FE10006093640770936507809366079093670704
:10FE20006FE72CCE90916F00292F227091FF05C0B3
:10FE300090916F009D7F90936F0034E0839FC0018D
:10FE40001124FC01EE57FF4E408151816281738184
:10FE5000FC01E55EF84F408351836283738381E048
:10FE600080931A07222329F080916F00826080938B
:10FE70006F000895BC012091180730911907409137
:10FE80001807509119072417350711F09A01F7CF79
:10FE900081E02617370709F080E008958F929F923E
:10FEA000AF92BF92CF92DF92EF92FF921F93CF93C8
:10FEB000DF93C82F83ED9BE09093AF098093AE0949
:10FEC0001092EF0B82E090E0A0E0B0E08093D80BBE
:10FED0009093D90BA093DA0BB093DB0B1092AD0982
:10FEE0001092A9091092AA091092AB091092AC09BC
:10FEF0008FEF9FEFDC018093A5099093A609A09353
:10FF0000A709B093A809CC2379F1C53008F0F8C04F
:10FF100040E060E070E0CB010E94BAD1882309F490
:10FF2000EFC020E1C29FC00111248B56984FFC0105
:10FF3000E254FE4F20812F7709F0E2C03C964081C9
:10FF4000518162817381443651056105710508F460
:10FF5000D7C03497C080D180E280F380C114D1042F
:10FF6000E104F10421F4CCC0C12CD12C760140E095
:10FF7000C701B6010E94BAD1182F882309F4C0C066
:10FF80008091B0079091B1078115924009F0B8C0F7
:10FF9000A091B507AA2309F4B3C06091B30770918B
:10FFA000B4076115710509F4ABC02091B207222393
:10FFB00009F4A6C0A093EA0B2093DC0B80E030E0AC
:10FFC00041E050E0C82FFA01082E02C0EE0FFF1FDB
:10FFD0000A94E2F72E173F0739F08F5FC83091F788
:10FFE00089E08093E50B8CC08093E50B2091BB07E3
:10FFF0003091BC072115310519F040E050E008C0F0
:020000021000EC
:100000002091C9073091CA074091CB075091CC0786
:100010002093DD0B3093DE0B4093DF0B5093E00B0E
:1000200046015701860E971EA11CB11C8092EB0B56
:100030009092EC0BA092ED0BB092EE0BE091B60714
:10004000F091B707F093F10BE093F00BB0E00E9452
:1000500082EA860E971EA81EB91E8092F20B90921D
:10006000F30BA092F40BB092F50B85E0EE0FFF1F9F
:100070008A95E1F7E150FE4FEF2FFF27E6958E0EB0
:100080009F1EA11CB11C8092E60B9092E70BA092E0
:10009000E80BB092E90B2091B8073091B907211510
:1000A000310521F0A90160E070E008C04091C5076A
:1000B0005091C6076091C7077091C807D701C60164
:1000C00088199909AA09BB09840F951FA61FB71F94
:1000D00004C0B695A79597958795CA95D2F7809352
:1000E000E10B9093E20BA093E30BB093E40B853FFD
:1000F0002FE09207A105B10528F48CE08093EF0B67
:1001000010E01AC0853F9F4FA105B10510F480E1B2
:1001100011C08091D1079091D207A091D307B091DF
:10012000D4078093F20B9093F30BA093F40BB0934E
:10013000F50B80E28093EF0B812FDF91CF911F9120
:10014000FF90EF90DF90CF90BF90AF909F908F90F7
:100150000895682F8AE99FE00C94D34ACF92DF92EA
:10016000EF92FF921F93CF93DF931092320A809108
:10017000650A882321F082E69AE00E94FB9810929B
:10018000D70B1092D40B85E38093D30B0E94F158C8
:10019000EB01A89561E08091D30B0E9429B683ED15
:1001A0009BE00E945C9A2398229A219A209A289A8E
:1001B00085E08093D50B82E58CBD1DBC1AE08FEFE6
:1001C0000E94619A1150D9F720E030E0A90160E067
:1001D00083ED9BE00E94669A182F8093D60B8130A6
:1001E00049F00E94F1586C1B7D0B613D774060F334
:1001F00081E054C02AEA31E040E050E068E083ED5D
:100200009BE00E94669A82FF03C01093D70B0EC03A
:1002100014E00E94749F8093D60B1150D1F78A3A54
:1002200011F082E03BC082E08093D70B8091D70B26
:10023000823021F0C12CD12C760105C0C12CD12CEB
:10024000E12C80E4F82E20E030E0A90167E383EDA3
:100250009BE00E94669AA701960169E283ED9BE00C
:100260000E94669A8093D60B882349F00E94F15829
:100270006C1B7D0B613D774030F38AE00FC08091AD
:10028000D70B823011F520E030E0A9016AE383ED5D
:100290009BE00E94669A882351F088E08093D40BFB
:1002A00083ED9BE00E945C9AE4EEFDE119C00E94A0
:1002B000749F807C803C19F483E08093D70B0E946C
:1002C000749F0E94749F0E94749F83ED9BE00E9424
:1002D0005C9A1092D50B81E0E1DD811131C015C02F
:1002E0008491EF012196882321F00E94E093FE0182
:1002F000F7CFE6EDFDE18491EF012196882309F423
:1003000056C00E94E093FE01F6CF80E0C7DD811168
:1003100017C0EFECFDE18491EF012196882321F0D5
:100320000E94E093FE01F7CFEBEBFDE18491EF013A
:100330002196882309F43BC00E94E093FE01F6CF8A
:1003400068ED7BE082E69AE00E94A898811116C0D1
:10035000EFECFDE18491EF012196882321F00E94CA
:10036000E093FE01F7CFEAEAFDE18491EF012196E7
:100370008823E9F00E94E093FE01F7CF81E08093AB
:10038000320AE4EEFDE18491EF012196882321F009
:100390000E94E093FE01F7CFEEE9FDE18491EF01C9
:1003A0002196882321F00E94E093FE01F7CF8BE194
:1003B000E2E6FAE0A1E8BAE001900D928A95E1F751
:1003C0008091600A9091610A9093800A80937F0ADD
:1003D000DF91CF911F91FF90EF90DF90CF90089524
:1003E00080913F0E823041F489E89DE19093A4070B
:1003F0008093A3070E940C940E94F1586093430ECF
:100400007093440E8093450E9093460E8091320A6D
:10041000882319F081E08093310A81E080933F0EB8
:100420000895CF93DF931092310A83E080933F0EBB
:1004300080918C0E8823B1F0E1E8FDE18491EF0119
:10044000882341F0082E000C990B83DE2196FE01D3
:100450008491F6CF8DE090E07CDE8AE090E0DF9141
:10046000CF9177CEE5E8FDE18491EF01882391F308
:10047000082E000C990B6DDE2196FE018491F6CFBB
:100480008F929F92AF92BF92CF92DF92EF92FF92A4
:100490000F931F93CF93DF9300D01F92CDB7DEB79A
:1004A000FC018381813079F5818181FF2CC08189B4
:1004B0009289A389B489892B8A2B8B2B09F448C094
:1004C0007F0140E050E0BA01CF010E9411988823DB
:1004D000D1F0F70185889688A788B08CC18CD28C22
:1004E00082E090E0A0E0B0E0F60180839183A283F7
:1004F000B3839E012F5F3F4FB501A401C6010E9447
:1005000083D2811102C080E03CC000E010E098017D
:10051000B501A401C6010E94F2D18823A1F389800C
:100520009A80AB80BC80F6018789803141F4F8EF76
:100530008F16FFEF9F06A104B10460F4DACF88EFB5
:1005400088168FEF9806A8068FE0B80618F4D1CF6A
:1005500081E017C0F701158A168A178A108E118A52
:10056000128A138A148A818180688183C7010E945C
:10057000D1D3882341F240E050E0BA01C7010E9484
:1005800011980F900F900F900F90DF91CF911F91C6
:100590000F91FF90EF90DF90CF90BF90AF909F9022
:1005A0008F9008951092340A1092310A8091FD0BB9
:1005B000882321F08AEF9BE00C94FB9808952F92FA
:1005C0003F924F925F926F927F928F929F92AF92E3
:1005D000BF92CF92DF92EF92FF920F931F93CF9330
:1005E000DF93CDB7DEB7C257D1090FB6F894DEBF9F
:1005F0000FBECDBF8C013B014A014DB75EB7E196FE
:100600005FAF4EAFE197AD961FAEAD971B0154E0C3
:10061000250E311C7E018FE5E80EF11C9DEE492E62
:1006200092E0592EE0E4F0E0EC0FFD1F3496E396E3
:10063000FFAFEEAFE397F3018781823008F462C128
:1006400084859585A685B7858F719927AA27BB27AD
:10065000892B8A2B8B2B09F055C11092420A42E458
:100660005AE0BE016F5F7F4FC1010E9469D3181627
:100670000CF048C18C85982F9871903129F4209105
:10068000AF0C2150223078F42981222309F43AC199
:10069000253E89F22E3279F22091420A2E3259F209
:1006A0008A7049F6B8C04DB75EB7AF965FAF4EAF30
:1006B000AF97BE016F5F7F4FC7010E9464D10115E4
:1006C000110521F0F801808181119BC021E081E0BA
:1006D00090E0F70101900020E9F73197EE19FF094A
:1006E0008E0F9F1F02964DB75EB7481B590B0FB672
:1006F000F8945EBF0FBE4DBF8DB79EB701965C01EB
:10070000211102C0B80102C062E273E0C5010E947B
:1007100006EEB701C5010E94E7ED62E273E0C50194
:100720000E94E7ED25961FAE259728961FAE2897C5
:1007300024961FAE1EAE249722965FAE4EAE229731
:1007400021E0A701B101E3968EAD9FADE3970E9432
:10075000879E81112AC08091AF0C811126C0E4EEE2
:10076000FDE184916F019FEFC91AD90A882321F016
:100770000E94E093F601F5CFEDE6FDE184916F0173
:100780002FEFC21AD20A882321F00E94E093F601CB
:10079000F5CF6701F60181916F01882319F00E945E
:1007A000E093F8CF8AE00E94E0938BE1FE01EC5BDE
:1007B000FF4FDE01959601900D928A95E1F7249600
:1007C0008EAD9FAD24979CA38BA35AA249A240E073
:1007D00050E0BE016F5D7F4FC501F1DECE01819615
:1007E0000E94B4A0CE01805C9F4F0E94B4A0AF963F
:1007F0004EAD5FADAF970FB6F8945EBF0FBE4DBF65
:100800001ACFF80101900020E9F73197CF01801B42
:10081000910B20E05ECF81E0903109F080E0809381
:10082000330A903141F08985873409F004CF8A85F5
:100830008E3709F400CF8091AF0C813029F08230DF
:10084000D9F18111F8CE0AC08091B00C9091B10C11
:1008500001969093B10C8093B00CEDCEBE016F5F0A
:100860007F4F85E39AE00E9464D10115110529F4B8
:1008700085E3C82E8AE0D82E09C06801F60181916F
:100880006F018823A9F30E94E093F8CFF6018191CC
:100890006F01882319F00E94E093F8CF80E20E9454
:1008A000E0936D8D7E8D8F8D98A14AE00E94019717
:1008B0008AE00E94E093BFCEBE016F5F7F4F85E369
:1008C0009AE00E9464D18114910441F065E37AE0DA
:1008D000C4010E94D4ED892B69F414C0AD96FFAD1C
:1008E000AD978F2F90E02091BC0F3091BD0F8217F4
:1008F000930741F0AD962FADAD972F5FAD962FAF1B
:10090000AD9799CEE1968EAD9FADE1970FB6F89475
:100910009EBF0FBE8DBFCE58DF4F0FB6F894DEBF1F
:100920000FBECDBFDF91CF911F910F91FF90EF9040
:10093000DF90CF90BF90AF909F908F907F906F90FF
:100940005F904F903F902F9008950F931F93CF93F8
:10095000DF93CDB7DEB76F970FB6F894DEBF0FBE4B
:10096000CDBF8B0122E02093AF0C9093BD0F8093FD
:10097000BC0F81E89AE00E94589A8BE1E1E8FAE026
:10098000DE01159601900D928A95E1F780917F0A1C
:100990009091800A9C838B838DEE92E09A83898369
:1009A000A801BE016F5F7F4F80E090E008DECE01BE
:1009B00001960E94B4A06F960FB6F894DEBF0FBEEA
:1009C000CDBFDF91CF911F910F9108952F923F924C
:1009D0004F925F926F927F928F929F92AF92BF924F
:1009E000CF92DF92EF92FF920F931F93CF93DF93FB
:1009F000CDB7DEB76F970FB6F894DEBF0FBECDBF91
:100A00006C012DB63EB61D8218861C821B828DEEAF
:100A100092E09A838983FB0180819E012F5F3F4F83
:100A200039018F3241F08DE79AE0F601918380839E
:100A3000F62E172F64C08EE59AE0F601918380832D
:100A40008B010F5F1F4F0115110509F456C04DB6FC
:100A50005EB66FE270E0C8010E94F2ED4C0108172B
:100A6000190708F048C07C01E01AF10AFF24C70109
:100A700001962DB73EB7281B390B0FB6F8943EBF31
:100A80000FBE2DBF8DB79EB701965C01A701B801BF
:100A90000E941BEEF501EE0DFF1D1082F601608134
:100AA00071816115710511F06C5F7F4F21E0A50127
:100AB000CE0105960E94879E811111C0B50189E57E
:100AC0009DE10E9486C58EE20E94E0938AE00E942A
:100AD000E0930FB6F8945EBE0FBE4DBE0EC0F60199
:100AE0007182608284010F5F1F4F0FB6F8945EBE63
:100AF0000FBE4DBEA8CFF02E02C0F12C10E0C301F6
:100B00000E94B4A08F2D912F0FB6F8943EBE0FBE59
:100B10002DBE6F960FB6F894DEBF0FBECDBFDF912E
:100B2000CF911F910F91FF90EF90DF90CF90BF90EA
:100B3000AF909F908F907F906F905F904F903F907D
:100B40002F900895CF92DF92EF92FF920F931F9311
:100B5000CF93DF9388E50E94414CD82E89E40E9410
:100B6000414CC82E882319F00E94DA4B1CC0DD20AE
:100B7000C1F00E940A4C20E030E040E251E40E94C3
:100B8000A1EA20E030E048EC51E40E94A2EA2AE029
:100B900037ED43EA5CE30E94BBE60E94E6EB65307A
:100BA00010F01FEF01C0162F89E50E94414C082F5D
:100BB0008AE40E94414CC82F882319F00E94DA4B26
:100BC0001CC00023C1F00E940A4C20E030E040E24B
:100BD00051E40E94A1EA20E030E048EC51E40E9498
:100BE000A2EA2AE037ED43EA5CE30E94BBE60E94FA
:100BF000E6EB653010F0DFEF01C0D62F8AE50E94EA
:100C0000414CE82E811105C081E50E94414CF82E2F
:100C100001C0F12CC11001C0C0E02C2F30E0D11078
:100C200001C000E0200F311D2130310521F4E11019
:100C30001AC0F11018C0EFECFDE18491EF0121968C
:100C4000811103C0E5E9F0E204C00E94E093FE01D7
:100C5000F4CF8491EF012196882309F455C00E94B6
:100C6000E093FE01F6CF17FD02C0D7FF17C0EFECEF
:100C7000FDE18491EF012196811103C0E6E7F0E2E6
:100C800004C00E94E093FE01F4CF8491EF0121960D
:100C90008823D1F10E94E093FE01F7CF0E940A4C15
:100CA0009B01AC01012F110F110BAD2FDD0FBB0B01
:100CB000FF2099F085E0809FF001819FF00D1124C5
:100CC000EA0FFB1FEE0FFF1FEE0FFF1FEA53FF4E51
:100CD000608171818281938103C060E070E0CB010B
:100CE000E5E0E09FE001E19FD00D1124CA0FDB1F7A
:100CF000CC0FDD1FCC0FDD1FCA53DF4E0E94A2EACE
:100D0000688379838A839B83DF91CF911F910F91B1
:100D1000FF90EF90DF90CF90089580916F00982F13
:100D2000927081FF05C080916F008D7F80936F006E
:100D30008091B4098093B3098093B2098093B1097B
:100D400084E68093B00928EE33E030934B0720937C
:100D50004A07992329F080916F00826080936F0089
:100D600081E080931A070E94116A0E94C2C9809193
:100D70007C10882321F084EA98E10E947EC68CE0F2
:100D8000E4EAF8E1A2E3B4E001900D928A95E1F77C
:100D90000C9494932F923F924F925F926F927F9216
:100DA0008F929F92AF92BF92CF92DF92EF92FF927B
:100DB0000F931F93CF93DF93CDB7DEB7CD54D109F7
:100DC0000FB6F894DEBF0FBECDBF85E40E948A4CFB
:100DD000882321F00E94DA4B7B0102C0E12CF12C28
:100DE00083E40E948A4C882321F00E94DA4B6AA394
:100DF00002C005E00AA385E50E948A4C882319F009
:100E00000E94FB4B03C085E50E94414C8CA7F7FC78
:100E100007C0812C912C16E1A12E13E4B12E06C03F
:100E2000812C912CBCE8AB2EB2E4BB2E83E50E9452
:100E30008A4C882321F00E940A4C4B015C01E1148A
:100E4000F10411F410924E0710923F10ED820E94AF
:100E5000F1582B013C011D8117FF05C00CE310E088
:100E600022E0298304C003E210E035E03983D30196
:100E7000C2018C53964FAF4FBF4F8093440790935E
:100E80004507A0934607B093470761E06E0D6230B7
:100E900080F0E3EEFFE184918F010F5F1F4F1A8313
:100EA0000983882309F45FC30E94E093E981FA81F2
:100EB000F2CFEDE0F0E284917F012FEFE21AF20A27
:100EC000882321F00E94E093F701F5CF0E94027978
:100ED0003D8137FF04C08FE780934D0708C04D81E7
:100EE000E42F440FFF0BE45BF84F8FE78083C501CD
:100EF000B4010E94E6EB072E000C880B990B0E94B0
:100F00005CE66A877B878C879D878981482F50E0C4
:100F10009801A8EEB3E00E9492EA6DA77EA78FA782
:100F200098AB8B019C01040D151D261D371D0AAFC2
:100F30001BAF2CAF3DAF81E0809320021D811F3F8E
:100F400039F40DE41FE11FAF0EAF07E11FE106C04A
:100F50000BE31FE11FAF0EAF04E01FE122961FAFAE
:100F60000EAF22974CA25DA26EA27FA249AA5AAAF6
:100F70006BAA7CAA1DAA1EAA1FAA18AE19AE188EAB
:100F800010E4198F0CE10A8F16E41B8F1C8E1D8E46
:100F90001E8E1F8E1C8A1D8A1E8A1F8A188A198A15
:100FA0001A8A1B8A19821A821B821C828FE790E0A0
:100FB000A0E0B0E08E839F83A887B987FFE7CF2E9C
:100FC000D12CE12CF12C18A619A61AA61BA611E00B
:100FD0001F861E862D961FAE2D97212C312C2E9606
:100FE0001FAE2E970D81802F000F990B9C01245B63
:100FF000384F24963FAF2EAF2497880F991F880F44
:10100000991FDC01A45BBB4FB9A3A8A3CA01052E9D
:10101000000CAA0BBB0B28968CAF9DAFAEAFBFAF39
:1010200028974C5F5F4FCA01550FAA0BBB0B2C963C
:101030008CAF9DAFAEAFBFAF2C97AAA10A2E000C0C
:10104000BB0BBBA3AAA380912002882309F489C209
:101050000E94F1584B015C0180914907882309F4F3
:10106000D4C00E94D5770D8107FD0CC0A8A1B9A1FD
:10107000BC912D96BFAF2D97E8A1F9A121803280B8
:1010800003810BC0009146042D960FAF2D97209041
:10109000470430904804009149042E960FAF2E97D4
:1010A0002D962FAD2D97322D432D2E965FAD2E9779
:1010B0006C8D7D8D8E8D9F8D0E9456E687FF0AC0B8
:1010C0002D960FAD2D970C8F2D8E3E8E2E960FAD3B
:1010D0002E970F8F288D398D4A8D5B8D2D966FAD94
:1010E0002D97722D832D2E969FAD2E970E9456E63A
:1010F00087FF0AC02D960FAD2D97088F298E3A8E47
:101100002E960FAD2E970B8F809144079091450737
:10111000A0914607B0914707A5019401281B390B00
:101120004A0B5B0B57FD10C00E94F477D501C40138
:101130008C53964FAF4FBF4F809344079093450712
:10114000A0934607B09347072D962FAD2D97322DCC
:10115000432D2E965FAD2E976A857B858C859D8568
:101160001123E9F10E9456E687FF4FC0B501A401A3
:101170004419550966097709DB01CA01885893416A
:10118000A109B109B7FD41C0D701C6010E811F8178
:1011900028853985801B910BA20BB30B1D81B5955A
:1011A000A7959795879517FF03C080934D0705C0B6
:1011B0002496EEADFFAD2497808348A759A76AA770
:1011C0007BA70A850C8F1B851D8F0C850E8F1D85B7
:1011D0001F8F8CA29DA2AEA2BFA210E016C00E94DB
:1011E000C8EC181694F4D501C4012CA13DA14EA160
:1011F0005FA1821B930BA40BB50BAC01BD0148583A
:1012000053416109710977FFCBC120E030E040EA2A
:1012100051E46A857B858C859D850E94A2EA2D9686
:101220002FAD2D97322D432D2E965FAD2E970E9418
:1012300056E687FF10C0EFE6FFE184918F010F5F54
:101240001F4F1A830983882309F48BC10E94E093FE
:10125000E981FA81F2CFD501C40129A93AA94BA9A4
:101260005CA9821B930BA40BB50BB7FD96C00E9423
:10127000EF758AE00E94E093D501C4018053984F36
:10128000AF4FBF4F89AB9AABABABBCAB0DA9011154
:1012900063C02EA93FA948AD59AD2D966FAD2D97CE
:1012A000722D832D2E969FAD2E970E94C8EC181696
:1012B0000CF041C028966CAD7DAD8EAD9FAD2897EA
:1012C0000E945CE62D962FAD2D97322D432D2E9644
:1012D0005FAD2E970E94A2EA6EAB7FAB88AF99AF4D
:1012E0002DA53EA54FA558A9280D391D4A1D5B1DEA
:1012F0002AAF3BAF4CAF5DAF2C966CAD7DAD8EADE4
:101300009FAD2C970E945CE69B01AC016A857B85B2
:101310008C859D850E94A1EA2D962FAD2D97322DAB
:10132000432D2E965FAD2E970E9456E6881F882784
:10133000881F8DAB32C0D501C4012AAD3BAD4CAD89
:101340005DAD821B930BA40BB50BB7FD26C04EAD54
:101350005FAD60E67FE11EC020E030E040EA51E48E
:101360006A857B858C859D850E94A1EA9B01AC01E5
:101370002D966FAD2D97722D832D2E969FAD2E97A6
:101380000E9456E687FF09C022964EAD5FAD2297B8
:101390006BE27FE18D810E942179D501C401880F24
:1013A000991FAA1FBB1F2CA13DA14EA15FA1821BAB
:1013B000930BA40BB50B84199509A609B7098138BD
:1013C0009F44A241B10580F0E6EEFEE184918F01D9
:1013D0000F5F1F4F1A830983882309F4C2C00E943C
:1013E000E093E981FA81F2CF2AA13BA14E855F8586
:1013F000241735070CF027CEE9E8FEE184918F0130
:101400000F5F1F4F1F830E83882329F00E94E093F4
:10141000EE81FF81F3CF1D8117FD03C006E113E0CC
:1014200002C000EF13E01F830E836E817F8188E787
:101430009EE10E9486C549815A816B817C8184E747
:101440009EE10E9450C58AE00E94E0936E817F81F8
:1014500083E69EE10E9486C5488959896A897B890D
:101460008FE59EE10E9450C58AE00E94E0936E8164
:101470007F818EE49EE10E9486C54C895D896E89DC
:101480007F898AE49EE10E9450C58AE00E94E09331
:101490001CA5112309F467C00D8107FF31C0298104
:1014A0003A814B815C812093340730933507409318
:1014B0003607509337072CEA35EC47E25EE368893C
:1014C00079898A899B890E94BBE660933007709373
:1014D000310780933207909333072CEA35EC47E2CB
:1014E0005EE36C897D898E899F890E947EEB609383
:1014F0002C0770932D0780932E0790932F0733C0EE
:1015000089819A81AB81BC8180933C0790933D0790
:10151000A0933E07B0933F072CEA35EC47E25EE329
:10152000688979898A899B890E94BBE6609338071C
:101530007093390780933A0790933B072CEA35EC78
:1015400047E25EE36C897D898E899F890E947EEBEC
:10155000609340077093410780934207909343073D
:1015600002C00E94027981E080933F10C35BDF4F8D
:101570000FB6F894DEBF0FBECDBFDF91CF911F91A4
:101580000F91FF90EF90DF90CF90BF90AF909F9022
:101590008F907F906F905F904F903F902F90089525
:1015A0000E851F85012B09F42BC148A459A46AA4F8
:1015B0007BA4480E591E6A1E7B1E28A539A54AA584
:1015C0005BA5281B390B4A0B5B0B6E817F818885DD
:1015D00099850E9435EAA30192010E9466EADA0128
:1015E000C9018C0D9D1DAE1DBF1D84319105A10546
:1015F000B105FCF06C017D018C3E9105A105B105A2
:101600002CF05BEEC52ED12CE12CF12C20E8C2167B
:10161000D104E104F104DCF08EEF90E0A0E0B0E052
:101620008C199D09AE09BF098E839F83A887B9874E
:1016300012C044E1C42ED12CE12CF12C04E110E0C5
:1016400020E030E00E831F832887398704C0CE82D4
:10165000DF82E886F986EBEDFFE184918F010F5F71
:101660001F4F882321F00E94E093F801F6CFC701B5
:10167000B6010E946C97E6EDFFE184918F010F5F48
:101680001F4F882321F00E94E093F801F6CF6E816E
:101690007F81888599850E946C97488D598D6A8DC8
:1016A0007B8D8FEC9FE10E9450C54C8D5D8D6E8DC2
:1016B0007F8D88EC9FE10E9450C50E851F85033009
:1016C00011050CF49DC06E817F81888599850E94EB
:1016D0005CE620E030E040E850E40E94BBE669832D
:1016E0007A838B839C83288D398D4A8D5B8D6C8D9D
:1016F0007D8D8E8D9F8D0E94A1EA2BED3FE049E408
:1017000050E40E94BBE620E030E040E05FE30E944E
:10171000BBE69B01AC0169817A818B819C810E942F
:101720007EEB69837A838B839C83C301B2010E9421
:101730005CE62FE632E143E85AE30E94BBE62B0168
:101740003C0149815A816B817C8182EC9FE10E943E
:1017500050C5B301A2018CEB9FE10E9450C52AE95C
:1017600039E949E15FE369817A818B819C810E943B
:10177000BBE669837A838B839C839B01AC010E94C7
:10178000A2EAA30192010E947EEB688B798B8A8B7F
:101790009B8B29813A814B815C81C301B2010E94FC
:1017A000BBE620E030E040E05EE30E94BBE66C8BED
:1017B0007D8B8E8B9F8BECEAFFE184918F010F5F15
:1017C0001F4F882319F0FCD7F801F7CF49815A81C0
:1017D0006B817C8186EA9FE10E9450C548895989C6
:1017E0006A897B8980EA9FE10E9450C54C895D89A6
:1017F0006E897F898AE99FE10E9450C58AE0E0D71F
:101800008E819F81A885B9858C0D9D1DAE1DBF1D44
:101810001D81B595A7959795879517FF03C0809370
:101820004D0705C02496EEADFFAD249780830E854D
:101830001F850F5F1F4F1F870E871A85188F0B8517
:10184000098F1C851A8F0D850B8F2401350111E03E
:10185000DCCCCF93DF93E4EEFDE18491EF012196A0
:10186000882319F0ADD7FE01F8CF83E50E94414CE3
:10187000882321F00E94FB4B80935202EAE3FEE1B1
:101880008491EF012196882319F09AD7FE01F8CFB1
:1018900080915202811103C0E6E3FEE102C0E2E35F
:1018A000FEE18491EF012196882319F089D7FE018A
:1018B000F8CFEAE2FEE18491EF012196882319F046
:1018C0007FD7FE01F8CF2091140430911504409188
:1018D000160450911704609198187091991880918E
:1018E0009A1890919B180E94A2EAAB01BC0188E271
:1018F0009EE10E9450C52091180430911904409136
:101900001A0450911B0460919C1870919D1880914D
:101910009E1890919F180E94A2EAAB01BC0185E23B
:101920009EE10E9450C520911C0430911D044091FD
:101930001E0450911F046091A0187091A11880910D
:10194000A2189091A3180E94A2EAAB01BC0182E206
:101950009EE10E9450C5EAE1FEE18491EF012196EB
:10196000882319F02DD7FE01F8CF2091140430916F
:10197000150440911604509117046091460270912D
:10198000470280914802909149020E94A2EAAB016D
:10199000BC0188E19EE10E9450C52091180430915D
:1019A000190440911A0450911B0460914A027091ED
:1019B0004B0280914C0290914D020E94A2EAAB0131
:1019C000BC0185E19EE10E9450C520911C0430912C
:1019D0001D0440911E0450911F0460914E027091AD
:1019E0004F0280915002909151020E94A2EAAB01F5
:1019F000BC0182E19EE10E9450C58AE0DF91CF9157
:101A0000DFC6FF920F931F93CF93DF93F82E092F1A
:101A1000162FEDE0FEE18491EF012196882319F065
:101A2000CFD6FE01F8CFEF2DF02F8491EF01219654
:101A3000882319F0C5D6FE01F8CFEBE0FEE18491D2
:101A4000EF012196882319F0BBD6FE01F8CF612F54
:101A500070E080E090E00E946C978AE0DF91CF9187
:101A60001F910F91FF90ACC64F925F926F927F9241
:101A70008F929F92AF92BF92CF92DF92EF92FF929E
:101A8000CF93DF93209114043091150440911604F4
:101A900050911704609132047091330480913404A2
:101AA000909135040E94A2EAAB01BC0188E09EE15E
:101AB0000E9450C5209118043091190440911A04D5
:101AC00050911B0460913604709137048091380462
:101AD000909139040E94A2EAAB01BC0184E09EE12E
:101AE0000E9450C520911C0430911D0440911E0499
:101AF00050911F0460913A0470913B0480913C0422
:101B000090913D040E94A2EAAB01BC0180E09EE1FD
:101B10000E9450C540913E0450913F0460914004A2
:101B2000709141048CEF9DE10E9450C580916F003F
:101B3000982F927081FF05C080916F008D7F8093F8
:101B40006F004090821050908310609084107090CD
:101B500085108090861090908710A0908810B0908B
:101B60008910C0908A10D0908B10E0908C10F0906B
:101B70008D10992329F080916F00826080936F000F
:101B8000E2EFFDE18491EF012196882319F018D648
:101B9000FE01F8CFC301B2010E946C97EEEEFDE1A9
:101BA0008491EF012196882319F00AD6FE01F8CF1F
:101BB000C501B4010E946C97EAEEFDE18491EF014A
:101BC0002196882319F0FCD5FE01F8CFC701B60194
:101BD0000E946C978AE0DF91CF91FF90EF90DF90A9
:101BE000CF90BF90AF909F908F907F906F905F90BD
:101BF0004F90E6C52F923F924F925F926F927F92E5
:101C00008F929F92AF92BF92CF92DF92EF92FF920C
